:020000040800F2
:10000000000001204D410008D1270008D327000837
:10001000D5270008D7270008D927000800000000CE
:10002000000000000000000000000000DB270008C6
:10003000DD27000800000000DF270008E127000896
:100040009D4100089D410008E52700089D410008EA
:100050009D4100089D410008F1270008F72700088E
:100060009D4100089D410008292800089D41000885
:10007000FD270008FF270008012800080D280008B8
:1000800019280008252800089D4100089D41000806
:10009000000000009D4100082B2800089D41000839
:1000A0009D4100089D4100089D4100089D410008B8
:1000B0009D4100089D4100089D4100089D410008A8
:1000C0009D4100089D4100089D4100089D41000898
:1000D0009D410008352800089D4100089D41000809
:1000E0009D41000831280008412800089D41000872
:1000F0009D41000800000000000000009D41000834
:100100009D4100089D4100084D2800089D410008C0
:100110009D4100089D4100089D4100089D41000847
:100120009D4100089D4100089D4100089D41000837
:080130009D4100089D410008FB
:1001380010B5054C237833B9044B13B10448AFF319
:1001480000800123237010BDCC08002000000000AF
:10015800D83C010808B5034B1BB103490348AFF36A
:10016800008008BD00000000D0080020D83C01082D
:1001780014214160704714207047406A704700009E
:10018800790100087F01000883010008990100082F
:1001980010B5044604F1100000F05CFCC4F8F80047
:1001A8000148C4F87C0110BD88010008F8B5E6B024
:1001B80004460D4616461F460A4906A800F0CAFE20
:1001C80070996F9A05910492009733466E996D9ACB
:1001D800039102922A466C990191214600F060F839
:1001E80067B0F0BD94010008F8B5E6B004460D46C6
:1001F80016461F46094906A800F0ACFE6F996E9A8C
:100208000491039200976D996C9A0291019233467A
:100218002A46214600F087F867B0F0BD940100082F
:1002280038B500281CBF01680029184A23D1184B8B
:100238001C684FF6F0710C404CF24025AC421FBFD1
:100248001B6819404CF27024A14212D1114D296843
:1002580079B911490B68C3F30B03B3F58A6F1FBF54
:100268000968C1F30B0140F28343994204BF01219D
:10027800117028B905E0094B994204BF012111709A
:100288004068BDE8324001F09FBE00BFE80800208A
:1002980000ED00E0002004E00010005C000037489A
:1002A8002DE9F04104460D46216816464A681F4666
:1002B80090478046B8F5403F2ED122680A99936846
:1002C800204698478046B8F5403F25D12368089ACC
:1002D8000799D3F80CC02046E0478046B8F5403F60
:1002E8001AD12368069A39461F692046B8478046BE
:1002F800B8F5403F10D1236829465D69324620464B
:10030800A8478046B8F5403F06D123680B9A09995B
:100318009D692046A847804621680A68204690477C
:100328004046BDE8F0812DE9F04104460D462168BC
:1003380016464A681F4690478046B8F5403F2ED17A
:1003480022680A999368204698478046B8F5403F46
:1003580025D12368089A0799D3F80CC02046E047AE
:100368008046B8F5403F1AD12368069A39461F6976
:100378002046B8478046B8F5403F10D12368294643
:100388005D6932462046A8478046B8F5403F06D109
:1003980023680999DD6900222046A847804621681C
:1003A8000A68204690474046BDE8F0814FF4403047
:1003B80070470000F0B50C4685B0114600281A4673
:1003C8001CBF0568002D0B4B11D082B104B971B95F
:1003D8000D9860B10F9E0E9F0A9B0290049603979A
:1003E8000B980C9E009001962046A8470346184695
:1003F80005B0F0BD020003002DE9F04F0646D0B06D
:100408000868F56DD6F860E0726EB76EF36E00BAE4
:1004180000906C46486800BA60600DF14008886832
:1004280000BAA060C86800BAE060086900BA206134
:10043800486900BA6061886900BAA061C86900BAF1
:10044800E061086A00BA2062486A00BA6062886A95
:1004580000BAA062C86A00BAE062086B00BA2063FA
:10046800486B00BA6063886B00BAA063C86B00BAB7
:10047800E063402058F80C1C58F820CC58F838ACE9
:100488008CEA010158F840CC8AEA01018CEA01099A
:100498004FEAF979401E48F8049BEBD187EA02003D
:1004A80000EA0E00784010EBF5610098DFF824C4EC
:1004B80041186144C81882EABE032B404FEAF06134
:1004C80053405918636859186144CF194FEAB50366
:1004D80083EABE01014081EABE0111EBF765A1681C
:1004E8004D196544A91883EAB0023A404FEAF1650C
:1004F8005A405519E26855194FEAB70282EAB0071F
:1005080065440F4005EBBE0E97EAB00717EBFE6592
:1005180027697D194FEAB10782EA0701654401EAB4
:100528000E01EB18514011EBF36561694D194FEA63
:10053800BE0187EA010E65440EEA030E15EBB00012
:100548008EEA070E0EEBF065D4F818E075446544A2
:10055800AA1881EAB30505404FEAF26E4D40AE4451
:10056800E569AE44E64477444FEAB00080EAB30E4A
:100578000EEA020E8EEAB30E0EEBF765D4F820E011
:1005880075446544691880EAB2053D404FEAF16E4A
:100598004540AE44656AAE44E6440EEBB3034FEA09
:1005A800B70787EAB20E0EEA010E8EEAB20E0EEB1C
:1005B800F365D4F828E075446544281887EAB1053E
:1005C8001D404FEAF06E7D40AE44E56AAE44E64415
:1005D8000EEBB2024FEAB30383EAB10E0EEA000E45
:1005E8008EEAB10E0EEBF265D4F830E0754465443E
:1005F800EF1983EAB00515404FEAF76E5D40AE4447
:10060800656BAE44E6440EEBB1014FEAB20282EAF2
:10061800B00E0EEA070E8EEAB00E0EEBF165D4F8B6
:1006280038E075446544EB1882EAB7050D404FEA97
:10063800F36E5540AE44E56BAE44E6440EEBB000B5
:100648004FEAB10181EAB70E0EEA030E8EEAB70E41
:100658000EEBF065D4F840E07544654481EAB30ECA
:10066800AA180EEA000E4FEAF2658EEA010E7544EA
:10067800DDF844E04FEAB000754480EAB30E654403
:100688000EEA020E15EBB7078EEAB30E0EEBF7650E
:10069800DDF848E04FEAB202754480EA020E65448C
:1006A8000EEA070E69188EEA000E0EEBF165DDF80A
:1006B8004CE07544654405EBB3034FEAB70E1427C5
:1006C8000DF1500CDFF810528EEA010B82EA0B0B89
:1006D8000BEBF36A5CF804BBDA44AA44504483EA9F
:1006E800B10B4FEAF06A8EEA0B0BDA445CF804BBF4
:1006F800DA44AA44524480EAB30B4FEAF26A8BEA1E
:10070800B10BDA445CF804BBDA444FEAB000AA44FF
:1007180080EA020BD6448BEAB30B0BEBFE6A5CF85B
:1007280004BBDA444FEAB202AA4482EA0E0B0AEB8F
:10073800B10180EA0B0B0BEBF16A5CF804BBDA44FD
:100748007F1DAA44282F0AEBB3034FEABE0EBBD382
:100758003C2F61D3502F4DD204EB870CC7F15407BF
:100768005E4CA7FB04A504465D4FA8088EEA010A63
:1007780082EA0A0A5CF804BB0AEBF3655D447D195A
:100788002C1983EAB10A4FEAF4658EEA0A0A55443D
:100798005CF804AB5CF804BB55447D19AA1884EADC
:1007A800B30A4FEAF2658AEAB10A55445D444FEA52
:1007B800B4047D1984EA020AAE448AEAB30A0AEB51
:1007C800FE655CF804AB55444FEAB2027D1982EA33
:1007D8000E0A15EBB10184EA0A0A5CF804BB0AEBBD
:1007E800F1655D447D1915EBB303401E4FEABE0E5B
:1007F800BCD12046F46D1B19F365336EC9183166F8
:10080800716E71447166B36ED218B266F16E40189B
:10081800F06650B0BDE8F08F4EEA010B0EEA010A0F
:100828000BEA020B4BEA0A0A0AEBF36554F827A015
:10083800DFF8B0C0554443EAB10B654403EAB10A96
:100848000BEA0E0B28184BEA0A0A7F1C0AEBF06524
:1008580054F827A0554440EAB30B654400EAB30AAC
:100868000BEAB10BAA184BEA0A0A7F1C0AEBF265DD
:1008780054F827A055444FEAB00040EA020B6544FB
:1008880000EA020A0BEAB30BAE444BEA0A0A7F1CE1
:100898000AEBFE6554F827A055444FEAB20242EA33
:1008A8000E0B654402EA0E0A0BEA000B15EBB101C8
:1008B8004BEA0A0A7F1C0AEBF16554F827A0554455
:1008C8007F1C65443C2F05EBB3034FEABE0EA3D350
:1008D80040E700BF9979825AA1EBD96ECDCCCCCC38
:1008E800D6C162CADCBC1B8F00B581B00168074A5B
:1008F800914200D110B9064801B000BD7C2113F027
:1009080051F94FF4003001B000BD00BFFC090008E8
:10091800030002002DE9F0410B4A92E8F85188B033
:10092800694681E8F8510268084B9A4200D118B923
:10093800074808B0BDE8F0811422083000F04FFBEA
:1009480008B0BDE8F08100BFDC090008FC09000818
:1009580003000200152904D20268044B9A4200D110
:1009680008B903487047083000F048BBFC09000884
:100978000300020010B481B013460268074CA2427B
:1009880000D118B901B010BC0548704701B000F19A
:10099800240210BC083000F035BB00BFFC09000879
:1009A8000300020010B481B013460268074CA2424B
:1009B80000D118B901B010BC054870470A4601B00B
:1009C80000F1240110BC083000F070BBFC090008DD
:1009D800030002000123456789ABCDEFFEDCBA981E
:1009E80076543210F0E1D2C300000000000000008D
:1009F80000000000F10800081D0900085D09000852
:100A08007D090008AD09000801040008790F0008F5
:100A1800C50F0008810F0008F0B5A3B004460B48C5
:100A280002900D4616461F46094B0822402104A88D
:100A380000F0D1FA28980190009733462A462146BB
:100A480002A800F01BF823B0F0BD00BFFC090008A5
:100A5800100A000810B5040008BF002408D0054893
:100A6800054B20600822402104F1080000F0B3FA89
:100A7800204610BDFC090008100A00082DE9F041C5
:100A880004460E46216817464A681D469047804628
:100A9800B8F5003F19D1226806999368204698470F
:100AA8008046B8F5003F10D123683146DE683A46E3
:100AB8002046B0478046B8F5003F06D12368079A1C
:100AC80029461D692046A847804621680A682046AD
:100AD80090474046BDE8F08110B500F033FA4FF476
:100AE800403400280EBF034C4FF4C07113F05AF87D
:100AF800204610BD0200030010B5044600F022FA9B
:100B080008B9054810BD0021A160D0F87C21116802
:100B180088474FF4403010BD0200030070B504460A
:100B28000D4600F00FFA064E40B1D0F87C0141683E
:100B38008847A84224BF65604FF44036304670BDF0
:100B4800020003002DE9FF4715000C4600D02CB128
:100B5800064600F0F7F95FEA000801D16448C3E0EF
:100B6800D8F8F80001684A689047B0F5003F17D1F7
:100B7800D8F87C118A68404690478146B9F1810FC0
:100B880080F09E80A94508F1FC0A17D2D8F8F80031
:100B98000368D3F80CC02A462146E047B0F5003F69
:100BA80040F08E80D8F8F8000368D3F810C06A4681
:100BB8005146E047B0F5003F76D10AE0002004E056
:100BC800215C0AF800100098401C00900098A84288
:100BD800F6D34FF0000C4749474A484B01AC009800
:100BE800844558D2D3E9007001ADC5E9007010788A
:100BF80000281ABF042086464FF0000E085854F803
:100C08000E5028443E4D05600127D0F800E087606B
:100C1800019D4F681AF80C007D408EEA050585F0A5
:100C2800040E65680F687D4085F0FC05754485F005
:100C3800A30568400AF80C000CF1010CCFE7D3E9D2
:100C4800004501A8C0E9004510782E4D002814BFC2
:100C58004FF0040E4FF0000E01A8744651F80EE054
:100C68000459A6440127CEF80050DEF80040CEF81B
:100C780008704D68019F40687D406C400D68684071
:100C880084F0040480F0FC00041984F057040AF886
:100C98000C400CF1010CCC45D1D3D8F8F800016810
:100CA8004A689047B0F5003F0AD1D8F8F8000368C1
:100CB800D3F80C804A465146C047B0F5003F01D0F2
:100CC800114811E0002006E05AF8201081F06A313E
:100CD8004AF82010401CB0EB990FF5D3B06840F0EB
:100CE8000100B0604FF4403004B0BDE8F08700BFA9
:100CF80002000300443D0108E8080020240F000812
:100D0800ADBE4ED70DBE75A10100030038B50C4627
:100D1800017A1546CA0702D500F014F908B908483F
:100D280032BDD0F8F80003682146DC682A46A0479F
:100D3800B0F5003F01D0034832BD4FF4403032BD1A
:100D480002000300010003002DE9F84191B00546B7
:100D58000E461746402101A812F024FF297AC80739
:100D680004D5284600F0EEF8040002D1DFF8A4808C
:100D78004BE0D4F8F800DFF8A0800368D3F810C07F
:100D88006A4601A9E047B0F5003F3ED1D4F8F80023
:100D980001684A689047B0F5003F36D1D4F87C1115
:100DA8008A6820469047D4F8F830024618461B68EF
:100DB800D3F80CC004F1FC01E047B0F5003F24D1A2
:100DC800D4F87C0141688847D4F8F83002461846C0
:100DD8001B68D3F80CC001A9E047B0F5003F14D157
:100DE800D4F8F8000268696893689847B0F5003F3E
:100DF8000BD1D4F8F80003681C693A463146A0477D
:100E0800B0F5003F08BF4FF44038404612B0BDE887
:100E1800F08100BF02000300010003002DE9F84142
:100E2800A5B0074688461646402115A812F0BAFE16
:100E380000220492402105A812F0B4FE387AC107B6
:100E48005ED5384600F07EF8050059D0D5F8F80090
:100E58002D4C0368D3F810C06A4605A9E047B0F5E1
:100E6800003F3CD1D5F8F80001684A689047B0F5D2
:100E7800003F34D1D5F87C118A6828469047D5F8C8
:100E8800F830024618461B68D3F80CC005F1FC017F
:100E9800E047B0F5003F22D1D5F87C01416888478A
:100EA800D5F8F830024618461B68D3F80CC005A9D7
:100EB800E047B0F5003F12D1D5F8F800026879682C
:100EC80093689847B0F5003F09D1D5F8F800036852
:100ED8001D6904AA15A9A847B0F5003F01D020460E
:100EE8000FE00A4B0A490B4A0396029101924046C9
:100EF8001C68049B009415AA796800F0E5F900E0E5
:100F0800054826B0BDE8F081010003004C3D01080A
:100F1800936E030026C703000200030004B001011A
:100F280000170145E10A0008010B0008250B00081D
:100F3800B50300084D0B0008150D0008510D0008F9
:100F4800250E00080168024A914218BF0020704728
:100F58002C0F000810B5040008BF002404D0034873
:100F68002060204609688847204610BD2C0F0008DD
:100F780020225C3012F014BEF0B58468A308002269
:100F880004F0030407E000F15C0555F8226035BA67
:100F980041F82250521C9A42F5D300220BE000F18E
:100FA8005C0502EB830755F82360D500C5F11805E9
:100FB800EE40CE55521CA242F1D3F0BD30B5C46804
:100FC80003690022E31AD5188C5C0544521C082AD0
:100FD8002C77F8D330BD0360C1600261704738B523
:100FE800044615460022626023685A68904700202C
:100FF8006061A061A5604FF4003032BD81604FF49C
:10100800003070472DE9F84304462079D4F80C8065
:10101800450748BF244845D466691D46A8F1010024
:1010280000EAD60306EBC506B6EBC50F666102D229
:10103800A669761CA6611746A66906EB5576A661D1
:101048000E46E918884225D2A8EB03094A463146DC
:10105800F81812F0A5FD2268136839460FE04246D9
:10106800384612F09DFD23681A6839462046904795
:1010780007E0311811F00300F1D122681368204607
:101088009847484600EB0809A9F10101A942F0D3A5
:10109800002300E000202A1A3118F81812F080FD09
:1010A8004FF40030BDE8F283040002002DE9FC4F44
:1010B800024685B0D0681369DFF86CC1DFF86C812F
:1010C800A0EB030A506840F004005060002703A812
:1010D80002900DF10C0ED8E9003403A8544DC0E974
:1010E80000342878534D00280CBF00230423994668
:1010F8005CF803305EF80940234401261D601C6833
:101108009E60DCF80430039DDCF80090DEF8046093
:101118005D406540484C654089EA0606474C664094
:101128007519474C6540D8E9006B03AC0028C4E941
:10113800006B0EBF002404200424029E5CF800000B
:10114800345920183F4C04600126046886600398CF
:10115800029E43406340384C7068634089EA00004F
:10116800364C6040034438484340280018BF0120EB
:101178005B1E9B41042F2CBFC0B2D80F02F1140391
:1011880053F8200007F00303C3F10303DB00D84042
:101198000DF807007F1C082F9DD315460C466A6979
:1011A800AB69E868D20842EA4372401E00EA0207C7
:1011B800002302409B420AD8524508D28020E055BD
:1011C8007F1C574516D2AAEB0701E01910E08020D2
:1011D800E05500E0E355E8687F1C8742FAD32A68A7
:1011E800136828469847BAF1000F03D051462046A5
:1011F80012F0D8FC2A68069E059F9368694628461F
:1012080098472A68D2F8009021462846C8472B6894
:10121800DA683946284690470EB1A86830604FF41E
:10122800003007B0BDE8F08F443D010854120008B3
:10123800E80800205FC5109304850012FC68017A55
:10124800C0F524FF24AF33D426AF698B04B0010165
:1012580000170145F8B501240094002300240DE08F
:10126800009D065D0F5D7E40F643761CF60F86F006
:10127800010635400095641C009DEB189442EFD39D
:101288001846F2BDF8B5002301240094002A11E0A5
:10129800009C85188F1815F8016C17F8015C6E40D2
:1012A800F643761CF60F86F0010634400094009C45
:1012B800E318521EECD11846F2BD00005D1200087A
:1012C8008D120008010000002DE9F84F1D46DDF8D9
:1012D80028900B9F0D9C4FF0FF3300930E469246CB
:1012E800D9F800B0804632465146D847834664B3A1
:1012F800D9F8043032465146404698476FEA0B0207
:10130800521C42EA0B0200996FEAD2735B1C194027
:10131800C2430091521C024300996FEAD2735B1CCE
:101328001940009186F05531484087EA000181F064
:101338005531216080F05531C943491C0843009A52
:101348006FEAD070401C82430092D9F80800012847
:1013580009D17540E943491C0D4300986FEAD572DD
:10136800521C90430AE0F11C85EA9102D243521CB8
:10137800154300986FEAD5735B1C984386F0AA362C
:10138800009086EA0B0686F0AA33F243DB430C98FA
:10139800C2F3C0725B1C42EAD3720099D243521C5A
:1013A80091430091774000998843009987F0AA37C4
:1013B8000F403843BDE8F28F034613F8012B002A8B
:1013C800FBD1181A0138704781F0004102E000BFD4
:1013D80083F0004330B54FEA41044FEA430594EAED
:1013E800050F08BF90EA020F1FBF54EA000C55EA28
:1013F800020C7FEA645C7FEA655C00F0E2804FEAF9
:101408005454D4EB5555B8BF6D420CDD2C4480EADA
:10141800020281EA030382EA000083EA010180EA0A
:10142800020281EA0303362D88BF30BD11F0004F58
:101438004FEA01314FF4801C4CEA113102D040428E
:1014480061EB410113F0004F4FEA03334CEA1333C9
:1014580002D0524263EB430394EA050F00F0A780E1
:10146800A4F10104D5F1200E0DDB02FA0EFC22FADC
:1014780005F2801841F1000103FA0EF2801843FAD0
:1014880005F359410EE0A5F120050EF1200E012AC1
:1014980003FA0EFC28BF4CF0020C43FA05F3C018FF
:1014A80051EBE37101F0004507D54FF0000EDCF178
:1014B800000C7EEB00006EEB0101B1F5801F1BD321
:1014C800B1F5001F0CD349085FEA30004FEA3C0C25
:1014D80004F101044FEA445212F5800F80F09A801B
:1014E800BCF1004F08BF5FEA500C50F1000041EB1F
:1014F800045141EA050130BD5FEA4C0C404141EB23
:101508000101013C28BFB1F5801FE9D291F0000F1D
:1015180004BF01460020B1FA81F308BF2033A3F1CC
:101528000B03B3F120020CDA0C3208DD02F1140CC3
:10153800C2F10C0201FA0CF021FA02F10CE002F1FE
:101548001402D8BFC2F1200C01FA02F120FA0CFCF7
:10155800DCBF41EA0C019040E41AA2BF01EB045140
:10156800294330BD6FEA04041F3C1CDA0C340EDC3E
:1015780004F11404C4F1200220FA04F001FA02F381
:1015880040EA030021FA04F345EA030130BDC4F13F
:101598000C04C4F1200220FA02F001FA04F340EA34
:1015A8000300294630BD21FA04F0294630BD94F0E5
:1015B800000F83F4801306BF81F480110134013DCC
:1015C8004EE77FEA645C18BF7FEA655C29D094EA3D
:1015D800050F08BF90EA020F05D054EA000C04BFBB
:1015E8001946104630BD91EA030F1EBF00210020A6
:1015F80030BD5FEA545C05D14000494128BF41F045
:10160800004130BD14F580043CBF01F5801130BDA8
:1016180001F0004545F0FE4141F470014FF0000033
:1016280030BD7FEA645C1ABF194610467FEA655CE4
:101638001CBF0B46024650EA013406BF52EA033586
:1016480091EA030F41F4002130BD00BF90F0000F74
:1016580004BF0021704730B54FF4806404F13204B0
:101668004FF000054FF0000150E700BF90F0000F69
:1016780004BF0021704730B54FF4806404F1320490
:1016880010F0004548BF40424FF000013EE700BF60
:1016980042004FEAE2014FEA31014FEA02701FBFF0
:1016A80012F07F4393F07F4F81F06051704732F022
:1016B8007F4208BF704793F07F4F04BF41F4002179
:1016C800704730B54FF4607401F0004521F00041D7
:1016D8001CE700BF50EA010208BF704730B54FF061
:1016E80000050AE050EA010208BF704730B511F062
:1016F800004502D5404261EB41014FF4806404F19A
:1017080032045FEA915C3FF4D8AE4FF003025FEA1F
:10171800DC0C18BF03325FEADC0C18BF033202EBA3
:10172800DC02C2F1200300FA03FC20FA02F001FAFD
:1017380003FE40EA0E0021FA02F11444BDE600BFA0
:101748004FF0FF3C06E000BF4FF0010C02E000BF85
:101758004FF0010C4DF804CD4FEA410C7FEA6C5C68
:101768004FEA430C18BF7FEA6C5C1BD001B050EA0B
:10177800410C0CBF52EA430C91EA030F02BF90EAF6
:10178800020F0020704710F1000F91EA030F58BFB5
:10179800994208BF90422CBFD8176FEAE37040F017
:1017A800010070474FEA410C7FEA6C5C02D150EAB5
:1017B800013C07D14FEA430C7FEA6C5CD6D152EA70
:1017C800033CD3D05DF8040B704700BF8446104635
:1017D80062468C461946634600E000BF01B5FFF734
:1017E800B7FF002848BF10F1000F01BD4DF808ED04
:1017F800FFF7F4FF0CBF012000205DF808FB00BFD5
:101808004DF808EDFFF7EAFF34BF012000205DF82E
:1018180008FB00BF4DF808EDFFF7E0FF94BF01207B
:1018280000205DF808FB00BF4DF808EDFFF7CEFF7C
:1018380094BF012000205DF808FB00BF4DF808EDBB
:10184800FFF7C4FF34BF012000205DF808FB00BF8C
:101858004FEA410212F5001215D211D56FF47873D0
:10186800B3EB625212D94FEAC12343F0004343EA73
:10187800505311F0004F23FA02F018BF404270474E
:101888004FF00000704750EA013005D111F00040D8
:1018980008BF6FF0004070474FF00000704700BF6E
:1018A80080F0004002E000BF81F0004142001FBF0D
:1018B8005FEA410392EA030F7FEA226C7FEA236C16
:1018C8006AD04FEA1262D2EB1363C1BFD21841400B
:1018D80048404140B8BF5B42192B88BF704710F0A1
:1018E800004F40F4000020F07F4018BF404211F044
:1018F800004F41F4000121F07F4118BF494292EAAC
:10190800030F3FD0A2F1010241FA03FC10EB0C00D7
:10191800C3F1200301FA03F100F0004302D5494264
:1019280060EB4000B0F5000F13D3B0F1807F06D311
:1019380040084FEA310102F10102FE2A51D2B1F109
:10194800004F40EBC25008BF20F0010040EA0300FE
:101958007047490040EB0000013A28BFB0F5000F7E
:10196800EDD2B0FA80FCACF1080CB2EB0C0200FA34
:101978000CF0AABF00EBC25052421843BCBFD04083
:101988001843704792F0000F81F4000106BF80F4FD
:1019980000000132013BB5E74FEA41037FEA226CC0
:1019A80018BF7FEA236C21D092EA030F04D092F08B
:1019B800000F08BF0846704790EA010F1CBF0020BF
:1019C800704712F07F4F04D1400028BF40F000401C
:1019D800704712F100723CBF00F50000704700F03C
:1019E800004343F0FE4040F4000070477FEA226263
:1019F80016BF08467FEA23630146420206BF5FEA34
:101A0800412390EA010F40F4800070474FF0000333
:101A180004E000BF10F0004348BF40425FEA000CFA
:101A280008BF704743F0964301464FF000001CE0A2
:101A380050EA010208BF70474FF000030AE000BFF8
:101A480050EA010208BF704711F0004302D5404236
:101A580061EB41015FEA010C02BF844601460020A8
:101A680043F0B64308BFA3F18053A3F50003BCFAC3
:101A78008CF2083AA3EBC25310DB01FA02FC634470
:101A880000FA02FCC2F12002BCF1004F20FA02F277
:101A980043EB020008BF20F00100704702F120026A
:101AA80001FA02FCC2F1200250EA4C0021FA02F2CB
:101AB80043EB020008BF20EADC7070474FEA40029F
:101AC800B2F1FE4F0FD34FF09E03B3EB12620DD964
:101AD8004FEA002343F0004310F0004F23FA02F0CE
:101AE80018BF404270474FF00000704712F1610F75
:101AF80001D1420205D110F0004008BF6FF000404C
:101B080070474FF00000704753B94AB9002908BF21
:101B180000281CBF4FF0FF314FF0FF3000F070B9C4
:101B2800ADF1080C6DE904CE00F006F8DDF804E02C
:101B3800DDE9022304B070472DE9F047089E0D4601
:101B480004460F46002B4AD18A42944665D9B2FA18
:101B580082F343B102FA03FCC3F120029F4020FA4A
:101B680002F217439C404FEA1C4E1FFA8CF5B7FB54
:101B7800FEF1220C0EFB117742EA074201FB05F049
:101B880090420AD91CEB020201F1FF3780F01B8159
:101B9800904240F2188102396244121AA4B2B2FB90
:101BA800FEF00EFB102244EA024400FB05F5A542B4
:101BB8000AD91CEB040400F1FF3280F00681A5422B
:101BC80040F203816444023840EA0140641B00216A
:101BD8001EB1DC400023C6E90043BDE8F0878B4214
:101BE80008D9002E00F0EC800021C6E9000508465F
:101BF800BDE8F087B3FA83F1002949D1AB4202D39B
:101C0800824200F2F780841A65EB0302012017462E
:101C1800002EE2D0C6E90047DFE702B9FFDEB2FADC
:101C280082F3002B40F08F808A1A4FEA1C471FFA74
:101C38008CFE0121B2FBF7F507FB1520220C42EAC6
:101C480000420EFB05F0904208D91CEB020205F198
:101C5800FF3802D2904200F2CA804546121AA4B256
:101C6800B2FBF7F007FB102244EA02440EFB00FE29
:101C7800A64508D91CEB040400F1FF3202D2A645A0
:101C880000F2BA801046A4EB0E0440EA05409FE734
:101C9800C1F120078B4022FA07FC4CEA030C05FA35
:101CA80001F420FA07F3FD40234300FA01F94FEA53
:101CB8001C401FFA8CFEB5FBF0F81C0C00FB1855F5
:101CC80044EA054408FB0EF5A54202FA01F20BD9D5
:101CD8001CEB040408F1FF3A80F08780A54240F22B
:101CE8008480A8F102086444641B9DB2B4FBF0F33D
:101CF80000FB134445EA044403FB0EFEA64508D93D
:101D08001CEB040403F1FF306BD2A64569D9023BF2
:101D1800644443EA0840A0FB0283A4EB0E049C42FF
:101D2800C6461D4655D352D056B1B9EB0E0364EBE7
:101D3800050404FA07F7CB40CC401F43C6E90074FA
:101D48000021BDE8F087C3F1200102FA03FC20FA64
:101D580001F225FA01F19D402A434FEA1C471FFA78
:101D68008CFEB1FBF7F007FB1015110C41EA054199
:101D780000FB0EF58D4204FA03F408D91CEB0101AF
:101D880000F1FF382FD28D422DD902386144491B0A
:101D980092B2B1FBF7F507FB151142EA014205FBC8
:101DA8000EF1914208D91CEB020205F1FF3816D258
:101DB800914214D9023D6244521A45EA004139E77A
:101DC8003146304609E73946E7E61046FCE6C145A4
:101DD800AAD2B8EB020E63EB0C050138A4E745461E
:101DE800EAE7034695E74046D1E7D0467CE7023D5F
:101DF800624433E708460BE76444023843E700BF10
:101E0800704700BF1348144A08B54FF00043C0E9B3
:101E180000230422002342610122C2614FF4805151
:101E280007220383C0E90233C0E90933C0E90C1271
:101E38000361837680F8203080F82C30826380F844
:101E48003C30C36404F092FF18B1BDE8084000F0CC
:101E580017BC08BDEC080020002401400268084BAC
:101E68009A4282B00AD14FF0B0431A6E42F400721F
:101E78001A661B6E03F400730193019B02B070474E
:101E8800002401400268054B9A4201BF4FF0B0425E
:101E9800136E23F400731366704700BF00240140DB
:101EA80030B585B000240546CDE901440394FFF719
:101EB800A9FF144805F0F2FA08B100F0E1FB114857
:101EC800039401A9CDE9015405F0AEF808B100F07A
:101ED800D7FB0C4805F00CFA08B100F0D1FB4FF025
:101EE800FF31084805F042F8064805F0B9FA0548F8
:101EF80005F096F80446034805F05CFA204605B05C
:101F080030BD00BFEC080020014B024A1A60704740
:101F1800EC0800200024014008B50948FFF7C0FF7D
:101F280068B1084BB3F8AA304FF6FF72934216BF58
:101F380040F6E442044B5343B3FBF0F398B208BDB8
:101F4800002000B40075FF1FD8084C0013B500230B
:101F5800ADF80630FFF7E0FF04461948FFF7A0FF89
:101F6800184BB3F8C820B3F8A8108A4204FB00F055
:101F780018D040F6E443B0FBF3F364205B1A434304
:101F8800521A93FBF2F31E331BB2ADF80630BDF8BC
:101F980006305BB21B02ADF80630BDF8060000B291
:101FA80002B010BD4FF47A7240F6FF73B0FBF3F342
:101FB8005343A3F53923A3F50C6340F6C412E0E7B5
:101FC800001000B00075FF1F4FF0B04382B09A6A4E
:101FD80022F480529A629A6C42F480529A649B6C02
:101FE80003F480530193019B002002B070474FF027
:101FF800B04382B09A6C02439A649B6C034001938D
:10200800019B02B0704708B50420FFF7F0FF0120DC
:10201800FFF7EDFF0220FFF7EAFF002211460B2031
:1020280005F0DAFA0B2005F009FB002211460C2016
:1020380005F0D2FA0C2005F001FB002211460D2014
:1020480005F0CAFA0D2005F0F9FA002211460E2013
:1020580005F0C2FA0E2005F0F1FA002211460F2011
:1020680005F0BAFA0F2005F0E9FA0022114610200F
:1020780005F0B2FA102005F0E1FA0022114611200D
:1020880005F0AAFA112005F0D9FA002236201146E7
:1020980005F0A2FABDE80840362005F0CFBA0000E6
:1020A80008B505F013FD10B16FF0040008BD064B2C
:1020B8009A6942F040429A614CF2FA321A6105F08C
:1020C80017FD0028F2D0EFE700400058F0B585B0C2
:1020D80000230C4600930646A8B3FFF7E1FF054628
:1020E80070BB05F0F3FC88BB1A481B4A0223019316
:1020F800D0F8E01506F1784302EA8121B3FBF1F745
:1021080001FB1733DB0A0293D0F8E00504F17841AC
:102118000139314402EA8022B1FBF2F002FB1011CE
:10212800C3EBD1230133694601A8039305F060FD91
:1021380020B102280CBF01256FF0010505F0D8FC7D
:10214800284605B0F0BD6FF00505F9E76FF0040506
:10215800F6E700BF0070FF1F00FCFF03014B18608B
:1021680000207047500900202DE9F04F89B0B0F1E8
:10217800006F06460F460092C0F0C580DFF89881D0
:10218800664DD8F8E03505EA832303F10063013B87
:10219800984200F2B880002800F0B880002900F0CA
:1021A800B58040EA02035B0740F0B080FFF778FF94
:1021B8000446A0BB05F08AFC002840F0AA80D8F8A5
:1021C800E01506F1784205EA8121B2FBF1F301FB43
:1021D8001322009B03F17843013B3344B3FBF1F036
:1021E80001FB1033DB0A01334FEAD22AA3EBD222D8
:1021F800012A039388BFC6F30A050AF58038C6F199
:10220800080398BF009D069388BFC5F500654FEA8F
:10221800C828B346039B9A4505D305F069FC2046B8
:1022280009B0BDE8F08FA6F10803069A1A44954252
:1022380019D804950197CDF814B04FF00009059B03
:1022480009EB0301049B99453ED3009BAB442F4403
:102258005D1BB5F5006F28BF4FF400650AF1010A50
:1022680008F50068D6E753F8081F5A68B2F1FF3F2F
:1022780008BFB1F1FF3FD8D0294B186810B96FF0EB
:102288000504CAE7B8F1000F04D04FF400624146D4
:1022980011F01AF8DFF88890D9F80030CBF30A006B
:1022A80039461844AAB211F00FF84FF400614046BD
:1022B800FFF70CFF08BBD9F8003001934FF4006317
:1022C800CDF814800493B8E7019B07914B4402931F
:1022D8000120D3E9002305F045FC88B90799019B43
:1022E800D1E9000259F80310029B5B689A4208BFC3
:1022F800884205D109F10809A1E76FF001048CE7CC
:102308006FF0030489E74FF0FF3488E76FF00504A6
:1023180085E76FF0040482E70070FF1F00FCFF03ED
:1023280050090020B1F1006F70B511D30B4BD3F8F1
:10233800E0650B4B03EA862303F10063013B9942F6
:1023480006D840B139B192B210F0BEFF002070BD7E
:102358004FF0FF30FBE76FF00500F8E70070FF1F54
:1023680000FCFF03B0F1006F10B40DD3084BD3F895
:10237800E045084B03EA842303F10063013B9842DC
:1023880002D810BCFFF7A2BE4FF0FF3010BC704758
:102398000070FF1F00FCFF034FF0B04382B0DA6CFF
:1023A8000243DA64DB6C03400193019B02B070477F
:1023B80070B586B01422002101A811F0BDFB0120E0
:1023C800FFF7EAFF0220FFF7E7FF0420FFF7E4FF2B
:1023D8004FF4007101224FF0904005F07DFD01257A
:1023E80002234FF4041401A94FF09040CDE90134C1
:1023F800224E039505F04AFC4FF4441301A94FF00F
:102408009040CDE90235019505F040FC2023CDE947
:10241800013401A900243046039405F037FC4FF439
:10242800007301A94FF09040CDE90135CDE903547F
:1024380005F02CFC04230DEB03013046CDE90135F2
:10244800CDE9034405F022FC22462146062005F08A
:10245800C3F8062005F0F2F822462146072005F0C9
:10246800BBF8072005F0EAF822462146162005F0B9
:10247800B3F8162005F0E2F806B070BD0004004875
:1024880008B51248124A134BC0E900230023012261
:10249800C0E90232C0E90433C0E90633036205F03B
:1024A8008FFE08B100F0ECF80848002106F008F8A3
:1024B80008B100F0E5F80548002106F027F818B142
:1024C800BDE8084000F0DCB808BD00BF140A0020D1
:1024D800005800405D3E302070B596B00546142285
:1024E800002103A811F028FB3822002108A811F0C8
:1024F80023FB2A68304B9A425BD18023089308A8B3
:102508004FF440230E9306F05DFD08B100F0B8F8D3
:102518004FF0B0444FF4C050E36C43F00103E36460
:10252800E36C03F001030293029B12230026CDE91A
:1025380003030323CDE905634FF09040042303A967
:10254800079305F0A3FBA36DDFF870C043F4800385
:10255800A365A36D1A4C03F480030193019B2662C3
:102568000D23C4E900C320468023C4E90266C4E9F8
:102578000436C4E9066605F0C1F808B100F080F831
:10258800104AEC63A562104C0E23C4E90023102105
:10259800002380222046C4E90213C4E90423C4E9C5
:1025A8000633236205F0AAF808B100F069F8AC63B5
:1025B800A56216B070BD00BF00580040440002403C
:1025C8005409002058000240B409002000B59BB00F
:1025D8004822002108A811F0AFFA1822002102A809
:1025E80011F0AAFA05F0B8FF4FF0B0420120D2F876
:1025F800903023F01803C2F89030D2F8003423F456
:10260800C06343F40073C2F80034D2F8003403F412
:10261800C0630193019B2423089381230B93002318
:10262800CDE91003B02208A8CDE9122306F00CF971
:1026380008B172B6FEE74F23CDE90230CDE90400B8
:10264800CDE90600022102A806F098FB08B172B68F
:10265800FEE71BB05DF804FB08B504F035FBFFF797
:10266800B5FFFFF7A5FEFFF7CEFCFFF709FF00F067
:10267800BEFD40F6B83000F03FFA00F0BFFDFCE7C1
:1026880072B6FEE700B58DB02C22002101A811F02A
:1026980053FA1748174B03601F2383604FF080429B
:1026A8000023C0E90433C0E9072383614FF4807332
:1026B800436206F00DFE08B1FFF7E2FF0C4806F092
:1026C80033FF08B1FFF7DCFF4FF0005300220793F8
:1026D800074808924FF4807301A9029206920B935F
:1026E80006F056FE08B1FFF7CBFF0DB05DF804FB0E
:1026F800680A00200028004010B5044690B038222F
:10270800002102A811F018FA2268194B9A422CD11C
:102718004FF48033029302A84FF480730F9306F0AE
:1027280051FC08B1FFF7ACFF4FF0B0430220D3F8DB
:10273800902042F40042C3F890209A6D42F48062DF
:102748009A659B6D002203F4806311460193019BF7
:1027580004F042FF022004F071FF00222A201146F3
:1027680004F03AFF2A2004F069FF10B010BD00BF42
:10277800002800407047000008B504F0BBFA044B7D
:102788000120C3F88800BDE8084005F03DBF00BF40
:102798000004005804F0B5BA08B504F0B2FA00F025
:1027A80059FCFFF705FEFFF72EFCBDE80840FFF7D0
:1027B80067BE08B504F09EFABDE808400121002074
:1027C80005F0D2BE70477047FEE7FEE7FEE7FEE77A
:1027D800FEE770477047704770470000014806F0F1
:1027E800C9BE00BF680A0020012005F07BBB02209B
:1027F80005F078BB70477047014805F0F9B800BF8D
:1028080054090020014805F0F3B800BF400B002030
:10281800014805F0EDB800BFE00A0020FFF7F2BF5D
:102828007047202005F05EBB70470000014807F0A4
:1028380065BA00BFA00B0020014806F0CDBC00BF60
:10284800680A0020014807F0C0B800BFCC0A002081
:102858002DE9F04389B080460020109E07908946F4
:1028680015461F46FDF7DCFCF0B9104CCDE9009089
:10287800CDE9020407AB0E480593142304933A46A6
:10288800434629460068FDF795FD2346324604F184
:10289800140153F8044B42F8044B8B42F9D1079BBF
:1028A800337509B0BDE8F0830120FAE7A00A0020DB
:1028B800403D01081FB50E4C00233C2202A8CDE97B
:1028C80002336275237500F0B9F8042303AA009453
:1028D80012210848FFF7BCFF07491422204611F0CF
:1028E8001BF9B0FA80F35B09637504B010BD00BF33
:1028F800B40A0020683D01084E0E0020054808B5BE
:102908000823036006F07CFE18B1BDE80840FFF715
:10291800B7BE08BDCC0A00204FF0B04307B55A6EC9
:1029280042F001025A665B6E002203F00103019334
:1029380011463220019B04F04FFE322003B05DF8AF
:1029480004EB04F07BBE00000CB407B5054A05ABE8
:102958001021019310F0C2FF03B05DF804EB02B040
:10296800704700BF7A3D010830B585B0044602A81B
:102978000D4610F0DFFDBDF90C30064A009310211A
:10298800029B2046FFF7E0FF2046FEF715FD288052
:1029980005B030BD7A3D01084FF0B04210B59368DC
:1029A80023F40043936010F04DFE0E4B01241C707D
:1029B80000F0B6F810F016FB0B4810F02DFB0B4B8F
:1029C8004FF400421A61204610F02CFBFFF79CFAE6
:1029D80000F012F910F022FC21462046BDE8104014
:1029E80010F03CBCD80A00207129000800400058AB
:1029F80010F04ABC08B5FFF78FFA40F6B833984292
:102A08000CD8B0F5E16F0BD3FE23A0F5E160584375
:102A18004FF49663B0FBF3F0C0B208BDFE20FCE7AC
:102A28000020FAE77FB5684600F0CAF80198FFF77A
:102A380045F800B207B05DF804FB0000194A38B544
:102A4800D2F88035591C044619D104F061F90546BD
:102A580004F06AF9054404F061F92B0EE3712B0CBC
:102A6800A3712B0A6371030EE370C0F30742C0F32E
:102A780007232571C0B2A2706370207038BD190A8F
:102A8800C3718171190C1B0E41710371D2F8843521
:102A9800C370D2F88405C0F30722C0F30743000EC1
:102AA800E9E700BF0070FF1F38B5094BD3F8803540
:102AB80003600133054609D104F02AF9044604F0FD
:102AC8002DF9444004F030F944402C6038BD00BF73
:102AD8000070FF1F0121022010F0AABB0021022074
:102AE80010F0A6BB00207047024B187808B100F020
:102AF800BBB87047D80A002082B00190019802B094
:102B080000F04EB94FF0B04382B0DA6C42F00202E6
:102B1800DA64DB6C03F002030193019B02B0704797
:102B28002DE9F043254C87B004F004F904F00AF9C4
:102B380004F010F90123002502934FF48059032370
:102B480001A9204604934FF4005803950595FFF713
:102B5800D9FFFFF7D7FFFFF7D5FFFFF7D3FFCDF872
:102B6800049005F093F801A920464FF40067CDF8CA
:102B7800048005F08BF801A920464FF40046019720
:102B880005F084F801A92046019605F07FF82A4649
:102B98004946204605F0A0F92A464146204605F058
:102BA8009BF92A463946204605F096F92A463146C9
:102BB800204605F091F907B0BDE8F083000400480D
:102BC80010B50446FFF7C2F9074BA36040F30F2086
:102BD800FEF720FF054B064A2360064B6060C4E9F8
:102BE8000323002010BD00BF0000484200007A44C3
:102BF8000D093E00AB03050000207047014B186823
:102C0800704700BFDC0A00200320704708B5014662
:102C18004FF47A7200238002890DFEF775FF08BD14
:102C28004FF47A73A0FB0303800A40EA835070478D
:102C3800034B98689A689042FBD1C043704700BF25
:102C48000028004008B5FFF7F3FF014B186008BDE6
:102C5800DC0A002008B5FFF7EBFF024B1B68C01A1F
:102C680008BD00BFDC0A0020024B187808B1FFF746
:102C7800DFBF7047D90A002010B5074B074C012267
:102C8800DA654FF48071204606F06CFA4FF0FF3396
:102C98002363002010BD00BF00280040680A002000
:102CA80002460021014806F076BC00BF680A0020F1
:102CB80002460121014806F06EBC00BF680A0020E8
:102CC80010B58CB02C220021044601A810F034FF66
:102CD800FFF7D2FF0C4B0D481B681C4400230893D8
:102CE80006934FF00053E443079301224FF4807397
:102CF80001A902940B9306F04BFB08B1FFF7C0FC47
:102D080000200CB010BD00BFDC0A0020680A0020BB
:102D180038B50546FFF78CFF02210446074806F040
:102D280041FCC4F309024FF47A71A2FB0121920A13
:102D3800A30A2A8043EA805038BD00BF680A0020F1
:102D48000148002106F02EBC680A00200148012134
:102D580006F028BC680A0020F8B50F4D2E78CEB9C9
:102D68000E4C4FF0FF372763FFF78CFCFFF784FF0B
:102D78004FF48071204606F0F5F92046276306F0E7
:102D8800B5FB32462046022106F005FCFFF75AFF44
:102D980001232B700020F8BDD90A0020680A002002
:102DA800014610B54FF47A7200238002890DFEF7B0
:102DB800ABFE0146FFF73CFF0446FFF739FF031B54
:102DC8008B4200D310BD00BFF7E710F043BD0000F1
:102DD80010B5064C0221204606F0E4FB0221421CF5
:102DE8002046BDE8104006F0D6BB00BF680A0020A8
:102DF8001648174A08B54FF4E133C0E90023002309
:102E08000C22C0E90233C0E90523C0E90733C0E951
:102E18000933036107F053FD08B1FFF731FC0B4894
:102E2800002107F0C8FE08B1FFF72AFC0748002177
:102E380007F0E1FE08B1FFF723FC044807F09BFE0A
:102E480018B1BDE80840FFF71BBC08BDA00B002067
:102E58000044004070B596B005461422002103A82E
:102E680010F06AFE3822002108A810F065FE2A68D2
:102E7800334B9A4261D10223089308A8314B0A9335
:102E880006F0A0F808B1FFF7FBFB4FF0B0430C21A8
:102E98009A6D2D4C42F400329A659A6D02F4003214
:102EA8000292029ADA6C42F00102DA64DB6C03F0F7
:102EB80001030193019B02230026CDE90313032399
:102EC800CDE905634FF09040072303A9079304F069
:102ED800DDFE1E4826621423C4E900031023C4E95A
:102EE800023620468023C4E90436C4E9066604F0A5
:102EF80005FC08B1FFF7C4FB154AEC67A562154C41
:102F08001323C4E90023204600238022C4E90233A6
:102F1800C4E90423C4E90633236204F0EFFB08B1D3
:102F2800FFF7AEFB2520C5F8804000220221A562EC
:102F380004F052FB252004F081FB16B070BD00BFE1
:102F48000044004004000C00400B002080000240B8
:102F58006C000240E00A002002680E4B9A4210B54D
:102F6800044616D14FF0B0420C21936D23F4003380
:102F780093654FF0904004F035FFE06F04F032FCA9
:102F8800D4F8800004F02EFCBDE81040252004F0A1
:102F980063BB10BD0044004008B50A46014602481C
:102FA80006F010FE002008BDA00B002013B5114B41
:102FB800114C18604FF40013009302AB13E906009C
:102FC800204607F07CFD2368DA69D103FCD4DA696E
:102FD8005202FCD59A68084842F480029A6007F0C9
:102FE800B4FD06490448012207F022FD002002B082
:102FF80010BD00BF340C0020A00B00203C0C0020AA
:1030080008B5074B1860FEF7FEFFFFF7F1FE054A0B
:10301800D2F8803043F00063C2F88030002008BD49
:10302800380C00200008005808B54FF0B043084895
:103038009A6B42F400329A639A6B22F400329A63D4
:10304800FFF78AFF0F2004F007FB002008BD00BF30
:10305800A00B002008B5074807F031FC08B1FFF7BE
:103068000FFB054804F04AFB18B1BDE80840FFF71C
:1030780007BB08BDA00B0020400B00200268044BD2
:103088009A4203D1034B00201B681847704700BFC2
:1030980000440040380C002002680B4B9A4210B5DF
:1030A80004460FD1094B1B682BB1D0F8902012B9F8
:1030B80007480121984720460549BDE810400122EC
:1030C80007F0B6BC10BD00BF00440040340C00201F
:1030D8003C0C002002480122102104F0FDBE00BF74
:1030E8000004004802480022102104F0F5BE00BF89
:1030F8000004004810B50A4C23780BB9E37C6BB187
:10310800FFF7D8FB0038074B18BF012040001870A4
:103118001B78022B02BF00232370E37410BD00BF8D
:103128004E0E0020440C002038B5114C2378F3B91A
:10313800E37CE3B90F4D2B68012B07D92B68042BCF
:1031480004D80D4A0421012000F016FA2B68042B3C
:103158000DD9FFF7AFFB0038084B18BF012040001E
:1031680018701B78022B02BF00232370E37438BD4C
:103178004E0E0020400C0020D43D0108440C0020D5
:1031880008B5FFF7A7FF01F0F9F9BDE80840FFF718
:10319800A9BF022801D8FFF79DBF7047022801D8B0
:1031A800FFF7A0BF70470000022808B51BD801220E
:1031B80010210D4804F090FE3220FFF79DFC0A48CC
:1031C8000022102104F088FE01221021064804F094
:1031D80083FE3220FFF790FCBDE808400248002239
:1031E800102104F079BE08BD00040048704708B5F6
:1031F800FFF7D2FBBDE8084000F064BB4FF0FF309A
:1032080010F0A6B87047704770470000014BD8709F
:10321800704700BF5C000020014B1874704700BF66
:103228005C00002020B1037813B1024810F0C0BA46
:10323800704700BF840D002008B50220002110F05F
:103248004FF8BDE80840014810F0B2BA9C0D0020C4
:103258000021012010F044B810B5094C60B120607D
:10326800084810F057FA2168064810F0DBFABDE864
:103278001040044810F09CBA42F210732360EFE744
:10328800740000209C0D002010B5094C20602368B4
:103298000BB9084B2360084810F03CFA216806482F
:1032A80010F0C0FABDE81040034810F081BA00BF22
:1032B8000C000020A0860100B40D002038B504469B
:1032C8000D4607484FF40061FFF74CF830B92A461D
:1032D80021460348BDE83840FEF746BF38BD00BF69
:1032E80000F003080A460149FFF71CB800F003087C
:1032F80038B50C4810F00EFA08F0D6F860B90A4C48
:103308000A480125257007F073FF2078294607F041
:103318009DFD044810F04CFABDE83840044810F010
:1033280047BA00BF9C0D0020000000205C00002070
:103338006C0D002008F056B930B585B0FFF75AFB80
:10334800002104464FF480700FF0CAFF684600F071
:10335800F7FF23B203EB4303FE2203EB4313B3FB54
:10336800F2F3314A0B211170304950680978DBB209
:103378008DF80C30017054680020607054681A256C
:10338800A57054680125E57054682371284B1C7892
:1033980044B118700C231370536861F07F011970E1
:1033A800052314E0234B2448197811B90178002922
:1033B800F6D0002101701970536802215971BDF8C7
:1033C80000305168180A88715168CB7108231B496D
:1033D8001B4C0978012988BF00235370637A33B1E5
:1033E80007F0D6FC012802D1204610F093F9154BBE
:1033F8000D48D978002207F0B7FD063012D107F042
:10340800C1FC0446104810F085F9104B0E481968A5
:10341800A14238BF214610F005FA0B4810F0C8F950
:1034280005B030BD0024EDE704000020370D002072
:10343800CC0D0020630E00204D0E0020440C00200F
:10344800380D00205C0000209C0D00207400002036
:1034580008B5104B0122002102201A700FF040FF1E
:103468000D4810F0A5F90D4B1B788BB10C4B1A7851
:1034780072B9DB7C63B90B4B1A68042A9EBF1A68C1
:1034880001321A600021BDE8084010200FF028BF63
:1034980008BD00BFCC0D0020B40D0020680D002031
:1034A8004E0E0020400C0020044B1B78022B03D149
:1034B800002108200FF014BF704700BF0000002053
:1034C80008B507F0FAFF80B907F062FC01280CD1B3
:1034D800BFF34F8F0549064BCA6802F4E0621343F5
:1034E800CB60BFF34F8F00BFFDE708BD00ED00E0E4
:1034F8000400FA0510B5044690B190F906307BB97E
:10350800084810F007F9084BE2791A70074B186859
:10351800FFF7BAFE064BBDE810401868FFF79CBEDF
:1035280010BD00BF380D0020680D00200C000020E1
:10353800740000207047704770477047022808B52C
:1035480001460FD0202810D0012811D14FF090400B
:1035580004F0BCFC01280BD100210220BDE8084082
:103568000FF0BEBE00210820F8E7024B01221A70B6
:1035780008BD00BFC80E002070B505460C461646AB
:1035880007F0D4FC0346002834D000241A4810F071
:10359800C1F81A4B18481968A14238BF214610F0E3
:1035A80041F9BDE87040144810F002B94A68F05C6F
:1035B800D0540133DAB29442F8D8114B0D701B780D
:1035C800012B88BF00244C700E4C637A33B107F08E
:1035D800DFFB012802D1204610F09CF80A4B0B486B
:1035E800D978002207F0C0FC0630CED107F0CAFB1C
:1035F8000446CBE70549DDE79C0D00207400002058
:10360800440C0020380D00205C000020040000203D
:10361800044B1B7823B9044A05210120FFF7ACBFEE
:10362800704700BF440C0020D93D010810B50024A4
:1036380090B03C22214601A8009410F07DFA2F4B4F
:103648002022DA7219788DF8001059788DF8011057
:1036580099788DF80210D9788DF8031019798DF8BA
:10366800041059798DF8051099798DF80610D979D3
:103678008DF80710197A8DF80810597A8DF8091005
:10368800997A8DF80A108DF80B2021460DF10B025E
:1036980058180131007B02F8010F1C29F8D193F862
:1036A80028208DF8282093F829208DF8292093F8D0
:1036B8002A208DF82A2093F82B208DF82B2093F8B8
:1036C8002C206AB193F83F2052B10DF12B01002252
:1036D8009818013290F82C0001F8010F142AF7D13C
:1036E80007484FF40061FEF73DFE20B90448402228
:1036F8006946FEF739FD10B010BD00BF7800002004
:1037080000F80308014940220FF0DEBD00F8030865
:1037180070B52A4D28796B794D2BC0B233D1C0EBE7
:10372800001080000A2838BF0A204FF47A735843E3
:10373800234BAC791860EB794D2BE4B22BD1C4EB59
:103748000414A40095F82C301E4E63BB95F83F3046
:103758004BBB42F21070FFF77FFD3068FFF794FD16
:103768002B7A194A1949DBB213706B7A184ADBB203
:1037780013700023EA1892F82C20D2B2CA540133ED
:10378800142BF7D170BD6B79482B0ABF4FF46163D6
:103798006B795843C6E7EB79482B0ABF4FF461634E
:1037A800EB795C43CEE7FFF757FD012C38BF0124C6
:1037B8004FF47A735C433460CFE700BF7800002091
:1037C800740000200C000020620E00204E0E002025
:1037D800440C002010B590B000213C2201A80091B3
:1037E80010F0AAF94022344968460FF06DFD9DF8A3
:1037F80000203AB99DF801001A2803D19DF802105B
:1038080001290ED0FFF712FF2C48142200210FF0D7
:1038180065FD4FF47A70FFF76FF9FFF779FF10B085
:1038280010BD274B1A70587099709DF80310D97005
:103838009DF8041019719DF8051059719DF806102E
:1038480099719DF80710D9719DF8081019729DF8A3
:10385800091059729DF80A1099729DF80B1001F021
:103868003F01D972D87AD1B288421BD89DF8282056
:1038780083F828209DF8292083F829209DF82A20FC
:1038880083F82A209DF82B2083F82B200DF12B019B
:1038980000229818013211F8014F80F82C40142AA0
:1038A800F7D1BAE701F140006844194410F8340C24
:1038B80008730132D6E700BF00F803084E0E002057
:1038C800780000201FB5002403A92046039407F0C0
:1038D800D7FD03A9012007F0D3FD384B38480094E1
:1038E80022464FF4FA710FF0B7FE364B3648009473
:1038F80022464FF4FA710FF0AFFE344B344800946F
:1039080001224FF4FA710FF0A7FE2046FEF726FCBD
:1039180008B1FEF7B5FE2F4B009400224FF4FA6170
:103928002D480FF099FE2D4A002101200FF094FD3B
:103938002B4A002102200FF08FFD2A4A0021042083
:103948000FF08AFD284A002108200FF085FD00F0BD
:103958007DFB2649264807F055FD264807F048FC18
:103968001B480FF025FF244B0021187807F06EFA4A
:1039780022490094224B0968224800220FF06CFE6D
:1039880020480FF015FFFFF725FF1F4A00211020E0
:103998000FF062FD1D4A00214FF480700FF05CFDAE
:1039A8001B4B1C4819681C4B009400220FF054FE56
:1039B80018480FF0FDFE04B010BD00BF41350008E7
:1039C800840D002043350008500D00203D350008C7
:1039D800380D0020B13400086C0D002051AD0008EE
:1039E800413300083D330008F932000800000301A4
:1039F800100000205C00002000000020740000205F
:103A0800413200089C0D002031310008893100083E
:103A18000C000020B40D00205934000810B5002413
:103A2800A2B021467C2203A8029410F085F8532303
:103A38008DF808304FF48D73ADF80A300123ADF8D6
:103A480004408DF80C30FEF7D5FF00B200EB4000C3
:103A5800FE2300EB4010B0FBF3F08DF80D0001A839
:103A680000F07EFC072498B958238DF80E303022D8
:103A78008021164810F060F8224602A9134810F079
:103A880094F8124A21460120FFF776FD22B010BDB6
:103A98008DF80E408DF80F0000F070FD0C4B1A6881
:103AA80012128DF810201A688DF811205A68121217
:103AB8008DF812205A688DF813209A689B688DF843
:103AC800153012128DF814200E24D0E7CD0D0020E9
:103AD800F40E002030B50378592B91B0044640F01D
:103AE800E881052959D84378443B162B55D8DFE897
:103AF80013F026015400160154001E01540054000E
:103B0800540054008800540001015400540054002B
:103B18008F0154005400A4005400540054001700AE
:103B28008578482D11D1B14A14210120FFF724FDD1
:103B380041F28830FEF7E0FF40F6B830FEF7DCFFD0
:103B480011B0BDE83040FFF7BBBC532D0ED1302279
:103B58008021A7480FF0F0FFFFF760FF41F288309F
:103B6800FEF7CAFFA24A152101207BE0432D16D19A
:103B7800002468468DF8004007F09EFA9C4A4C23C2
:103B880013701A2393709DF800305470012041334C
:103B9800D07013710521FFF7EFFC11B030BD442D33
:103BA800FBD1934C592323705A236370A57000F0FE
:103BB800B8FB2C228021201D0FF0BEFF00232570AA
:103BC800637001251A23A370E5702571FEF712FFB3
:103BD8008849FE23B0FBF3F04B6864229BB2B3FB29
:103BE800F2F3A3714B6800EB40009BB200EB40106E
:103BF800B3FBF2F102FB11336071E3712246082135
:103C0800B2E78378303BDBB2092BC6D87A497B4AC6
:103C18000B700B78DBB25372754A592313704D231E
:103C280053700B783033937003210120FFF7A4FC05
:103C380011B0BDE83040FFF7F9BC8578482D16D1A2
:103C48006B4A56231370002353701A23937003236F
:103C58001371172353710B23012093710A23D0701A
:103C6800D371082111B0BDE83040FFF785BC432D62
:103C780093D15F4C00213C2201A800910FF05CFF1A
:103C88006846FFF73FFD2422802104F10C000FF065
:103C980053FF9DF8003063709DF80130A3709DF8C4
:103CA8000230E3709DF8033023719DF8043063718E
:103CB8009DF80530A3719DF80630E3719DF8073033
:103CC80023729DF80830257063729DF80B509DF89B
:103CD8000930A3729DF80A30E3722A4603A92573B6
:103CE80004F10D000FF061FF05F10D012246C9B284
:103CF800012050E7807839280CD83038C0B2FFF757
:103D080048FA3B4A2378137063785370A37893700A
:103D1800032129E711B0BDE83040FFF779BC80786E
:103D28003928F7D83038C0B2FFF738FAE9E7807891
:103D38003928EFD83038C0B2FFF736FAE1E7837890
:103D4800303BDAB2092AE5D8C0783038C2B2092A3D
:103D5800E0D82179A1F14802D2B20B2ADAD8284D4D
:103D680045FA02F2D507D5D40A224D2902FB0300F1
:103D780036D13C2358434FF47A735843214B18608B
:103D8800214B1860FFF768FA194A23781370637893
:103D98005370A3789370E378D37023791371052156
:103DA8000120FFF7E9FB154B00221A701A225A70FE
:103DB80001229A70DA70A278303A02EB8201E27836
:103DC800303A02EB4102D2B21A7122795A710F4A83
:103DD8001278D2B21A72084A1278D2B25A7227E707
:103DE8004829C8D14FF46163C4E700BFDF3D01082B
:103DF800CD0D0020F40E0020440C00207800002097
:103E0800DEF7FFFF740000200C000020620E002087
:103E18008278303AD3B2092B3FF67CAFC378303B77
:103E2800D9B209293FF676AF0079A0F14801C9B2A5
:103E38000B293FF66FAF624D45FA01F1C9073FF50F
:103E480069AF0A214D2801FB02332DD13C2253438F
:103E58004FF47A7253435B4A13601068FFF714FA01
:103E6800594A2378137063785370A3789370E37872
:103E7800D3702379137105210120FFF77DFB534B84
:103E880000221A701A225A7001229A70DA70A278E7
:103E9800303A02EB8201E278303A02EB4102D2B2C8
:103EA8009A712279DA7192E74828D1D14FF4616288
:103EB800CDE7502B48D102297FF66FAE4378303BCF
:103EC800012B3FF66AAE8378312B7FF466AE0B295F
:103ED80004D8FFF79DFB00213B4A45E63B4D0234E1
:103EE800002214F8013FA918303B0132DBB20C2A3A
:103EF8000B73F6D1FFF77AF9334B50221A211A7057
:103F08009970002201215A70D97003F8041FA9186A
:103F18000132097B0C2A01F1300103F8011FF6D1A7
:103F280000232B701A236B700123AB70EB70284BA6
:103F38001B78DBB22B72274B1B78DBB26B72EA72F1
:103F4800FFF774FB1121C7E7412B7FF426AE4378B6
:103F5800432B7FF422AE16297FF41FAE1E4D421C60
:103F6800002312F8011FE9540133142BF9D1FFF78C
:103F7800C1F81A4B5B7D012B19D114490023EA5C67
:103F8800C8180133D2B2142B80F82C20F7D1114B6A
:103F980000221A701B78DBB24B72FFF747FB0A4A04
:103FA800631E1534A34206D1074A1621DCE5094BE6
:103FB80002221A70F3E713F8011F02F8011BF1E758
:103FC800DEF7FFFF0C000020CD0D00207800002058
:103FD800620E0020440C00204E0E0020B40A00207F
:103FE80038B504460D4661B316480FF0E1FB2B784F
:103FF8003BB334B36068237818B3032B0CD00B2B76
:1040080017D0022B1DD1617801291AD00B0618D4BC
:10401800BDE83840FFF75EBD6378012B11D1007809
:10402800012802D0022800D058B9BDE8384006F06F
:10403800C3BE6378012B04D10378034A03F001035C
:10404800137038BD500D0020370D0020034B00229F
:10405800C3E902220122C3E900227047640E00204E
:1040680000487047640E00204FF0B04382B0DA6C0D
:104078000243DA64DB6C03400193019B02B0704792
:104088002DE9F04186B000240220154D0594FFF774
:10409800EBFF0420FFF7E8FF124F03944FF48076FC
:1040A80001230DEB0001CDE90163284603230493A6
:1040B8004FF4005803F0EAFD01A93846CDF8048012
:1040C80003F0E4FD22464146384603F005FF284642
:1040D8002246314603F000FF204606B0BDE8F081D5
:1040E8000004004800080048032810B50ED801282D
:1040F80010D868B902460B484FF4807103F0ECFE03
:10410800002209484FF4005103F0E6FE002010BDDC
:104118000122F0E7002203484FF4807103F0DCFE2F
:104128000122EEE70004004800080048022070471A
:10413800002070470120704700280CBF0F20162070
:10414800704700000D48854602F0BCFD0C480D493B
:104158000D4A002302E0D458C4500433C4188C42DA
:10416800F9D30A4A0A4C002301E013600432A24240
:10417800FBD30FF0E9FCFEF76FFAFEE70000012021
:1041880000000020CC08002094480108CC0800203A
:10419800382E0020FEE74FF0B04382B0DA6C42F0D0
:1041A8000102DA64DB6C03F001030193019B02B0A6
:1041B8007047000030B587B0FFF7EDFF4FF480512E
:1041C80001224FF0904003F087FE01224FF4006176
:1041D8004FF0904003F080FE4FF4C0551123CDE915
:1041E800015301A901234FF09040039303F04EFDC2
:1041F80008240A2500224FF480514FF0904003F024
:104208006BFE0120FEF778FC01224FF480514FF03D
:10421800904003F061FE0120FEF76EFC013DE9D1FC
:104228004FF400614FF0904003F050FE08B9013C94
:10423800DFD14FF400614FF0904003F047FE68BBB8
:10424800FFF7A9FF04240123039001A92A48CDE917
:10425800014303F01BFD284C01220421204603F0F2
:104268003BFE2120FEF748FC00220421204603F0F3
:1042780033FE2120FEF740FC01220421204603F0F2
:104288002BFE2120FEF738FC20460022042103F0F3
:1042980023FE4FF42570FEF72FFCDDE7FFF77BFFC9
:1042A8004FF0B04300249A6D42F480029A659B6DEA
:1042B80003F4800300934FF4C052009B1223CDE90E
:1042C80001230323CDE9034304230DEB03014FF03E
:1042D8009040059303F0DAFC08480949094B8460CB
:1042E800C0E900130123C0E90334C0E9074444616D
:1042F80003F066FF07B030BD00040048740E0020CC
:10430800005800401A091020FFF754BF40B94B1E4F
:104318005A425A414FF400714FF0904003F0DCBD0F
:10432800704708B50120FEF734FF6420FEF7E4FB70
:1043380000F024F9BDE808400120FEF72FBF000077
:10434800054B1A6802805A689B684381034B0281B7
:1043580001221A70704700BFF40E00204D0E002095
:1043680010B5044600F008F810F0FF001FBFEE2358
:104378002370AA23637010BD2DE9F3470024304E43
:10438800304D346021462046FFF7C0FF214601200A
:10439800FFF7BCFF21460220FFF7B8FF2A4F4FF076
:1043A8005208A146012195F8640185F86081C5F895
:1043B8006891FFF7ABFF0320FEF79EFB00228821E0
:1043C800284602F0E5FB0DF10602C021284602F05E
:1043D8002DFC80BBBDF806204EF6AA639A422AD16E
:1043E8004FEA440A0AF1540A5FFA8AFA5146284603
:1043F80000F034F9F8B90DF10602C021284685F815
:1044080060A102F013FCB0B9284600F0EBFA90B9AD
:10441800326801231A4432603A68C5F86831A3400B
:1044280013433B600134032C05F5C875BAD13068D5
:1044380002B0BDE8F0870021E0B2FFF767FFF1E7BF
:10444800EC0E0020BC000020E80E00202DE9F74FFC
:10445800354C834604F5966A4FF00A094FF00E086A
:1044680048F2E8074FF490164FF48045D4F86821D5
:10447800002A51D0204600F0A9FD0DF102020DF1ED
:104488000101204600F05CFB0DF1030201A9204662
:1044980000F0A1FE0021204600F0E4F801220021EE
:1044A800204600F0A3F901221146204600F09EF9AB
:1044B800BBF1020F0ED81D4B1D4A33F81B501D4B84
:1044C80012F80B8053F82B601B4A1C4B12F80B9008
:1044D80053F82B702A460121204600F0D2F93246C3
:1044E8000021204600F0CDF93946204600F0D4F8E6
:1044F80042460021204600F0D1F84A4601212046D4
:1045080000F0CCF80DF102020DF10101204600F097
:1045180017FB0122C4F87C2104F5C8745445A5D1C1
:1045280003B0BDE8F08F00BFBC000020F43D0108D7
:10453800143E0108FC3D0108173E0108083E010829
:1045480010B50B7E9BB9D0F87C21098912B1C0E95E
:104558005E1310BD084BD0F878411A68C2F5807315
:104568004B4304FB02331B12C0F87831F1E70123F7
:10457800C0F87C31EDE700BFB80000202DE9F84F06
:10458800DFF8C0A0304DFFF7BFFEDAF800300BB1FE
:104598002B6813B9FFF7F0FE28602B682B4E002418
:1045A800A34234607460B46049DDDFF8A480294D0B
:1045B800DFF8A4B02046FFF749FF88F80040D5F897
:1045C8006831012B31D103FA04F90A272249284618
:1045D80000F05CFCB0B959462846FFF7B1FF9BF8DC
:1045E80018307BB9D5F8783146F82430DAF800303D
:1045F80043EA0903CAF8003098F8003043F0010391
:1046080088F800300120FEF777FA9BF818301BB1C4
:10461800013F17F0FF07D9D1D5F8783140F6C41219
:10462800002B08BF134646F8243005200134FEF756
:1046380063FA032C05F5C875C1D198F80030BDE8B8
:10464800F88F00BFE80E0020F00E0020F40E0020C6
:104658004D0E0020BC000020CC0E00204A088A2104
:1046680002F096BA152906D8044BCB40DB0702D5D1
:104678000174002070476FF0070070470B0030008E
:1046880010B50A460C46092102F0A4FA18B9237895
:1046980003F00103237010BD01F06BBE01F053BDA0
:1046A80001F04DBEF7B500230C46174601210DF168
:1046B800070206468DF8073002F08CFA0546D8B98D
:1046C800012F9DF8073026D1042C3AD8DFE804F0F2
:1046D80003171A1D200043F01004A3420CD02246F1
:1046E8000121304602F054FA054628B9716986F866
:1046F80030413046FFF7D0FF284603B0F0BD43F005
:104708002804EAE743F00404E7E743F04004E4E759
:1047180043F08004E1E7042C13D8DFE804F0030633
:10472800090C0F0003F0EF04D7E703F0D704D4E730
:1047380003F0FB04D1E703F0BF04CEE703F07F04E6
:10474800CBE76FF00305D7E713B500230C460DF14F
:10475800070201218DF8073002F03CFA78B99DF87C
:104768000730C3F300122270C3F3C002A270C3F370
:1047780080026270C3F38012DB09E270237102B019
:1047880010BD37B50D460DF10202F821044602F0BE
:104798004DFA70B901AA0421204602F067FA40B91F
:1047A800BDF802201AB1019BB3FBF2F32B602B6812
:1047B800A36103B030BD037F0B700020704737B58D
:1047C8000D460DF106022021044602F02FFA28B901
:1047D800BDF8063023B9236A2B60207703B030BDBB
:1047E800DB002B60236201232377F7E70529F8B55F
:1047F80004460E46154635D862B100EB8103012107
:104808005A6B0023701E042807D8DFE800F00E1743
:104818001A1D240011460123F4E784F828103444B3
:10482800E5B984F82850002007E0C2F34F2244215C
:10483800204602F0BDF90028F1D0F8BD84F82A100E
:10484800EDE784F82B10EAE75B00FE2260212046A2
:1048580002F0D5F9EFE71B01EF22F7E7012384F80F
:104868002830E0E76FF00300E7E7052996BF401816
:10487800002390F82830137094BF00206FF00300D5
:10488800704770B54318044693F828000E4615463D
:1048980018B904EB8106726370BD05291BD8DFE8DF
:1048A80001F0030912141616626304EB8604002053
:1048B8006563F1E7C2F34F224421204602F078F9FC
:1048C8000028E9D1F1E7E263EFE72264EDE7C2F3FC
:1048D8004F226421F1E76FF00300DDE737B50446A6
:1048E800154605292CD8DFE801F0030717191B1B0B
:1048F800436B2B60002021E00DF10602442102F0F9
:1049080095F9D8B9BDF8062053029AB12B60A36374
:10491800012384F8293011E0C36BEAE7036CE8E768
:104928000DF10602642102F081F938B9BDF80630AC
:104938005B02DEE7A36B2B6084F8290003B030BD6F
:104948006FF00300FAE737B50D460DF107020121B4
:10495800044602F03FF938B99DF8073084F8303141
:10496800DB092B7084F84C3003B030BD2DE9F843D7
:10497800037C0C4601F8083B0546FFF702FF40BBE5
:10498800207304F110012846FFF719FF08BB04F152
:104998001401284600F021FCD8B904F1240705F1D8
:1049A800270904F1170806463A46B1B22846FFF728
:1049B80095FF70B9013619F8013F08F8013F062E36
:1049C80007F10407F0D104F13C012846FFF7BBFFCB
:1049D80008B1BDE8F883211D2846BDE8F84301F079
:1049E80030BD0000F0B50022054693B0882102F0E2
:1049F800CFF84FF47A72A5F852214FF4C872A5F88F
:104A080054214C4AC5F8582100234B4A85F8F03008
:104A1800C5F8D4202B6202A92846FFF7A7FF044651
:104A280070B9ADF8080002AE0FCE05F110070FC738
:104A38000FCE0FC70FCE0FC796E80F0087E80F00FD
:104A48003E4BC5F834314FF4FA730126A5F83831D6
:104A58004FF42063A5F83C313246802185F8506137
:104A6800284602F095F832460746FF21284602F00C
:104A78008FF8002211460743284602F089F83C4384
:104A880064B204430DF107029121284602F0A2F80E
:104A980064B29DF8073085F83A3104433246002164
:104AA800284602F075F864B204430022FF21284624
:104AB80002F06EF864B2044300228021284602F016
:104AC80067F864B2204340B2002488BBA1B2012237
:104AD80028460134FFF78AFE062CF6D140BB04466F
:104AE8006885024604212846FFF780FE00BB02467F
:104AF80005212846FFF77AFED0B94FF490136B636F
:104B08004FF4804201212846FFF7BBFE80B94FF4DD
:104B18000C13FF22C5E90F3085F830210121284602
:104B280002F036F8012385F8323108B985F81541C5
:104B380013B0F0BD856B0100A47009006400840304
:104B4800012300F079BD2DE9F0428EB00C460C230C
:104B580004AA1421054602F005F8844600286CD101
:104B68009DF81A309DF81B609DF817209DF81810C5
:104B7800A07506EB03269DF81630206002EB032291
:104B88009DF81930606003EB01239BB25B029DF82E
:104B9800121023619DF81330B5F8520103EB01237D
:104BA80092B252029BB2E260A382B0F57A7F9DF87E
:104BB800101095F83171B6B20AD0704300F5FA704A
:104BC8004FF47A76B0FBF6F02E7F002E39D186B2FC
:104BD800002F40D0B001C0B2B608E0750DF10F004B
:104BE8002681CDE90040284601F086FE844620BB98
:104BF8009DF80FE084F818E005F150060FCE07AFD6
:104C08000FC796E80700E37D87E80700D4E90301AA
:104C1800A28AADF83020D4E90149CDE90A01CDE9ED
:104C2800084907AC8DF833308DF834E00FCC503597
:104C38000FC597E8070086E8070060460EB0BDE894
:104C4800F0822E8C5E43B2EB262F4FEA262C04D13D
:104C580057B948F6E0260020BFE780B25043A2EBE0
:104C68000C06B0FBF6F0B2E742F2B826B2E7000055
:104C7800F7B517460E210DF106021D460B4C0646E8
:104C880001F0D4FFBDF8063004EA43433B6050B955
:104C98000DF106020C21304601F0C8FFBDF80630C0
:104CA80004EA43442C6003B0F0BD00BF0000FE1FBF
:104CB80073B590F8DA30013B022B06460C4634D81F
:104CC80001AB6A460121FFF7D3FF009BB3F57F0FC5
:104CD800054603D8019BB3F57F0F23D915BB34B123
:104CE8001349304602B0BDE8704001F00FBC042201
:104CF800FF21304601F04CFF2A4604467021304619
:104D080001F046FF2A460443FF21304601F040FFE8
:104D180064B204432A468021304601F039FF64B268
:104D2800044365B2284602B070BD0025FAE700BF0B
:104D38005F06002037B5044601228021057C01F07A
:104D480027FF0122FF21204601F022FF0022114601
:104D5800204601F01DFF94F83A219121204601F0E8
:104D680017FF01220021204601F012FF0022FF2137
:104D7800204601F00DFF00228021204601F008FFA7
:104D8800012D29D0032D37D0002D3CD101222946F1
:104D9800204601F0FDFE01238DF80730A0B103B0D5
:104DA80030BD01460DF10702204601F013FF9DF8C2
:104DB8000730DB0705F1010508D538B9B5F5FA6FF5
:104DC800EFD16FF00600EAE70546F0E7B5F5FA6FB0
:104DD80008BF6FF00600E2E718B929462046FFF73A
:104DE80067FF02220021204601F0D2FE0028D6D11A
:104DF800042384F83231D2E718B901212046FFF79D
:104E080057FF0422EEE76FF00700C8E738B5057CC6
:104E1800044625B1204600F054FD28B138BDFFF7FF
:104E280089FF0028F6D0F9E7002DF7D1032384F88D
:104E38003231F3E773B50646002501220B213046CF
:104E480001F0A6FE002204460B21304601F0A0FE28
:104E58000DF1070204431321304601F0BBFE9DF813
:104E6800073064B2044301355B0760B2EDB205D088
:104E7800032D08D00028E0D002B070BD032D08BF74
:104E88006FF00B00F8E76FF00B00F5E738B500237B
:104E9800037404460D46FFF7B9FF50B9294620466A
:104EA800FFF751FE28B901462046BDE83840FFF714
:104EB800C1BF38BD152970B5054616461C4667D1D1
:104EC8000122FF2101F064FE002211460446284613
:104ED80001F05EFE00220443FF21284601F058FE3F
:104EE80064B2044301228021284601F051FE64B2D5
:104EF800044302228521284601F04AFE64B2044395
:104F08000422FF21284601F043FE64B20443002234
:104F1800CD21284601F03CFE64B204431122CC2185
:104F2800284601F035FE64B204430722FF212846D3
:104F380001F02EFE64B204430022BE21284601F08F
:104F480027FE64B204430622FF21284601F020FE12
:104F580064B204430922CC21284601F019FE64B248
:104F680004430022FF21284601F012FE64B20443E4
:104F78000122FF21284601F00BFE64B200220443FF
:104F88001146284601F004FE64B2204340B270BDC9
:104F9800042A17D80A2101F0FBFD0028F7D1231EA7
:104FA80018BF01231B01EF228421284601F027FEA8
:104FB8000028ECD185F8DA6001462846BDE8704043
:104FC800FFF738BF6FF00A00E1E7000070B594B052
:104FD80005464022002104A80EF0AEFD0023012161
:104FE8002846ADF806308DF803308DF8043002936A
:104FF80000F0B8FC95F8142195F81311012A04D88B
:1050080040F0AD80202940F2AC8001AA02A92846D0
:1050180000F02DFB0446002840F09E8095F85031A2
:10502800002B40F0A280D5F84C11284601F06EFA0A
:105038000446002840F09080234621460422284652
:10504800FFF738FF0446002840F086800122FF2140
:10505800284601F09DFD0DF10602064684212846EA
:1050680001F0E4FD22460643FF21284601F090FDA9
:1050780076B2064374B2002C6ED1BDF806301B011F
:10508800C5F8D43004A92846FFF770FC0446002868
:1050980062D10DF103012846FFF7F2FA0446002811
:1050A8005AD19DF8033085F8313104AE0FCE05F1A1
:1050B80010040FC40FCE0FC40FCE0FC496E80F0014
:1050C80084E80F000DF103020121284601F082FD5A
:1050D8000446002840D19DF8033085F83031024657
:1050E80001462846FFF7DEFA0446A8BB024602211D
:1050F8002846FFF7D7FA044670BB0323014685F814
:1051080032310DF10502284601F019F9044618BBA1
:105118009DF8053085F8E8300DF105020121284693
:1051280001F00DF90446B8B99DF8053085F8E0306E
:1051380003AA0321284600F001FF044660B9039B37
:10514800C5F8E43003AA0421284600F0F7FE044617
:1051580010B9039BC5F8DC30204614B070BD0C298B
:1051680051E7284600F010F954E701495DE700BF10
:105178006C05002013B50C460DF10702132101F050
:1051880029FD9DF8073013F0180F03F0070218BF28
:105198006FF00500226002B010BD13B590F8DA3048
:1051A800042B0C460BD101A9FFF7E4FF019B042B4C
:1051B80001D1012300E00023237002B010BD01AA31
:1051C800142101F007FD0028F7D19DF80430DB0712
:1051D800EFD42070F1E700F04ABA13B50C460DF190
:1051E8000602282101F022FD78B9BDF80620C2F395
:1051F8000B0312F4006F18BFA3F580534FF0FA02A7
:1052080014BF13FB02F35343236002B010BDF0B583
:105218004FEAD20C4FF0FF341C6002F007026646DA
:1052280000278E4200D207B1F0BD845D664503BFFA
:105238001441E4B215463D4614F0010704D005EBCD
:10524800C6051D600136ECE70135082D4FEA540408
:10525800F2D1F7E7034B800953F82000003818BF54
:10526800012070471808002010B5B1EBD20F4FEAA3
:10527800D20402F0070381BF01229A40035D134361
:105288008ABF03556FF03100002010BD0A4606237F
:10529800B02101F049BC0A460623B02101F062BCE6
:1052A8002DE9F04F85B08046109E0E9D01968A46E6
:1052B80093461C464FF00009119B994508D10023DD
:1052C800129A1660F3B16FF0310005B0BDE8F08FA7
:1052D80001AB324629465846FFF799FF019F7B1CD0
:1052E8000DD00F9BF818FFF7B5FF504507D13A4688
:1052F8002046FFF7B9FF7E1C09F10109DCE76FF0D2
:105308003103DDE721464046FFF7C0FF0028DCD126
:1053180002A94046FFF7BFFF2544234602AAAB4235
:10532800D3D013F8014B12F8011B8C42F7D0CAE70F
:1053380070B5C02288B00E46012190F8304105466C
:1053480001F026FCF0B901A92846FFF79FFDC8B96E
:105358000122FF21284601F01BFC98B93246B621EC
:10536800284601F063FC68B90246FF21284601F08F
:105378000FFC38B922460121284601F009FC08B97A
:1053880085F8304108B070BDF0B50F4689B01646B3
:10539800FF210122044601F0FBFB0246A8B94F2178
:1053A800204601F0F5FB80B92C224E21204601F061
:1053B800EFFB024648B9FF21204601F0E9FB20B97E
:1053C800B422B621204601F0E3FB0025C4F824519D
:1053D800A4F82851DEB9354607ABB422CDE90373EA
:1053E8000623CDE90032029504F5927304F595720F
:1053F80031462046FFF754FF30B9012384F81531B0
:1054080084F8137184F8146109B0F0BD013505F111
:10541800B400FFF71FFF0028DED12C2DF6D1DBE703
:1054280010B541F001020021044601F0B1FB78B942
:10543800204600F046FA58B901462046FFF7FAFC24
:1054480030B9024601462046BDE8104001F0A0BB35
:1054580010BD2DE9F74F4FF0000B88461746FF2186
:10546800012205461E469DF838A09DF83C908DF80F
:1054780007B001F08DFB5A4604465946284601F00C
:1054880087FB5A460443FF21284601F081FB64B29A
:10549800044364B2B8F1000F32D0BAF1000F06D05D
:1054A8000C9ACB21284601F095FB204344B2B9F170
:1054B800000F07D00DF10702EE21284601F08AFB04
:1054C800204344B20122FF21284601F061FB01225A
:1054D80004430021284601F05BFB64B20443002228
:1054E800FF21284601F054FB64B29DF807300D9A5D
:1054F800204323F0100340B2137003B0BDE8F08FCF
:10550800BAF1000F06D03A46CB21284601F040FBFD
:10551800204344B2B9F1000FD4D033468022EE21A3
:10552800284601F06CFBCBE72DE9F04387B09146A4
:105538000022054688468DF817201E461BB390F8B2
:10554800307101221146284601F022FB044658BB5F
:1055580040212846FFF764FF044628BBB9F1010F34
:1055680013D10DF11703CDE90290CDE9008302466E
:10557800034649462846FFF76CFF40B104462046DB
:1055880007B0BDE8F0831F46DBE788F80000002E6F
:10559800F5D03A460121284601F0FAFA04460028D7
:1055A800EDD185F83071EAE7002388F8003020460D
:1055B800E4E72DE9F043054687B0884691461E4644
:1055C80023B390F8307102220121284601F0E0FA55
:1055D800044660BB01462846FFF722FF044630BB5D
:1055E800B9F1010F14D10DF11703CDE902090093A8
:1055F80002460346CDF8048049462846FFF729FFAE
:1056080040B10446204607B0BDE8F0831F46DAE7FC
:1056180088F80000002EF5D03A460121284601F00E
:10562800B7FA04460028EDD185F83071EAE700237F
:1056380088F800302046E4E7F8B51D4616460023F2
:105648002A4690F830710446FFF76EFF70B903469A
:105658002A4631462046FFF7ACFF38B93A460121C1
:10566800204601F095FA08B984F83071F8BD2DE9A3
:10567800F04F002393B0CDE90A12C0F82431A0F806
:1056880028310122FF21CDE90E33B0F83C818DF895
:10569800343005468DF8353001F07AFA0446002892
:1056A80040F0E38002464F21284601F071FA044693
:1056B800002840F0DA802C224E21284601F068FAB2
:1056C8000446002840F0D1800246FF21284601F018
:1056D8005FFA0446002840F0C880B422B621284664
:1056E80001F056FA0446002840F0BF8002468021A7
:1056F800284601F04DFA0446002840F0B6800346DB
:105708000DF135020DA92846FFF796FF044600283B
:1057180040F0AB800323CDE90203B421062305F54D
:10572800957A05F592790EAECDE9003104960146D9
:105738004B4652462846FFF7B3FD0446002840F082
:1057480094800DF1360128460E9FFFF7F1FD0446BF
:10575800002840F08A80BDF83630434540F2AA80E0
:10576800C5F82401A5F8280107F1B400FFF772FD78
:1057780008B92B2F7DD90623B4224FF0030BCDE9AE
:105788000032CDE9027B04964B4652460121284659
:10579800FFF786FD002840F08B800DF13601284682
:1057A8000E9FFFF7C5FD064600287CD1BDF83630B0
:1057B800434540F2828001260696BDF836304345BF
:1057C80060D2A3EB080383EAE372A2EBE3729DF8CD
:1057D8001860099205F592734FF0030B0793079B26
:1057E80018689B881090ADF844303A460FAB0621F4
:1057F8005046FFF70CFD0F9F7B1C56D007F1B400F5
:10580800FFF728FD069B98423CD10BF101033A466D
:1058180048460893FFF728FD002849D149462846FD
:10582800FFF734FD002843D10DF136012846FFF774
:105838007FFD00283CD1BDF83620A2EB0803002BE1
:10584800B8BF5B42424516D9099A934218D910A9A4
:105858002846FFF71BFD079A079903461098106022
:10586800BDF844208A806BB11C46204613B0BDE8C1
:10587800F08F013778E7DDF820B009930137AEE7FC
:10588800DDF820B00A9BC3F800B00B9B1E70012303
:1058980085F815310A9B1B6885F813310B9B1B781B
:1058A80085F81431E1E70446DFE76FF03104DCE7FF
:1058B8000446DAE70026B3467EE7012383460693CB
:1058C8007BE737B5002304468DF807304FF4FA65B7
:1058D8000DF107012046FFF760FC58B99DF8073025
:1058E800012B07D0013D03D0204601F0E5F9EFE791
:1058F8006FF0060003B030BD02464FF0804393427C
:1059080002D8002013B970479B08F8E7C1189142E4
:105918004FEA50009CBFC018521A9B08F2E773B5B3
:1059280000228321054601F033F9044688B94FF473
:10593800FA660DF107028321284601F04BF99DF81C
:1059480007300343DBB204461BB9013EF1D16FF0C7
:10595800060401228321284601F01AF9204340B2A7
:1059680002B070BD2DE9F04F90F8F06091B04FF0A3
:105978000009072ECDE9079904460F4600F0A282D8
:105988000122802101F004F901228046FF212046EE
:1059980001F0FEF84A4648EA00084946204601F068
:1059A800F7F84FFA88F848EA00080622FF2120464F
:1059B80001F0EEF84FFA88F848EA00080DF11502F0
:1059C8008321204601F006F99DF815204FFA88F842
:1059D80048EA000842F004028321204601F0D8F882
:1059E8004FFA88F848EA00080722FF21204601F00C
:1059F800CFF84FFA88F80122812148EA00082046AA
:105A080001F0C6F84FFA88F848EA0008204601F085
:105A180053F94FFA88F848EA000801228021204605
:105A280001F0B6F84FFA88F848EA000517F0010BBC
:105A38006DB200F01E82F20700F11E826B229421E3
:105A4800204601F0A5F880462046FFF768FF06AA21
:105A580048EA00089021204601F008F945EA0805BF
:105A6800069B6DB22422942105432046C3F3062ADF
:105A7800C3F3C03901F08CF86DB205432046FFF737
:105A88004EFF6DB2054306AA9021204601F0EEF8BC
:105A9800069B6DB21BBA2522942105432046099323
:105AA80001F076F86DB205432046FFF738FF6DB276
:105AB800054306AA9021204601F0D8F8069B6DB24E
:105AC8001A0E05431B0C6DB28DF828208DF829306D
:105AD80017F00203029300F0DB8016F0020840F092
:105AE800D78002229421204601F052F801902046E6
:105AF800FFF715FF019B0DF1160203439021204685
:105B08001D4301F067F86DB27B22942105432046BE
:105B180001F03EF86DB205432046FFF700FF6DB275
:105B280005430DF117029021204601F053F86DB29C
:105B3800772294210543204601F02AF86DB20543E7
:105B48002046FFF7ECFE6DB2054306AA90212046D9
:105B580001F08CF8069B5A0E8DF82C20C3F3864270
:105B68008DF82D20C3F3C6228DF82E206DB2C3F315
:105B78000612DB0003F07803942105438DF82F20EB
:105B8800204678228DF8153001F002F86DB20543F1
:105B98002046FFF7C4FE6DB2054306AA90212046B1
:105BA80001F064F8069B9DF8152002EB53728DF8FE
:105BB8003020C3F386528DF83120C3F3C6328DF8F6
:105BC8003220C3F306228DF833206DB2C3F34602A8
:105BD8009B0103F04003942105438DF834202046AF
:105BE80079228DF8153000F0D3FF6DB205432046B9
:105BF800FFF795FE6DB2054306AA9021204601F0F5
:105C080035F8069B9DF8152002EB93628DF8352038
:105C1800C3F3C6428DF83620C3F306328DF8372019
:105C28006DB2C3F346129B0003F07C039421054335
:105C38008DF8382020467A228DF8153000F0A8FF1C
:105C48006DB205432046FFF76AFE6DB2054306AA0A
:105C58009021204601F00AF8069B9DF815208DF842
:105C68003E8002EB93728DF83920C3F3C6526DB2B1
:105C78008DF83A20C3F3064205438DF83B20C3F361
:105C88004622C3F386036DB28DF83C208DF83D3073
:105C980017F00403019300F0F180730700F1EE8020
:105CA8007B229421204600F073FF80462046FFF7B0
:105CB80036FE07AA48EA00089021204600F0D6FFE1
:105CC80045EA08084FFA88F848EA00057C2294213A
:105CD800204600F05DFF6DB205432046FFF71FFE2A
:105CE8006DB2054308AA9021204600F0BFFF6DB2AF
:105CF800732294210543204600F04AFF6DB2054304
:105D08002046FFF70CFE6DB2054306AA90212046F7
:105D180000F0ACFF069B6DB21B0274229421054370
:105D280020461FFA83F800F033FF6DB20543204682
:105D3800FFF7F5FD6DB2054306AA9021204600F055
:105D480095FF6DB29DF81B307522942105432046BE
:105D580043EA080800F01CFF6DB205432046FFF730
:105D6800DEFD6DB2054306AA9021204600F07EFFB5
:105D7800069B6DB21B029BB27622942105432046F6
:105D8800039300F005FF6DB205432046FFF7C7FDFA
:105D98006DB2054306AA9021204600F067FF6DB258
:105DA8009DF81B20039B05436DB2134300228121FC
:105DB8002046039300F0ECFE06220543FF2120460F
:105DC80000F0E6FE6DB205430DF115028321204671
:105DD80000F000FF9DF815206DB2054302F0FB02AC
:105DE8008321204600F0D4FE6DB205430122FF2135
:105DF800204600F0CDFE6DB2054301220021204669
:105E080000F0C6FE6DB205430022FF21204600F0D7
:105E1800BFFE6DB2054300228021204600F0B8FE87
:105E28006DB205436DB2039BFDB9BBF1000F29D1DB
:105E3800029AAABB019AAAB1720713D4079AC4F8A6
:105E48001821089AC4F81C214FEA4822C4F82021D6
:105E58003BB1A3F5C8534FF47A7253431B095B4215
:105E68001BB2E3603E4384F8F060284611B0BDE8F9
:105E7800F08FD946DA462BE6CA4629E64FF00008E5
:105E8800434693E7F007D3D40998BDF8282084F84F
:105E980013A184F81491C4F82A01A4F82E21C7E7A5
:105EA800B107C7D49DF8162084F8F1209DF8172073
:105EB80084F8F2200BA904F1F30002930DF068FEB8
:105EC800029BB7E74D46D0E750B10138002330F0C8
:105ED800FF019AB203F1010303D100EB022080B263
:105EE80070474008F3E7C3B2000A03FA00F0013034
:105EF80070470000084B5A434FF47A7302F5FA7260
:105F08004FF4FA60B2FBF0F0B2FBF3F203FB0100CE
:105F1800B0FBF2F0704700BF002F3A00064B5A431F
:105F28004FF47A7002F5FA72B2FBF0F24A4302F5C6
:105F3800FA72B2FBF0F07047002F3A002DE9FF41EA
:105F480002294FF00005074616468DF80350ADF8B4
:105F580004501CD80DF102022946FEF7A1FB0446A5
:105F680030B90DF103024621384600F033FE0446ED
:105F78009DF80300FFF7B7FF81B29DF8022038466D
:105F8800FFF7CCFF3060204604B0BDE8F08103295C
:105F980018D10DF102022946FEF782FB04460028BB
:105FA80046D101460DF102023846FEF779FB044658
:105FB80028B901AA5121384600F038FE0446BDF838
:105FC8000400D7E7042935D102A9FEF7BDFB9DF8E7
:105FD8000B30ABB10DF1020229463846FEF760FBE3
:105FE800044658B901AA5121384600F01FFE04465C
:105FF800BDF80400FFF777FF85B214B1002015E063
:106008001D460DF1020201213846FEF749FB044600
:106018000028F3D10DF106027121384600F006FE82
:106028000446BDF80600FFF75EFF80B2401BA3E7F9
:106038002846A7E728462C46A4E7F0B5022985B0EC
:10604800054616461ED80DF105020021FEF728FB6D
:106058000446A0B99DF8052031462846FFF74AFFB7
:1060680083B2B3F5807F9ABF00F1FF32D2B2FF222C
:10607800A5F8D8204621284600F08AFD0446204687
:1060880005B0F0BD03291FD10DF105020021FEF76F
:1060980007FB9DF80520314604462846FFF72AFFEE
:1060A80080B2FFF711FF0246ADF80600A5F8D80048
:1060B800002CE4D15121284600F07AFD044600283E
:1060C800DDD1C5F8E460DAE7042939D102A9FEF781
:1060D8003BFB9DF80B70B7B10DF105020021284676
:1060E800FEF7DEFA04460028C9D10DF10602512157
:1060F800284600F09BFD0446BDF80600FFF7F3FEB6
:1061080087B2002CBBD10DF1050201212846FEF70C
:10611800C7FA04460028B2D19DF805203146284622
:10612800FFF7E8FE3844FFF7CFFE71210246284604
:1061380000F03EFD04460028A1D1C5F8DC609EE7CA
:106148006FF003049BE7F0B585B000238DF80330AA
:10615800D30705460F46164605D439B9A2F10C03F4
:10616800DAB2062A11D96FF00300E6E0012921D13D
:10617800A2F10803DAB2062AF5D8062B1AD8DFE806
:1061880003F03B1969198A199D00062B12D8DFE81C
:1061980003F004112D112F11310018225721284620
:1061A80000F0F6FC08225621284600F0F1FC0028F1
:1061B80040F0C3807408013CE4B2002F00F09180E5
:1061C800012FD0D101AA04212846FFF7B7FE50B904
:1061D80022467021284600F0DBFC20B9019A0421F0
:1061E8002846FFF72AFF85F8E06099E03022D5E7D6
:1061F8004022D3E75022D1E71022482100F0C8FC02
:1062080008224721284600F0C3FC02220446322116
:10621800284600F0BDFC0C2204433021284600F03B
:10622800B7FC64B204430122FF21284600F0B0FC09
:1062380064B2044364B230223021284600F0A8FC3E
:1062480000220443FF21284600F0A2FC64B2204348
:1062580040B2ACE72822482100F09AFC08224721E6
:10626800284600F095FC032204463221284600F017
:106278008FFC044364B209223021284600F088FCD0
:1062880001220443FF21284600F082FC64B2044343
:1062980064B22022D0E73822482100F079FC082295
:1062A8004721284600F074FC032204463221284680
:1062B80000F06EFC044364B20822DDE74822114670
:1062C80000F066FC08224721284600F061FC032202
:1062D80004463221284600F05BFC044364B20722DE
:1062E800CAE702AA03212846FFF728FEB0B903AA85
:1062F80002212846FFF722FE80B92246502128466F
:1063080000F046FC50B9029A03212846FFF795FE93
:1063180020B9039A02212846FFF78FFE85F8E86026
:1063280058B969692846FEF7B7F930B9024601231A
:106338000DF103012846FFF73CF905B0F0BD13B590
:10634800144629B1012910D06FF0030002B010BD26
:106358000DF10702502100F03DFC0028F6D19DF810
:10636800073001335B002370F0E70DF1070270215D
:10637800F1E7F0B5002385B04FF4FA62CDE90023C8
:1063880044F61F63994206460F4604D86FF003058A
:10639800284605B0F0BD02A9FEF7D6F90546002843
:1063A800F6D19DF809209DF8083013439DF80A207E
:1063B8001343A7F636341BD06A4602213046FFF74E
:1063C800BDFD00283BD19DF808302BB1009B03F29E
:1063D8004E239C42DAD9E41A9DF80A3023B3009B75
:1063E80003F2B223B4EB430F4FEA4302CED9A41A07
:1063F8009DF80B305BB101AA03213046FFF79EFDE3
:10640800019B03F52573A342C0D2C0B9E41A9DF8D5
:106418000C30002BBCD0A4F2262204213046FFF712
:106428000CFE77610546B3E79DF80930002BDFD0F5
:10643800009B03F525739C42A8D9E41AD8E70546C2
:10644800A6E770B54FF4FA6286B00023CDE90223BF
:1064580040F636330B600C4604A90646FEF774F97D
:106468000546002836D19DF811209DF810301343B9
:106478009DF81220134319D002AA02213046FFF7D3
:106488005DFD002840D19DF810302BB1029B03F22E
:106498004E222368134423609DF81230EBB1029B0F
:1064A80003F2B222236803EB420323609DF8133002
:1064B800EBB99DF814305BB101AA04213046FFF70F
:1064C8003DFD019B03F22622236813442360D8B9BB
:1064D80023687361284606B070BD9DF81130002B03
:1064E800E4D0029B03F5257223681344DDE703AA71
:1064F80003213046FFF722FD039B03F5257223682D
:10650800134423600028D4D00546E3E72DE9F74378
:10651800002406460D46204615F80480B8F1000F01
:1065280000D010B103B0BDE8F083671CB8F1FF0FCD
:1065380015F8079029D1A71CEB5DB9F1030F36D8E0
:10654800DFE809F0020B131B271D2C44E27802EB4D
:106558000323A6F834313C46DEE7271D2C44E278B5
:1065680002EB0323A6F83631F5E7271D2C44E27821
:1065780002EB0323A6F83831EDE7271D2C44E27817
:1065880002EB0323A6F83C31E5E7B8F1040F0ED877
:1065980002344246291901A80DF007FB434601AA17
:1065A8004946304604EB080700F0BEFAD3E76FF01F
:1065B8000300D0E773B500230E4613600DF1070101
:1065C80005461446FEF7F7F840B99DF807302BB199
:1065D800B38A2A6A534380331B0A236002B070BD12
:1065E80013B5CB681360144601AAFFF7E3FF18B987
:1065F8002368019A1344236002B010BDF8B5B0F8BF
:106608005451D0F8580168438030000A0E4645437B
:10661800DDE90717144652B1B60206EB5202B2FB87
:10662800F4F202EB4202524302F50042140C069ABD
:10663800534301F50042120C06200332B2FBF0F27C
:10664800C2EBC202B2F5803F38BF033103F5004305
:106658003EBFB1FBF0F1C1EBC10101F500414FEACA
:10666800134334BF090C1B4903FB03F338BF4943E9
:1066780003EB57030B44B3FBF7F39B03FE2205F12F
:1066880020007F33B3FBF2F35C434FF47A7704F5D1
:10669800FA748009B4FBF7F42401FFF72DF904F527
:1066A800FA74BC4228BF4FF4FA63064629BFB4FB0C
:1066B800F3F300205B19B4FBF7F428BFB3FBF4F045
:1066C800FFF71AF9099B864294BF1E6018600020E4
:1066D800F8BD00BF0000F0FF2DE9F04F91B0CDE903
:1066E8000723036A0E930B6909930546CB680B933E
:1066F8000F460FAAFFF774FF0EAA39462846FFF780
:1067080059FF58BB0F9C95F8E0B0D5F8DC300593DD
:106718004FF47A7606FB04F101F5004104910E99D5
:106728000A910499D5F8E4300693BBF1080F04F1F7
:1067380080040CBF0223032324F0FF0A090C95F8F8
:10674800E820DFF8A081CDF83CA00C9109D1079B87
:10675800C3F80080089BC5F84081186011B0BDE8F7
:10676800F08F06990D932846FFF7C4FB5A46059902
:1067780081462846FFF7BEFB0D9B5B490C9A814476
:1067880003FB09F94FEAC92940F2776309F5FA7959
:10679800240AB9FBF6F903FB09F909F5FA79B9FBFB
:1067A800F6F909FB04F404F18003099C74430C40D6
:1067B800B4FBF2F44D4A1B0A944228BF1446012B3D
:1067C80038BF01230C204FF4167258435443FFF787
:1067D80093F83B7E3A894FEA400B002B7FD1424920
:1067E800049B0B4003F5FA71414B5A4341F25C2379
:1067F800B2FBF3F20A9B7343B3F5481F28BF4FF46B
:106808004813A1EB4303B1FBF6F1B3FBF6F31B020C
:10681800B3FBF1F63602C6F58036564306F5004658
:10682800360C06F5803676087643B60B4FF448707A
:10683800704304F5004300F500401B0C5B43000C5B
:1068480000FB0030FFF758F803046422323341F2AA
:106858008837B3FBF2F340F6B532B3FBFBF302FB28
:106868000377244B9F429CBF42F21073B7FBF3F7A8
:10687800DDE90532134403F5FA734FF47A7B4FF4DC
:10688800FA62B3FBFBF0B3FBF2F202F5C812B2FBFB
:10689800F0F088BF4FF47047FFF72EF8000200F5BC
:1068A800FA70B0FBFBF0404307FB0700FFF724F842
:1068B8000BFB00F0079B0B9A404528BF4046186029
:1068C800089BC5F84001CDE902934FF44873009343
:1068D8000194334651462846FFF790FE3EE74FF4B1
:1068E8008036A3E7AE878F020000FFFF666666006A
:1068F8009A9906000F279F242DE9F04F8BB00027A7
:1069080011F0780FDDE914B80446019299468DF824
:106918000E708DF80F708DF810708DF81170ADF83D
:1069280012700997C1F3C30A00F0AF80AAF10503FA
:10693800DBB20A2B01D86B4AD75C0DF10E0200219D
:106948002046FDF792FF9DF80E500646D5B1002867
:1069580040F09D8009AB05AA59462046FFF7BCFECA
:10696800002840F09680099BABF80A30014606AA39
:106978002046FDF7B3FF069D25B1059B9D422CBF20
:106988000025012520B904AA02212046FDF76DFF44
:106998009DF8106026B300287DD107AA0221204661
:1069A800FDF79CFF88B90122FF21204600F0F0F88E
:1069B80058B90DF11202B621204600F037F920B976
:1069C8000246FF21204600F0E3F8BDF81230079E8A
:1069D8005B02C4F848311EB19E422CBF0026012636
:1069E80028B90DF1110203212046FDF73EFF9DF85D
:1069F800113093B1002873D1B9F1000F03D0019B76
:106A08001B02B3FBF9F908AA03212046FDF766FF2C
:106A1800089B4B4594BF0023012320B9012F3CD18B
:106A2800FF2288F8002098F800200AB9ABF80A205D
:106A38000DF10F02012120460193FDF716FF08BB57
:106A48009DF80E20019B002A08BF0125BAF1040F0A
:106A580018BF9DF80F2084F82E501ABFB2FA82F2A0
:106A68005209012284F82F209DF81020002A9DF851
:106A7800112008BF0126002A08BF012384F83060CE
:106A880084F831300BB0BDE8F08F012755E70025B9
:106A98007EE735467CE70026A9E70AF1FF32092A96
:106AA8000AD8DFE802F0050505090907090B070BF5
:106AB8000522B6E70422B4E7012E01D10322B0E78C
:106AC800BAF1040F01D0012B01D10222A9E7012D4F
:106AD8001BBF002388F8003088F800502B46A2E737
:106AE8000023A0E71A3E010807B502F10A03009344
:106AF80093B20A4690F86011D0F85C0101F0B2FB3D
:106B080003B05DF804FB13B502F10A0390F8604185
:106B18000093D0F85C0193B20A4644F0010101F0F9
:106B280037FC02B010BD00003F2BF8B50E460546F5
:106B380011461C4611D80A4F38461A4600F8016B10
:106B48000DF033F8621C39462846FFF7CDFF0028C0
:106B58000CBF00206FF01300F8BD6FF00300FBE7D7
:106B6800000F002073B515468DF8071001220DF1AE
:106B7800070104461E46FFF7B7FF28B932462946E3
:106B88002046FFF7C0FF08B16FF0130002B070BDD8
:106B980008B5064B19705A7019460222FFF7A4FF70
:106BA800002814BF6FF01300002008BD000F00205C
:106BB80008B5074B1970110A59709A7019460322C3
:106BC800FFF792FF002814BF6FF01300002008BDE4
:106BD800000F002037B515468DF8071001220DF17A
:106BE80007010446FFF780FF28B9012229462046FD
:106BF800FFF789FF08B16FF0130003B030BDF7B598
:106C080015460DF1070206460F461C46FFF7E2FF40
:106C180050B99DF807301D4044EA05023946304610
:106C28008DF80720FFF7B4FF03B0F0BD73B5144625
:106C38008DF8071001220DF107010646FFF754FFF2
:106C480018B16FF0130002B070BD074D022229463B
:106C58003046FFF758FF0028F3D12A786B7803EB0A
:106C680002232380EFE700BF000F002073B514460E
:106C78008DF8071001220DF107010646FFF734FFD2
:106C880018B16FF0130002B070BD0A4D04222946F6
:106C98003046FFF738FF0028F3D16B782A781B04B9
:106CA80003EB0263EA781344AA7803EB0223236018
:106CB800E9E700BF000F002008B50220FBF71CFF22
:106CC800002008BD7047000010B5032000F072FCDA
:106CD80001F0AAFD064B18600F20FBF703FF0446DE
:106CE80018B9FBF770FD204610BD0124FBE700BF73
:106CF800280800204FF0E022136923F002031361F3
:106D080070474FF0E022136943F0020313617047A4
:106D1800014BD3F8900570470070FF1F014BD3F863
:106D2800940570470070FF1F014BD3F89805704712
:106D38000070FF1F024A536823F001035360704735
:106D4800002004E0024A536823F0020353607047AE
:106D5800002004E0024A536823F00403536070479C
:106D6800002004E08068C0F380007047F7B5002376
:106D780001930446002800F0E980856D25B9FBF7EA
:106D88006DF8E56584F8545023689A68D00040F19E
:106D9800A1809A68D10000F1B480A26D42F010027F
:106DA800A265E26D42F00102E26501251846FFF78F
:106DB800D9FFA26D02F01002024340F0C980A26D13
:106DC800206922F4817242F00202A2659A68D20711
:106DD8005DD4226BA67E94F82CC0003A18BF01221D
:106DE8001703D4E902120A43217E42EA8132617E06
:106DF80042EAC13242EA4632002842EA4C02B4BFB3
:106E080020F000414FF400113A430A4394F820104F
:106E1800012903D1002E76D142F48032616A21B172
:106E2800A66A01F4E07131430A43D968E66C21F49B
:106E3800FE3121F4FF711143D96094F83C20616858
:106E4800012A01F0404C4CEA060609D1D4E9102782
:106E58003A433243A66C324342EA0C0242F001063E
:106E68001F693E4A3A4032431A6121F00042B2F1AA
:106E7800804F0CD0B1F1004F09D0394ED6F8082711
:106E880001F4701122F470120A43C6F808275A69EF
:106E9800666BA16B22F0070232435A615A6922F0ED
:106EA800700242EA01125A61002835D19A6A62F0EA
:106EB8000F029A625B6903F007039E423CD10023EC
:106EC800E365A36D23F0030343F00103A36528469C
:106ED80003B0F0BD9A68234922F0104222F017024D
:106EE80042F080529A60204A1268B2FBF1F20132F5
:106EF80052000192019A002A3FF44BAF019A013ADD
:106F0800F7E7002552E7A16D41F02001A165E16D89
:106F180041F00101E16581E7B0F5001FCAD19A6A25
:106F2800E269013A92006FF00F0102F01C0201FAC7
:106F380002F2216E0A43BCE7A36D23F0120343F06B
:106F48001003A365E36D43F00103E3650125BEE784
:106F5800A36D43F01003A365F8E700BF02FCFF1F11
:106F680000200140400D030028080020F8B54569BD
:106F7800082D04460E460AD00368DB68D80705D5F5
:106F8800A36D43F02003A3650120F8BD0425FBF79A
:106F9800ABFD074623681A682A4221D0A26D42F445
:106FA8000072A265DA6812F4406F14D1A27E92B919
:106FB8001A6812070FD51846FFF7D4FE28BB5A687F
:106FC80022F00C025A60A26D22F4807222F00102B3
:106FD80042F00102A265207E00BB0C221A60D4E7B1
:106FE800711CD8D0FBF780FDC01BB04201D8002E21
:106FF800D0D123681B682B40CCD1A26D84F85430C3
:1070080042F00402A2650320BFE7A26D42F020020D
:10701800A265E26D42F00102E265DCE70020B4E718
:107028000368186C70470000F7B50023019390F8C7
:107038005430012B044600F0C58005680669012319
:1070480080F854302846FFF78DFE002840F0B480C1
:10705800D1E90020022826F0040300F08280B3F171
:10706800004FC2F3110E13D1AB6A43EA0E03AB62B1
:107078008B68686903EA022323F07C4323F0FF034B
:1070880020EA02210B43002A6B6126DB002055E031
:10709800236E00F01F074FF00F0C0CFA07FC6FEA85
:1070A8000C0623EA0C0CBEF1000F11D1C2F3846365
:1070B800BB4043EA0C0323668008E3690130984229
:1070C800D6D8A86AC2F38363BB4006403343CEE7F1
:1070D80092FAA2F3B3FA83F3EAE73B493B48D1F8C3
:1070E8000837824203F0E07519D11B02CED4D1F8DB
:1070F800083723F0E0732B4343F40003C1F8083743
:10710800334B1A68334BB2FBF3F20C2302FB033305
:107118000193019B002BB9D0019B013BF8E72E4856
:10712800824210D113F08070B0D1D1F8083723F023
:10713800E0732B4343F08073C1F80837002384F8C9
:10714800543003B0F0BD254882429FD113F480002B
:107158009CD1D1F8083723F0E0732B4343F4800324
:10716800EAE7B3F1004F01BFAB6AC2F311018B43E9
:10717800AB62002A8ADA154813498242D1F80837E7
:1071880009D1D1F8082703F0A07322F0E072134365
:10719800C1F808377AE71048824204D1D1F80827A5
:1071A80003F44003F1E70D4882427FF46FAFD1F852
:1071B800082703F0C073E8E7A26D42F02002A26539
:1071C8001846BBE70220BCE700200140001000B0D1
:1071D80028080020400D0300004000B8002000B43B
:1071E800026838B504461046FFF7BCFD08B9002010
:1071F80038BD9368990707D4936823F0004323F0B8
:10720800170343F010039360FBF76EFC05462368F1
:107218009B685B07EBD5FBF767FC401B0228F6D998
:1072280023689B685A07F2D5A36D43F01003A36542
:10723800E36D43F00103E3650120D9E773B500234B
:10724800026801939368DD07044602D5002002B066
:1072580070BD9168214B194209D0A36D43F010030A
:10726800A365E36D43F00103E3650120EFE793684D
:1072780023F0004323F0170343F001039360184BF6
:10728800D3F8083718021CD4637E012BDED0FBF735
:107298002BFC144E054622681368DB07D6D4936886
:1072A800D9075FBF9368334043F001039360FBF74E
:1072B8001BFC401B0228EED923681B68DA07EAD4B6
:1072C800CBE7094B094A1B68B3FBF2F3013301937F
:1072D800019B002BD8D0019B013BF8E717000080E9
:1072E80000200140E8FFFF7F28080020400D030030
:1072F80038B504460068FFF735FD054620BB94F80D
:107308005430012B20D0012384F854302046FFF755
:1073180095FFB0B9A36D226823F4706323F00103CD
:1073280043F48073A3651C23E065136084F854005C
:10733800936823F0004323F0170343F0040393609A
:1073480038BD84F85450FBE70220F9E7026838B5E5
:10735800936891680446C80701D4002038BD99078E
:10736800FBD4936803F00503012B19D1936823F02C
:10737800004323F0170343F00203936003231360D1
:10738800FBF7B2FB054623689B68DB07E5D5FBF7EF
:10739800ABFB401B0228F6D923689B68DA07F2D5B5
:1073A800A36D43F01003A365E36D43F00103E365A8
:1073B8000120D3E770B5044600284BD0836D43F015
:1073C80002038365FFF70CFF054668B92046FFF7FF
:1073D800BDFF054608B90123A3652268936823F019
:1073E800104323F01703936023685A6822F46772E6
:1073F80022F003025A6040F29F321A60D968164A96
:107408000A40DA601A6922F040421A615A6922F089
:1074180007025A611A6A02F0F0221A625A6A02F0E6
:10742800F0225A62DA6A02F0F022DA629A6A0B4AA9
:1074380000269E62D2F8083723F0FE73C2F8083798
:107448002046FAF71FFDE6652666A66584F85460AF
:10745800284670BD0125FBE700023E83002001405D
:1074680010B590F85430012B044615D0012380F84C
:107478005430FFF7B5FE58B92046FFF767FF38B913
:10748800A36D23F4807323F0010343F00103A36584
:10749800002384F8543010BD0220FCE7F7B5002320
:1074A800019390F85430012B04467FD0012380F8D3
:1074B8005430FFF74BFF23689A6812F00102054623
:1074C80007D0A36D43F01003A365002384F854305C
:1074D8002DE0A16D364F21F4817141F00201A165C3
:1074E800DE68D96826F4FF4626F07C0621F40041C0
:1074F800360421F00301360CD96008209968394018
:1075080041F0004199609968002913DA0199013125
:1075180001910199B1F52E3FF5D3A36D23F0120324
:1075280043F01003A365002384F85430012528464E
:1075380003B0F0BDD3F8B410013801F07F010A445C
:10754800DCD199681A48014041F001019960D3F8EB
:10755800B41021F07F0141EAD202C3F8B4209A683E
:10756800024042F002029A60FBF7BEFA074623681F
:107578009A68D20708D4DA683243DA60A36D23F038
:10758800030343F001039FE7FBF7AEFAC01B022891
:10759800EDD923689B68D907E9D5A36D43F010039B
:1075A800A365E36D43F00103E365BFE70225BEE78A
:1075B800E8FFFF7F0749CA6822F4E0620302120469
:1075C80003F4E063120C134343F0BF6343F4003346
:1075D800CB60704700ED00E0164B30B5DC68C4F3B3
:1075E8000224C4F10703251D042B28BF0423062DFC
:1075F8004FF0FF358CBF033C002405FA03F321EA62
:107608000303A54022EA0502A340002843EA020337
:10761800ACBF00F16040084A4FEA0313B8BF00F05E
:107628000F00DBB2AABF00F56140135480F80033A5
:1076380030BD00BF00ED00E014ED00E0002807DBDE
:10764800044A4109012300F01F00834042F8213019
:10765800704700BF00E100E000280CDB4309064941
:1076680000F01F0020330122824041F82320BFF39D
:107678004F8FBFF36F8F704700E100E070B5D0E91E
:1076880013456560446D14B1D0E916456560D0E9CD
:10769800105404F01C060124B4406C600468636054
:1076A8008368102B0BBFA260A160E160E26070BD2F
:1076B8000268416CD3B210B5083B1424B3FBF4F351
:1076C8000B4CA24288BF0B4A21F0030199BF01F17C
:1076D800804202F50232521807338264064AC264B5
:1076E80003F01F03012202FA03F3036510BD00BF74
:1076F800070402401C0802408008024038B50028F0
:107708005ED002682F4B9A424FF014014CD82E4B92
:107718001344B3FBF1F32D499B00C0E91013022376
:1077280080F825301368056923F4FF4323F07003BC
:107738001360D0E9024323432B43456911682B4367
:1077480085692B43C5692B43056A2B430B4313609B
:10775800FFF7AEFFB4F5804F04BF002343604268D3
:10776800816C02F07F030B60D0E91314013A032AFD
:107778004C6020D8164A174981651A44013B92008B
:10778800012103F0030301FA03F300214265C365F5
:107798001160114A536400230122C36380F8243026
:1077A80080F82520184638BD0C4B1344B3FBF1F381
:1077B8000B499B00B1E70023C0E91533C365EAE72D
:1077C8000120F0E707040240F8FFFDBF0000024077
:1077D8003F8200104009024000090240F8FBFDBF4B
:1077E8000004024038B5002841D00268136823F02D
:1077F800010313601F4B9A424FF0140130D81E4BFF
:107808001344B3FBF1F31D499B00C0E91013012495
:1078180003F01C0304FA03F3002515604B60FFF71F
:1078280047FF836C41681D60D0E913325A604A1ED5
:10783800032A06D8124B0B449B0094401D60114B41
:107848005C640023C363C0E91533C0E90B33C0E9A6
:107858000D33C36580F8253080F82430184638BDCC
:10786800094B1344B3FBF1F308499B00CDE7012012
:10787800F5E700BF07040240F8FFFDBF0000024023
:107888003F82001000090240F8FBFDBF00040240DF
:1078980070B590F82450012D04463BD090F825602F
:1078A8000125AE4280F824504FF000062CD1022565
:1078B80080F825500568C6632E6826F001062E60FC
:1078C800FFF7DCFE036BBBB12B6843F00E032B60A4
:1078D800A36C1A68D20342BF1A6842F480721A6015
:1078E800636D1BB11A6842F480721A602B6843F00A
:1078F80001032B60002070BD2B6823F004032B606C
:107908002B6843F00A03E2E78023C36380F824600E
:107918002846F0E70220EEE7034640B190F825201C
:10792800022A06D00422C263002280F82420012003
:1079380070470268806C116821F00E0111600168BF
:1079480021F480710160116821F001011160D3E90F
:10795800100202F01C0101228A404260D3E913217F
:1079680051605A6D32B1116821F480711160D3E908
:10797800162151600122002083F8252083F8240075
:10798800704710B590F82530022B03D00423C36349
:10799800012010BD03681A6822F00E021A601A68E6
:1079A80022F001021A60826C136823F4807313605A
:1079B800D0E9101303F01C02012393404B60D0E977
:1079C80013325A60436D33B11A6822F480721A6018
:1079D800D0E916325A60012380F82530836B0024E1
:1079E80080F8244013B198472046D2E71846D0E7DC
:1079F80070B4426C046C036826681D6802F01C02AF
:107A08000421914031420FD015F0040F0CD01A68B0
:107A180092065EBF1A6822F004021A60036B616066
:107A2800002B33D070BC184702219140314217D047
:107A380015F0020F14D01A68940606D41A6822F0BA
:107A48000A021A60012280F82520114A93428CBF4D
:107A5800104B114B5960002380F82430C36ADFE7CC
:107A680008219140314211D029070FD5196821F01A
:107A78000E011960012303FA02F26260C36380F801
:107A88002530002380F82430436BC9E770BC704769
:107A98008000024000040240000002400A4A536984
:107AA80043F4802330B55361EFF3108472B600239A
:107AB800CD58C5500433B3F5807FF9D11369DB0382
:107AC800FCD484F3108830BD00400058064B5A6936
:107AD800002ABFBF054A9A6002F188329A60BABF8D
:107AE8005869C00F002070470040005823016745BF
:107AF800044B5A6942F000425A615869C043C00FAA
:107B0800704700BF0040005870B50546FAF7ECFF13
:107B1800124E04463369D90313D43369DA0744BFD4
:107B2800012232614CF2FA32134011D10B4E306906
:107B380010F480200BD0FAF7D7FF001BA842F6D329
:107B480004E0FAF7D1FF001BA842E3D3032070BD7D
:107B5800024A1361024A01205360F8E700400058C6
:107B6800400F00202DE9F041184D98462B78012B45
:107B780006460C46174626D001232B704FF47A7020
:107B880000236B60FFF7C0FFA0B9012E16D1104A81
:107B9800536943F0010353612760BFF36F8FC4F843
:107BA80004804FF47A70FFF7AFFF094A536923EA5C
:107BB8000603536100232B70BDE8F0813946204647
:107BC800FFF76CFFEDE70220F6E700BF400F00204B
:107BD80000400058054A536923F47E7343EAC00005
:107BE80040F4803040F00200506170470040005877
:107BF8002DE9F041234F3B78012B054688463FD0BD
:107C080001233B704FF47A7000237B60FFF77CFF01
:107C1800044688B92B68042B13D11B4A536943F4D3
:107C2800803343F0040353614FF47A70FFF76CFF1D
:107C38000446154B1A681B6800233B702046BDE8B4
:107C4800F0814FF0FF33C8F800306E68D5E9013293
:107C58001344B3420AD93046FFF7BCFF4FF47A7099
:107C6800FFF752FF50B1C8F800600446064A53694E
:107C780023F47E7323F002035361DAE70136E5E764
:107C88000224DBE7400F0020004000582DE9F04FA8
:107C9800524C00234FF00F090A6832FA03F501D15C
:107CA800BDE8F08F012505FA03F818EA020200F092
:107CB8008E804E68032706F003054FEA430E07FA45
:107CC8000EFC6F1E012F6FEA0C0C32D8876807EA8A
:107CD8000C0ACF6807FA0EF747EA0A078760476871
:107CE80027EA0808C6F300179F4047EA08074760D5
:107CF800C76807EA0C088F6807FA0EF747EA08070B
:107D0800022DC76017D14FEAD30800EB880803F0AB
:107D1800070AD8F820704FEA8A0A09FA0AFB27EA04
:107D28000B0B0F6907FA0AF747EA0B07C8F8207028
:107D380001E0032DDCD1076805FA0EF507EA0C0708
:107D48003D4316F4403F056041D023F0030707F197
:107D5800804707F5803703F0030CBD684FEA8C0CA9
:107D68004FF0070E0EFA0CFEB0F1904F25EA0E0EFA
:107D78002FD01B4DA8422ED005F58065A8420CBF18
:107D88000225072505FA0CF545EA0E05BD602568AC
:107D9800D74316F4801F0CBF3D4015432560656826
:107DA80016F4001F0CBF3D4015436560D4F88050A1
:107DB80016F4803F0CBF3D401543C4F88050D4F8FA
:107DC8008450B60354BF3D401543C4F88450013372
:107DD80062E70025D6E70125D4E700BF0008005870
:107DE80000040048374A2DE9F04F00234FF0010AFC
:107DF8004FF0070B4FF00F0931FA03F401D1BDE83A
:107E0800F08F0AFA03FC1CEA010654D023F003049D
:107E180004F1804404F5803403F00307A568BF002B
:107E28000BFA07F8B0F1904F08EA050E45D0264D39
:107E3800A84244D005F58065A8420CBF0225072555
:107E4800BD40754517D1D2F8805025EA0605C2F81D
:107E58008050D2F8845025EA0605C2F88450156887
:107E680025EA06051560556825EA06055560A568E2
:107E780025EA0805A560056803265C0006FA04F4EF
:107E880023FA06F6254300EB8606056003F007058E
:107E9800376AAD0009FA05F527EA050737628568EC
:107EA80025EA04058560456825EA0C054560C5682E
:107EB80025EA0404C46001339EE70025C0E70125D4
:107EC800BEE700BF000800580004004803691942D3
:107ED80014BF0120002070470AB181617047816298
:107EE80070470000044AD168014208B502D0D0604A
:107EF800FBF724FB08BD00BF0008005803689A6917
:107F0800910744BF00229A629A69D2075EBF9A69B4
:107F180042F001029A61704730B5039D04682B4313
:107F280043EA0243064A6068C1F309010B4342EA87
:107F3800555223F0004320EA02000343636030BD3A
:107F4800FF63FF0303682DE9F0419C6914F01004F6
:107F580005460F4616466FD010220024DA61A04667
:107F68002B689A69900661D4B8F1000F35D044F0B7
:107F7800040401202E68B369D90541BF4FF480720B
:107F8800F26144F0010401205A0541BF4FF48062B8
:107F980044F00804F26101209B054FD54FF40073AB
:107FA80044F00204F3612846FFF7A8FF736823F042
:107FB800FF7323F48B3323F4FF7323F001037360FF
:107FC8006B6C23436B64202385F84130002385F8CC
:107FD800423085F84030012032E07A1CC1D0FAF7EF
:107FE80083FD801BB84201D8002FB9D12B6859688E
:107FF80095F8422098690004D2B20AD5490408D4F9
:10800800202A06D05A6842F480425A60FAF76CFD7A
:1080180006462B689B699B06A2D4FAF765FD801B70
:108028001928F6D920244FF0010899E7B8F1000F74
:108038009DD12022DA619AE720469BE70028B2D139
:10804800BDE8F08170B504460D46164623689B6965
:108058009B0701D5002070BD324629462046FFF710
:1080680071FFA0B96A1CF1D0FAF73EFD801BA84247
:1080780001D8002DEAD1636C43F020036364202308
:1080880084F84130002384F8423084F840300120DD
:10809800E1E770B504460D46164623689B695B0701
:1080A8000ED4324629462046FFF74CFF38BB2368DA
:1080B8009A69910625D59A69520703D5228D0AB186
:1080C800002070BD9A6912F010021CBF1022DA61FC
:1080D8004FF0200118BF04226264D9615A6822F067
:1080E800FF7222F48B3222F4FF7222F001025A60EE
:1080F800002384F8411084F8423084F8403001208D
:10810800DFE7FAF7F1FC801BA84201D8002DC4D1A3
:10811800636C43F020036364202384F84130002318
:10812800EBE72DE9F041069F0446884616461D46B2
:108138002268936938EA03030CBF01230023B34282
:1081480001D0002015E06B1CF3D0FAF7CDFCC01B62
:10815800A84201D8002DEBD1636C43F0200363647F
:10816800202384F84130002384F8423084F84030DA
:108178000120BDE8F08170B504460D461646236817
:108188009B699B0601D5002070BD324629462046D2
:10819800FFF7D8FE90B9FAF7A7FC801BA84201D8D0
:1081A800002DECD1636C43F020036364202384F832
:1081B8004130002384F8423084F840300120E3E75E
:1081C80010B5044600284AD090F8413003F0FF0269
:1081D8001BB980F84020FAF77FF9242384F841304E
:1081E80023681A6822F001021A60626822F070623D
:1081F8001A619A6822F400429A60D4E9022101299E
:1082080024D142F400429A605A6842F0007242F463
:1082180000425A60DA6822F40042DA60D4E90421A4
:108228000A43A16942EA0122DA60D4E907210A4334
:108238001A601A6842F001021A6000202023606464
:1082480084F84130206384F8420010BD42F40442AF
:1082580002299A6004BF4FF400625A60D4E70120F3
:10826800F3E700002DE9F347984690F841300A9F5C
:10827800202B04460E46914640F0868090F8403008
:10828800012B00F081804FF0010A80F840A0FAF736
:108298002BFC19230546009052464FF40041204616
:1082A800FFF73FFF18B1012002B0BDE8F087212396
:1082B80084F84130102384F842306064A4F82A809E
:1082C800638DC4F824909BB2FF2B60632F4B26D993
:1082D800FF22228500934FF0807331462046FFF736
:1082E8001BFE638D9BB22A4639462046FBB9FFF731
:1082F80042FF0028D7D123682021D9615A6822F08B
:10830800FF7222F48B3222F4FF7222F001025A60CB
:1083180084F8411084F8400084F84200C4E7628D74
:10832800009392B222854FF00073D2B2D5E7FFF7DF
:1083380089FE0028B7D1636A226813F8011B91628D
:108348006362638D228D013B9BB26385638D013A25
:1083580092B29BB22285002BC3D0002AC1D10095CE
:108368003B4680212046FFF7DCFE00289BD1638D29
:108378009BB2FF2B03D9FF2222850090ABE7628DC9
:10838800009092B22285CEE702208DE7002000807F
:108398002DE9F347984690F841300A9F202B044670
:1083A8000E46914640F0878090F84030012B00F04F
:1083B80082804FF0010A80F840A0FAF795FB192354
:1083C8000546009052464FF400412046FFF7A9FEAB
:1083D80018B1012002B0BDE8F087222384F84130AB
:1083E800102384F842306064A4F82A80638DC4F8AE
:1083F80024909BB2FF2B6063304B26D9FF22228545
:1084080000934FF0807331462046FFF785FD638D5A
:108418009BB22A4639462046FBB9FFF7ACFE002836
:10842800D7D123682021D9615A6822F0FF7222F43B
:108438008B3222F4FF7222F001025A6084F8411054
:1084480084F8400084F84200C4E7628D009392B239
:1084580022854FF00073D2B2D5E7FFF71AFE002845
:10846800B7D123685A6A636A1A70636A228D013326
:108478006362638D013B9BB26385638D013A92B25F
:108488009BB22285002BC2D0002AC0D100953B4662
:1084980080212046FFF745FE00289AD1638D9BB2C4
:1084A800FF2B03D9FF2222850090AAE7628D009056
:1084B80092B22285CDE702208CE700BF002400801D
:1084C80010B590F84120202A0346D4B21CD190F868
:1084D8004020012A18D0242280F841200268106820
:1084E80020F001001060106820F4805010601068BF
:1084F800014311601168002041F00101116083F807
:10850800414083F8400010BD0220FCE710B590F808
:108518004120202A0346D4B21BD190F84020012ADA
:1085280017D0242280F841200268106820F001004A
:108538001060106820F4706040EA01211160116831
:10854800002041F00101116083F8414083F84000A8
:1085580010BD0220FCE70000024A136843F4807350
:1085680013607047000400580D4B10B55B690C464A
:1085780028B99A0507D500F027F820B110BD9B054A
:1085880001D400F019F8074A1369012C23F00403F9
:10859800136101D130BFF1E740BF20BF20BFEDE735
:1085A8000004005800ED00E0024B186800F4C060B9
:1085B800704700BF00040058024A136843F4804320
:1085C80013607047000400580C4A136823F4804372
:1085D80013600B4B1B6832214B430A49B3FBF1F381
:1085E8005169890500D533B9536913F4007F14BF65
:1085F800032000207047013BF2E700BF0004005849
:108608002808002040420F000B4A136823F0070394
:1086180043F002031360094B1A69012842F004026F
:108628001A6105D130BF1A6922F004021A61704735
:1086380040BF20BF20BFF6E70004005800ED00E06F
:108648004FF0B0431868C0F3404070474FF0B04354
:108658001868C0F3400070474FF0B042536823F4E5
:108668007F4343EA0023536070474FF0B0431868D4
:10867800C0F34060704700007FB54FF0B0432C4A0C
:10868800D3F80831C0F3031003F00F0352F8204069
:10869800284A52F82330B4FBF3F4FFF785FF264B42
:1086A800054693E80700B5F5007F04AB03E907002A
:1086B80010D0224B9C4218D303F5B70303F67F531F
:1086C8009C4229D903F5741303F510639C4225D8FD
:1086D80002230BE01A4B9C4207D91A4B9C421BD928
:1086E80003F5370303F5D853F0E7002304AA02EB98
:1086F800830353F80C4C144D2B6823F007032343D2
:108708002B60FAF7F1F906462B6803F007039C4241
:1087180006D1002004B070BD0123E7E70024EAE792
:10872800FAF7E2F9801B0228EED90320F2E700BF2E
:10873800883E0108283E0108F03C0108C0CF6A00C5
:10874800BFEA21013F933402004000584FF0B04384
:1087580010B59A68D96812F00C0205D00C2A4AD1D3
:1087680001F00303012B50D14FF0B0412B480B68A7
:1087780013F0080306D00B6813F0080337D1D1F8BB
:10878800941007E00C68240756BFD1F894300968A4
:10879800C3F3032350F82330002A0CBF18460020E7
:1087A8004FF0B0418A6802F00C020C2A1ED1CA6848
:1087B80002F00302022A2ED0032A06D10B68184AB7
:1087C80013F4801F174B18BF13464FF0B042D06800
:1087D800D168D268C0F306205843C1F302130133AD
:1087E800B0FBF3F0530F0133B0FBF3F010BD0B688F
:1087F800C3F30313CEE7042A0AD0082A05D11B685D
:1088080013F4801304D10748CAE700231846C7E7C2
:1088180003480023C4E7024BD7E700BF883E01089E
:108828000024F4000048E80108B5FFF78FFF4FF077
:10883800B043044A9B68C3F3031352F82330B0FBD8
:10884800F3F008BD283E01082DE9F0410446002850
:1088580053D04FF0B0439D68DE6803689B0605F06F
:108868000C0506F0030668D5026A1DB10C2D46D129
:10887800012E44D1002A40D04FF0B043A16A1A68B3
:10888800170756BFD3F894301B681B0903F0F00391
:1088980099421FD90846FFF7EFFE00282DD14FF067
:1088A800B042136843F0080313601368A16A23F009
:1088B800F0030B431360606AFFF7CEFEFFF7B4FFC7
:1088C800AB4B1860AB4B1868FAF70CF9002834D09A
:1088D800BDE8F0814FF0B042136843F0080313601D
:1088E800136823F0F0030B431360606AFFF7B4FECC
:1088F8000846FFF7C1FE0028E0D00120E8E74FF066
:10890800B043002A54D01A6842F001021A60FAF7FC
:10891800EBF80746FFF79AFE002842D04FF0B04226
:10892800136843F0080313601368A16A23F0F00387
:108938000B431360606AFFF78FFE2368D80748D49B
:108948002368990700F18C8023681E0740F1FA809C
:10895800A3694FF0B046002B00F0E180D6F89430C0
:10896800E16903F01002914200F0C48003F00302B1
:10897800022AC2D0D80740F1B380D6F8943023F049
:108988000103C6F89430FAF7AFF80746D6F89430E2
:10899800990740F1A580FAF7A7F8C31B112BF5D961
:1089A80004E0FAF7A1F8C01B0228B3D903208FE727
:1089B8001A6822F001021A60FAF796F80746FFF7DC
:1089C80045FE0028B9D0FAF78FF8C01B0228F6D95F
:1089D800ECE7082D03D00C2D05D1032E03D16368D5
:1089E800002BADD189E74FF0B043A1681A6822F493
:1089F80080120A431A606268B2F5803F10D11A6883
:108A080042F480321A60FAF76FF80746FFF718FE4B
:108A1800002895D1FAF768F8C01B6428F6D9C5E78D
:108A2800B2F5041F04D11A6842F400121A60E6E78E
:108A3800196821F480311960196821F4001119604E
:108A4800002AE0D1FAF750F80746FFF7F9FD0028A9
:108A58003FF476AFFAF748F8C01B6428F5D9A5E7C4
:108A6800042D236903D00C2D0ED1022E0CD1002B1E
:108A78003FF443AF4FF0B0426169536823F0FE43BF
:108A880043EA016353605FE74FF0B046BBB1336818
:108A980043F480733360FAF727F8074633685A05BA
:108AA80007D57368626923F0FE4343EA0263736083
:108AB8004AE7FAF719F8C31B022BEFD976E73368B0
:108AC80023F480733360FAF70FF8074633685B05C1
:108AD8007FF53AAFFAF708F8C31B022BF6D965E71A
:108AE8004FF0B042E169D2F8943023F010030B4301
:108AF800C2F894304FF0B047D7F8943043F00103F0
:108B0800C7F89430F9F7F0FF0646D7F894309A077B
:108B180018D4F9F7E9FF831B112BF6D946E7D6F8E5
:108B2800943023F00103C6F89430F9F7DDFF0746C7
:108B3800D6F894309B0705D5F9F7D6FFC31B112B40
:108B4800F6D933E72368580754D50B4F3B68D90546
:108B580014D4FFF701FDF9F7C7FF06463B68DA05AD
:108B68000CD4F9F7C1FF831B022BF7D91EE700BF0E
:108B7800280800202C08002000040058E3684FF063
:108B8800B046002B58D023F08003052B02BFD6F83F
:108B9800903043F00403C6F890304FF0B046F9F730
:108BA800A3FFD6F8903043F001030746C6F890308B
:108BB80041F28838D6F890309B0705D4F9F794FF2E
:108BC800C31B4345F6D9F1E6E36823F00403812B80
:108BD8001BD1F9F789FFD6F8903043F08003C6F827
:108BE800903007464FF0B04641F28838D6F89030BA
:108BF800180504D5E06A00284AD1002068E6F9F78C
:108C080073FFC01B4045F1D9D0E6F9F76DFFD6F8E0
:108C1800903023F08003C6F8903007464FF0B046F6
:108C280041F28838D6F890301905E3D5F9F75CFF9A
:108C3800C01B4045F6D9B9E6F9F756FFD6F890308B
:108C480023F080030746C6F8903041F28838D6F8FA
:108C580090301A0516D4F9F747FFD6F8903023F06C
:108C68000103C6F8903007464FF0B04841F2883605
:108C7800D8F890309B07BDD5F9F736FFC31BB34230
:108C8800F6D993E6F9F730FFC01B4045DFD98DE6EA
:108C98000C2D4ED04FF0B04302281A6822F0807293
:108CA8001A6033D1F9F720FF0546FFF7DEFC38BB21
:108CB800D4E90C314FF0B0420B43D0682D49014044
:108CC8000B43E16B0B43216C0B43616C0B43A16BB2
:108CD80043EA0123D360136843F080731360D368B9
:108CE80043F08053D360F9F7FFFE0446FFF7BDFC5D
:108CF800002882D1F9F7F8FE001B0A28F6D955E6B4
:108D0800F9F7F2FE401B0A28CFD94FE6F9F7ECFE37
:108D18000446FFF7AAFC30B94FF0B042164BD168B1
:108D28000B40D360D4E5F9F7DFFE001B0A28F0D921
:108D38003CE601283FF4CCAD4FF0B043226BDB6832
:108D480003F0030191427FF4D8AD616B03F0700228
:108D58008A427FF4D2ADA16B03F4FE42B2EB012F3D
:108D68007FF4CBAD626C03F0604393423FF445AFB0
:108D7800C3E500BF8C80C111FCFFFEEE2DE9F04178
:108D88000D46044610B90120BDE8F081684E3368ED
:108D980003F007038B4216D323689A0727D54FF0B1
:108DA800B047A268BB6823F0F0031343BB60F9F730
:108DB8009BFE0646BB68DB0319D4F9F795FE831BB7
:108DC800022BF7D911E0336823F007030B43336014
:108DD800F9F78AFE0746336803F00703AB42DBD096
:108DE800F9F782FEC01B0228F5D90320CCE72368D7
:108DF800580617D54FF0B0476269D7F8083123F005
:108E08000F0343EA1213C7F80831F9F76DFE064657
:108E1800D7F80831D90305D4F9F766FE831B022B6E
:108E2800F6D9E2E723685A0713D54FF0B047E2684E
:108E3800BB6823F4E0631343BB60F9F755FE0646AD
:108E4800BB689B0305D4F9F74FFE831B022BF7D9A8
:108E5800CBE72368180714D54FF0B0472269BB68E1
:108E680023F4605343EAC203BB60F9F73DFE0646AC
:108E7800BB68590305D4F9F737FE831B022BF7D9D2
:108E8800B3E72368DA070FD4294C236803F00703F4
:108E9800AB4239D8FFF7C8FC264B1860264BBDE813
:108EA800F0411868F9F71EBE6268022A1DD1FFF763
:108EB800C7FB00283FF467AF4FF0B04641F288384F
:108EC800B36823F003031343B360F9F70DFE0746B5
:108ED800B368626803F00C03B3EB820FD4D0F9F7E0
:108EE80003FEC01B4045F3D97FE7032A02D1FFF7F1
:108EF800BCFBDEE712B9FFF7A9FBDAE74FF0B04396
:108F08001B685B05D8D43EE7236823F007032B438F
:108F18002360F9F7E9FD0646236803F00703AB422F
:108F2800B8D0F9F7E1FD801B0228F5D95DE700BF4D
:108F380000400058280800202C08002008B5FFF73A
:108F480073FC4FF0B043044A9B68C3F3022352F802
:108F58002330D84008BD00BF683E010808B5FFF7B8
:108F680063FC4FF0B043044A9B68C3F3C22352F832
:108F78002330D84008BD00BF683E01084FF0B04319
:108F8800D3F89000C0F3400070474FF0B041020999
:108F9800D1F8883002F47F22000123EA020300F4AA
:108FA8007F200343C1F8883070474FF0B041020C6E
:108FB800D1F88830120423EA020343EA0040C1F8DA
:108FC8008800704770B5066816F48036044638D0B5
:108FD800FFF7C2FAF9F788FD614E05463368DB05ED
:108FE80029D54FF0B043616BD3F8902002F440725A
:108FF800914214D0D3F89010D3F8902042F48032E4
:10900800C3F89020D3F8902021F4407022F48032E5
:109018008D07C3F89020C3F8900000F190804FF0BE
:10902800B042616BD2F8903023F440730B43C2F81E
:109038009030002605E0F9F757FD401B0228CDD9EE
:1090480003262568E8070AD54FF0B0416268D1F8D1
:10905800883023EA124392B21343C1F88830A90733
:109068000AD54FF0B041A268D1F8883023EA1243FC
:1090780092B21343C1F88830AA0609D54FF0B0421E
:109088002169D2F8883023F440630B43C2F8883052
:10909800AB0502D5206AFFF788FF680502D5606A2C
:1090A800FFF783FF290502D5A06AFFF77EFF6A064E
:1090B80002D56069FFF769FF2B0602D5A069FFF7A3
:1090C80064FFE80502D5E069FFF75FFFE90610D500
:1090D8004FF0B042E168D2F8883023F440730B4374
:1090E800C2F88830B1F5807F02BFD36843F080733F
:1090F800D3602A040ED54FF0B042216BD2F88830E5
:1091080023F040430B43C2F8883019B9D36843F0C1
:109118008073D3606B0410D54FF0B042E16AD2F887
:10912800883023F040530B43B1F1005FC2F8883018
:1091380003D1D36843F48033D360304670BDF9F768
:10914800D3FC41F288360546FFF718FF01283FF4A3
:1091580066AFF9F7C9FC401BB042F5D970E700BF0C
:109168000004005830B590F82C30012B02464FF01F
:10917800020022D0174B82F82D00CA24012582F85C
:109188002C505C6253245C62B1F5807F146B996942
:1091980014D121F488519961596C24F0010421F00B
:1091A800004159641463DD650A4BFF2159620020B0
:1091B800012382F82D3082F82C0030BD21F40851AB
:1091C8009961D96C24F0020421F00041D964146338
:1091D800D865E9E70028004070B50B4E036B756D44
:1091E8001D40EA07044603D50123F365F9F7EDFDB1
:1091F800AB0704D50223F365204600F0CBF9012321
:1092080084F82D3070BD00BF0028004038B50A4CE6
:10921800E36823F02003E360F9F766FC0546E3689A
:109228009B0601D5002038BDF9F75EFC401BB0F560
:109238007A7FF4D90320F6E7002800402DE9F041B1
:10924800114DEC6814F0400407461AD1EB6843F05E
:109258008003EB60F9F748FC4FF003080646EB681B
:109268005B0601D4032C02D12046BDE8F081F9F752
:109278003BFC801BB0F57A7F84BF87F82D800324E0
:10928800EDE70024F0E700BF0028004038B50F4C98
:10929800E36823F08003E360A3699B06054606D4D0
:1092A800FFF7B4FF10B1032085F82D0038BDA3697E
:1092B80023F02003A361FFF7A9FF10B1032085F86D
:1092C8002D00A36943F02003A361EFE700280040C5
:1092D80038B5044600284BD090F82D3003F0FF0233
:1092E8001BB980F82C20F9F707FA0223214D84F8DE
:1092F8002D30EB68DB0632D4CA236B6253236B62D2
:109308002046FFF79BFF78BBAB6923F08E6323F001
:109318004003AB6121696368AA690B431343A269DF
:109328001343AB61D4E9022343EA02432B61D4E936
:109338000931EA680B4322F4F8521343EB602046E4
:10934800FFF7A4FF80B9D4E90713AA690B4322F0F9
:109358006042134362691343AB61FF236B620123CD
:1093680084F82D30002002E0024BFF225A6238BDFB
:109378000120FCE7002800400023092803D840EA20
:109388000310C0B270470A380133C0B2F5E70000D5
:109398002DE9F04790F82C30012B05464FF00200DC
:1093A80069D0012385F82C304E4B85F82D00DE68F6
:1093B80006F44076B6F5807F78D04C69087891F845
:1093C800019091F802A091F82470002A55D19B6968
:1093D80013F0400308BFCB70FFF7CEFF8046484626
:1093E800FFF7CAFF02465046FFF7C6FF81463846D8
:1093F800FFF7C2FF0B6ACF78234343EA875343EA58
:10940800090343EA084343EA022343EA0063354A6F
:10941800CA205062532050628C6A8869B4F5807FF4
:10942800946945D124F4885494610124D465B6F52F
:10943800807F09BFCB6913640343536418BF50642A
:10944800284B4A681A672A6B42F001022A639A6914
:1094580042F488529A61244AD2F8803043F40033A7
:10946800C2F880301F4BFF225A620020012385F882
:109478002D3085F82C00BDE8F087B4F1803F07D087
:10948800B4F5000F04D09B6913F0400308BFCB70FC
:109498000B6ACA781C4344EA0A0444EA004343EAD4
:1094A800092343EA825343EA0763B0E70023AEE7A0
:1094B80024F4085494610224D465B6F5807F09BF6A
:1094C800CB6993640343D36418BFD064054B4A68DF
:1094D8005A672A6B42F002022A639A6942F40852D8
:1094E800B8E700BF002800400008005890F82C207A
:1094F800012A03464FF0020012D00A4A83F82D00D1
:10950800CA21516253215162916941F02001916150
:10951800FF2151620020012283F82D2083F82C00BE
:10952800704700BF0028004090F82C20012A03460D
:109538004FF0020019D00D4A83F82D00CA2151625C
:109548005321516291690A4841F080019161D0F834
:10955800801041F48021C0F88010FF215162002062
:10956800012283F82D2083F82C0070470028004042
:1095780000080058064B5A6D520610B5044603D52C
:109588004022DA65F9F724FC012384F82D3010BD58
:10959800002800407047890001F1804101F5314100
:1095A8000A607047890001F1804101F5314108687E
:1095B80070470000034AD2F8903043F40043C2F8E1
:1095C8009030704700040058034AD2F8903023F4D2
:1095D8000043C2F89030704700040058074B1A68DF
:1095E80022F040021A6040F441704FF4B8521860FB
:1095F8005A601A6842F040021A6070470000015829
:1096080037B5054600284ED0837903F0FF046BB1C7
:10961800032C0BD0254B4FF400629A612868FFF7A2
:10962800DDFF002401232B71AC602FE000236B7158
:109638002846F9F771F91E4AD2F8903043F480535E
:10964800C2F89030002CE5D102234FF0B042AB7144
:10965800D2F8943023F40043C2F89430154B1B68B9
:109668001C214B43DB0C64214B430193019B93B9B1
:109678000124AC60FFF79EFF0C4B9A6842F400622D
:109688009A604FF400629A61002CC7D00123AB7135
:10969800204603B030BD019B013B0193D2F89430C2
:1096A8005B04E3D4E6E70124F2E700BF00040058B6
:1096B800000800582808002037B5174D2B680246C7
:1096C8001C204343DB0C6420434314480193019B53
:1096D80093B901209060114C21732B681C214B43D6
:1096E800DB0C64214B430193019B6BB90120906013
:1096F8000A4BDB6803B030BD019B013B01938368D3
:109708009C07E4D50020E6E7019B013B0193A36891
:10971800DB07E9D5ECE700BF280800200000015866
:1097280037B5184D2B6802461C204343DB0C6420D8
:10973800434315480193019BA3B901209060124C43
:10974800FF2323732B681C256B43DB0C64256B43B9
:109758000193019B73B9012090600B4BDB680B7080
:1097680003B030BD019B013B019383689C07E2D5A0
:109778000020E4E7019B013B0193A368DB07E8D5E0
:10978800EBE700BF28080020000001580F4B13B575
:109798001B680F4C182253431B0D64225343014688
:1097A80001936269019B02F0040223B902238B60D2
:1097B800012002B010BD019B013B0193606910F0CC
:1097C8000200F6D0002AECD11046F2E72808002063
:1097D8000004005807B50379012B0FD10A4B1B6809
:1097E800182253431B0C0193FFF7EEFE019B013B2C
:1097F8000193019B002BF9D1FFF7DCFE03B05DF864
:1098080004EBFFF7C3BF00BF28080020F8B51E46C9
:109818008379012B154604460F46DAB22DD14379D8
:10982800012B2AD0022342718371FFF7D3FF0D2148
:109838002046FFF7C9FEFFF73FFF390A2046FFF72A
:109848003BFFF9B22046FFF737FF2E44B5420ED151
:109858002046FFF7AFFEFFF799FFA0680123003805
:10986800A3714FF0000318BF01206371F8BD15F80C
:10987800011B2046FFF720FFE8E70220F6E7F8B5CE
:109888001E468379012B154604460F46DAB22FD1BE
:109898004379012B2CD04271FFF79CFF1D212046F4
:1098A800FFF792FEFFF708FF390A2046FFF704FF8B
:1098B800F9B22046FFF700FF00212046FFF7FCFE23
:1098C8002E44B5420ED12046FFF774FEFFF75EFF27
:1098D800A06801230038A3714FF0000318BF0120CE
:1098E8006371F8BD29462046FFF71AFF0135E8E7FE
:1098F8000220F6E7F8B51F468379012B1546044682
:109908000E46DAB22CD14379012B29D04271FFF7E8
:1099180061FF06F0EF03A3F1840253425341237120
:1099280031462046FFF750FEFFF7C6FE2F44AF42F0
:1099380010D1FFF73FFE842E02D02046FFF726FF06
:10994800A06801230038A3714FF0000318BF01205D
:109958006371F8BD15F8011B2046FFF7ADFEE6E779
:109968000220F6E7F8B51E468379012B1546044612
:109978000F46DAB227D14379012B24D04271FFF781
:1099880029FF39462046FFF71FFEFFF795FE002105
:109998002046FFF791FE2E44B5420ED12046FFF730
:1099A80009FEFFF7F3FEA06801230038A3714FF00A
:1099B800000318BF01206371F8BD29462046FFF750
:1099C800AFFE0135E8E70220F6E737B50023ADF82A
:1099D800043001AA022312210546FFF7C3FFBDF890
:1099E8000440022364BA01AAA4B219462846FFF724
:1099F80081FFE20702D5284609F0F6F9A30702D548
:109A0800284609F0F7F9600702D5284609F01CFA3C
:109A1800210702D5284609F01DFAE20602D5284694
:109A280009F01EFAA30602D5284609F007FA6006CF
:109A380002D5284609F0E4F9210606D514F4807108
:109A480018BF0121284609F0E1F9A20502D52846E8
:109A580009F0ECF9630402D5284609F007FA03B0C7
:109A680030BDF8B51E468379012B154604460F46CE
:109A7800DAB227D14379012B24D04271FFF7AAFE2D
:109A88000E212046FFF7A0FDFFF716FE39462046B7
:109A9800FFF712FE2E44B5420ED12046FFF78AFD8D
:109AA800FFF774FEA06801230038A3714FF000038C
:109AB80018BF01206371F8BD15F8011B2046FFF798
:109AC800FBFDE8E70220F6E7F8B51E468379012B8F
:109AD800154604460F46DAB22BD14379012B28D01C
:109AE8004271FFF777FE1E212046FFF76DFDFFF755
:109AF800E3FD39462046FFF7DFFD00212046FFF74A
:109B0800DBFD2E44B5420ED12046FFF753FDFFF78B
:109B18003DFEA06801230038A3714FF0000318BF71
:109B280001206371F8BD29462046FFF7F9FD01358C
:109B3800E8E70220F6E7026852E8003F23F0C00396
:109B480042E8003102680029F5D102F1080353E820
:109B5800003F23F4000302F1080C4CE8003100290F
:109B6800F3D12023C0F888307047000010B5026890
:109B780052E8003F23F4907342E80031026800295C
:109B8800F5D10F4C02F1080353E8003F234002F1DE
:109B9800080C4CE800310029F4D1C36E012B07D121
:109BA80052E8003F23F0100342E800310029F7D1C2
:109BB8002023C0F88C300023C366436710BD00BF64
:109BC800FEFFFFEFF8B504461346D4F88850202D61
:109BD80032D1F1B1EAB1E06FA4F85620A4F85420CC
:109BE80000262122C4F890602165C4F888202268E4
:109BF80088B1124FC762124F0763124F2832C0E96B
:109C08000D76FDF745FE30B11023C4F89030C4F846
:109C1800885001200FE0236840221A62226802F16E
:109C2800080353E8003F43F0800302F1080141E8CC
:109C380000300028F3D1F8BD0220FCE7519C000851
:109C4800999C0008A59C000808B50346806A1B6813
:109C58001B6813F0200317D1A0F85630026802F1F0
:109C6800080353E8003F23F08003083242E800313C
:109C780002680029F2D152E8003F43F0400342E86D
:109C880000310029F7D108BDF9F7F8F9FBE770476B
:109C980008B5806AFFF7FBFF08BD7047806A38B5D2
:109CA8000468D0F88830D0F88C50A268120606D51F
:109CB800212B04D10023A0F85630FFF73CFFA368FE
:109CC8005B0606D5222D04D10023A0F85E30FFF7ED
:109CD8004DFFD0F8903043F01003C0F89030FFF7F4
:109CE800DCFF38BD08B5806A0023A0F85E30A0F814
:109CF8005630FFF7D2FF08BD704700000368D969E6
:109D08001A682DE9F04140F60F0631429D68044675
:109D180010D18E0640F1978002F0200605F080579A
:109D28003E4300F09080436F002B00F08580BDE833
:109D3800F0411847AB4EAC482E401040304300F07D
:109D48008280CF0709D5D00507D501201862D4F83D
:109D5800900040F00100C4F890008F0709D5E8078B
:109D680007D502201862D4F8900040F00400C4F827
:109D780090004F0709D5E80707D504201862D4F8E2
:109D8800900040F00200C4F890000F070BD502F0D5
:109D98002000304307D008201862D4F8900040F023
:109DA8000800C4F890000E050AD5500108D54FF4F4
:109DB80000601862D4F8903043F02003C4F8903063
:109DC800D4F89030002B37D08B0609D502F020024A
:109DD80005F080552A4303D0636F0BB1204698479E
:109DE8002668D4F89020B36802F0280203F04003F4
:109DF80053EA0205204621D0FFF7B8FEB3685F0694
:109E080017D5226802F1080353E8003F23F0400306
:109E1800083242E800310029F3D1D4F8800040B17B
:109E2800724B8363FDF7ADFD30B1D4F88000836BCE
:109E38007DE72046FFF731FFBDE8F081FFF72DFFF2
:109E4800C4F89050F8E7E06E012840F08980CE060B
:109E580040F18680D00640F1838010221A629A6809
:109E680051064BD5D4F8802011684A6892B2002A6E
:109E7800E2D0B4F85C009042DED9A4F85E200A680B
:109E880092062FD453E8002F22F4807243E8002171
:109E98000029F7D103F1080252E8002F22F001024D
:109EA80003F1080040E800210029F3D103F108027A
:109EB80052E8002F22F0400203F1080040E8002198
:109EC8000029F3D12022C4F88C20E16653E8002F42
:109ED80022F0100243E800210029F7D1D4F88000CD
:109EE800FDF71AFD02232367B4F85E30B4F85C105E
:109EF800C91A89B22046FFF7FFFE9DE7B4F85E2035
:109F0800B4F85E00B4F85C1080B292B2002893D026
:109F1800891A89B200298FD053E8002F22F4907251
:109F280043E800200028F7D1314D03F1080252E838
:109F3800002F2A4003F1080646E800200028F4D143
:109F48002022C4F88C206067E06653E8002F22F0D6
:109F5800100243E800200028F7D102232367C9E74D
:109F6800CF0209D56E0207D54FF4801220461A6237
:109F7800BDE8F04100F0A0BD08060BD502F0800056
:109F880005F40005284305D0A36F002B3FF454AF18
:109F98002046CCE64F0611D556060FD553E8002FBC
:109FA80022F0400243E800210029F7D12023C4F819
:109FB8008830A1672046F9F761F83DE70D0206D51C
:109FC800500004D52046BDE8F04100F077BDCB0134
:109FD8007FF532AF002ABFF62FAF2046BDE8F0412B
:109FE80000F06BBD0100001020010004ED9C00088A
:109FF800FEFFFFEFD0F88C20B0F86010222A08B5D9
:10A00800036855D15B6A826D0B401370836D013311
:10A018008365B0F85E30013B9BB2A0F85E30B0F8C3
:10A028005E309BB2002B42D1026852E8003F23F415
:10A03800907342E8003103680029F5D103F1080262
:10A0480052E8002F22F0010203F1080C4CE800212D
:10A058000029F3D12022C0F88C20184A4167934286
:10A06800016705D1C26E012A0ED0F9F715F81EE076
:10A078005A681102F6D553E8002F22F0806243E8AF
:10A0880000210029F7D1EDE70022C26653E8002F2E
:10A0980022F0100243E800210029F7D1DA69B0F86C
:10A0A8005C10D20644BF10221A62FFF725FE08BDD5
:10A0B8009A6942F008029A61F9E700BF00800040FF
:10A0C800D0F88C20B0F86010222A08B5036852D165
:10A0D8005A6A1140826D22F8021B8265B0F85E2030
:10A0E800013A92B2A0F85E20B0F85E2092B2002A3F
:10A0F80040D153E8002F22F4907243E80021002950
:10A10800F7D103F1080252E8002F22F0010203F10F
:10A11800080C4CE800210029F3D12022C0F88C203B
:10A12800174A41679342016705D1C26E012A0ED0D2
:10A13800F8F7B2FF1EE05A681102F6D553E8002F6F
:10A1480022F0806243E800210029F7D1EDE70022E0
:10A15800C26653E8002F22F0100243E800210029CC
:10A16800F7D1DA69B0F85C10D20644BF10221A623F
:10A17800FFF7C2FD08BD9A6942F008029A61F9E743
:10A18800008000402DE9F74F0368B0F86080DF6970
:10A198001A689D68D0F88C1001922229044640F074
:10A1A800B480B0F86890DFF86CA1DFF86CB10026D5
:10A1B800B9F1000F01D0BB0621D4B4F85E309BB2D0
:10A1C800D3B1B4F868209A4216D9226802F108037C
:10A1D80053E8003F23F08053083242E800312268F8
:10A1E8000029F2D14D4B636752E8003F43F020034A
:10A1F80042E800310029F7D103B0BDE8F08F2368A9
:10A20800A26D5B6A03EA08031370A36D0133A365AB
:10A21800B4F85E30013B9BB2A4F85E302368DF6976
:10A2280078072CD0F9070AD5019AD20507D501215C
:10A238001962D4F8901041F00101C4F89010B807E1
:10A2480009D5E90707D502211962D4F8901041F021
:10A258000401C4F890107A0709D5E80707D5042146
:10A268001962D4F8903043F00203C4F89030D4F85F
:10A27800903023B12046FFF710FDC4F89060B4F881
:10A288005E309BB2002B93D1216851E8003F23F444
:10A29800807341E8003023680028F5D103F10802F3
:10A2A80052E8001F01EA0A0142E800100028F5D12F
:10A2B80020215B45C4F88C10606720670AD0596874
:10A2C800090207D553E8001F21F0806143E8001018
:10A2D8000028F7D1E16E012913D1E66653E8001F83
:10A2E80021F0100143E800100028F7D1D969CA0607
:10A2F80044BF102119622046B4F85C10FFF7FCFC3B
:10A3080056E72046F8F7C8FE52E79A6942F0080275
:10A318009A6171E7FEFFFFEF00800040FD9F000893
:10A328002DE9F74F0368B0F86080DF691A689D6807
:10A33800D0F88C1001922229044640F0B280B0F87F
:10A348006890DFF868A1DFF868B10026B9F1000F5E
:10A3580001D0BB0621D4B4F85E309BB2D3B1B4F8B7
:10A3680068209A4216D9226802F1080353E8003F90
:10A3780023F08053083242E8003122680029F2D1E4
:10A388004C4B636752E8003F43F0200342E800313A
:10A398000029F7D103B0BDE8F08F2368A26D596A90
:10A3A80008EA010122F8021BA265B4F85E20013A0E
:10A3B80092B2A4F85E20DF6978072CD0F9070AD595
:10A3C800019AD20507D501211962D4F8901041F0FD
:10A3D8000101C4F89010B80709D5E90707D502218B
:10A3E8001962D4F8901041F00401C4F890107A076B
:10A3F80009D5E80707D504211962D4F8903043F04D
:10A408000203C4F89030D4F8903023B12046FFF707
:10A4180044FCC4F89060B4F85E309BB2002B95D130
:10A42800216851E8003F23F4807341E80030236835
:10A438000028F5D103F1080252E8001F01EA0A01D9
:10A4480042E800100028F5D120215B45C4F88C10A3
:10A45800606720670AD05968090207D553E8001FCA
:10A4680021F0806143E800100028F7D1E16E01294E
:10A4780013D1E66653E8001F21F0100143E80010ED
:10A488000028F7D1D969CA0644BF102119622046AD
:10A49800B4F85C10FFF730FC58E72046F8F7FCFDED
:10A4A80054E79A6942F008029A6173E7FEFFFFEFEA
:10A4B80000800040C9A0000838B504460368216937
:10A4C800A2681D68C0690A4361690A437D4902435D
:10A4D80029400A431A605A68E16822F440520A4344
:10A4E8005A60794AA16993421CBF226A11439A684B
:10A4F80022F06E4222F430620A439A60DA6A616A94
:10A5080022F00F020A43DA62704A93421CD14FF0DC
:10A51800B043D3F8883003F0030343F44033A3F582
:10A528004033013B022B00F2C780694A9B5CB0F5BF
:10A53800004F40F08980082B24D8DFE803F061C081
:10A548008323802323236500624A934209D14FF075
:10A55800B043614AD3F8883003F00C0343F4402336
:10A56800E4E7594A93420DD14FF0B043D3F888300D
:10A5780003F44063B3F5006F1AD005D853B1B3F5AF
:10A58800806F12D0012009E0B3F5406FFAD14FF483
:10A5980000400EE0FEF7D2FC58B900204FF001133E
:10A5A800A3660023C4E91D3338BDFEF7CFF8F3E7EF
:10A5B8004A4865684A4B626A05EB450133F8122040
:10A5C800B0FBF2F39942DDD8B3EB053FDAD80023AC
:10A5D8001946F7F799FA090241EA10616B08000277
:10A5E800C0182A464FF0000341F10001F7F78CFA32
:10A5F8003C4BA0F540729A42C4D82368D860CCE797
:10A60800FEF79CFC0028C8D06168354B626A33F8B5
:10A618001220B0FBF2F24B0803EB42034FF6EF7245
:10A62800B3FBF1F3A3F110019142ABD823F00F0271
:10A63800216892B2C3F342031343CB60ADE7FEF740
:10A6480085F8DFE72548DFE7082B9BD801A252F8F9
:10A6580023F000BFA5A60008B1A60008BDA6000803
:10A668008DA50008B7A600088DA500088DA50008CF
:10A678008DA5000881A600084FF400406368616A50
:10A68800174A32F81120B0FBF2F000EB5300B0FB90
:10A69800F3F04FF6EF73A0F11002ACE7FEF74EFCB3
:10A6A80000283FF47AAFE9E7FEF758FCF8E7FEF731
:10A6B8004DF8F5E70948E1E7B0F5004FF4D1FEF7AA
:10A6C8004DFC9FE7F369FFCF008000400038014050
:10A6D800C83E010800440040CB3EF5070024F400C2
:10A6E800D83E0108FFFC0F00836ADA0710B506D5CB
:10A6F8000168C46A4A6822F4003222434A609C070F
:10A7080006D50168046B4A6822F4803222434A6005
:10A71800590706D50168446B4A6822F4802222430F
:10A728004A601A0706D50168846B4A6822F4004219
:10A7380022434A60DC0606D50168C46B8A6822F4A5
:10A74800805222438A60990606D50168046C8A689B
:10A7580022F4005222438A605A060FD50168446CDD
:10A768004A6822F480122243B4F5801F4A6005D15A
:10A778004A68846C22F4C00222434A601B0606D54C
:10A788000268C16C536823F400230B43536010BD67
:10A798002DE9F041DDF8188004460E4615461F469F
:10A7A8002268D36936EA03030CBF01230023AB42B6
:10A7B80001D0002027E0B8F1FF3FF2D0F8F794F974
:10A7C800C01B4045206802D8B8F1000F1DD150E8E1
:10A7D800003F23F4D07340E80032002AF7D100F19B
:10A7E800080353E8003F23F0010300F1080141E8A2
:10A7F8000032002AF3D12023C4F88830C4F88C3002
:10A8080084F884200320BDE8F08103685A07C7D57F
:10A81800C3691B05C4D54FF40063036250E8003FC9
:10A8280023F4D07340E80032002AF7D100F108037E
:10A8380053E8003F23F0010300F1080141E800322A
:10A84800002AF3D12023C4F88830C4F88C30C4F827
:10A858009030D5E773B504460026C0F89060F8F745
:10A8680043F923681B681A07054619D423681B682F
:10A878005B070AD56FF07E43009300222B464FF406
:10A8880080012046FFF784FFB0B900202023C4F8D8
:10A89800883084F88400C4F88C30E06620670CE0C7
:10A8A8006FF07E430093324603464FF40011204672
:10A8B800FFF76EFF0028D9D0032002B070BD10B595
:10A8C800044650B3D0F888301BB980F88430F8F7C4
:10A8D800C1FA22682423C4F88830136823F00103DE
:10A8E80013602046FFF7E8FD012816D0A36A13B1CC
:10A8F8002046FFF7F9FE23685A6822F490425A600E
:10A908009A6822F02A029A601A6842F001022046E8
:10A918001A60BDE81040FFF79DBF012010BD000080
:10A9280030B581658168A0F85C200023B1F5805FAF
:10A93800A0F85E20436735D10369002B40F2FF136E
:10A9480018BFFF23A0F860300023C0F890302223FE
:10A95800C0F88C30016801F1080353E8003F43F068
:10A968000103083141E800340368002CF2D1456E38
:10A9780084680169B5F1005F34D1B0F86850954238
:10A9880030D8B4F5805F1DD1254A264C002918BF60
:10A9980022464267C1B153E8002F42F4807243E86F
:10A9A8000021F7E729B90369002B14BF7F23FF2390
:10A9B800C8E7B1F1805FC5D10369002B0CBF7F23C5
:10A9C8003F23BFE7174AE4E703F1080252E8002FE4
:10A9D80042F0805203F1080040E800210029F3D139
:10A9E800002030BDB4F5805F0FD10F4A0F4C00290D
:10A9F80018BF2246426751B153E8002F42F49072C3
:10AA080043E800210029F7D1EAE7084AF2E753E8CA
:10AA1800002F42F0200243E800210029F7D1DFE7A8
:10AA280029A300088DA10008C9A00008FD9F0008FF
:10AA3800D0F88C30202B30B415D1B9B1B2B1002385
:10AA48000468C3660A4B9C420AD063681B0207D598
:10AA580054E8003F43F0806344E80035002DF7D107
:10AA680030BCFFF75DBF022030BC70470120FBE718
:10AA780000800040436E30B52BB90123A0F86A303E
:10AA8800A0F8683030BD0368094D9A689968094C88
:10AA9800490FC2F342626B5C615CDB00B3FBF1F30C
:10AAA800A0F86A30AB5CA25CDB00B3FBF2F3E7E72B
:10AAB800F83E0108F03E01087047704770471FB51F
:10AAC80004AB03E9060090F88430012B04463AD021
:10AAD800012380F884302423C0F8883003681A687A
:10AAE80022F001021A609A6822F440120A439A601E
:10AAF80071B95A68BDF80C009DF80E1022F01002CA
:10AB080002435A605A6822F07F4242EA01625A6060
:10AB18001A6842F001021A60F7F7E6FF6FF07E420A
:10AB2800034600924FF4800100222046FFF730FED2
:10AB380038B92023C4F88830002384F8843004B05E
:10AB480010BD0320F8E70220F9E790F88430012BC4
:10AB58000FD0012380F88430016851E8002F42F0BB
:10AB6800020241E80023002BF6D180F88430184611
:10AB780070470220704710B590F88430012B0446C6
:10AB880017D02423C0F8883003681A68196821F0A0
:10AB98000101196042F000524FF0005141661A60FD
:10ABA800FFF768FF2023C0F88830002084F884006D
:10ABB80010BD0220FCE770B590F88430012B0446E4
:10ABC80017D005682423C0F888302E682B6823F036
:10ABD80001032B60AB6823F060431943A960FFF7BA
:10ABE80049FF20232E60C0F88830002084F88400B4
:10ABF80070BD0220FCE770B590F88430012B044644
:10AC080017D005682423C0F888302E682B6823F0F5
:10AC180001032B60AB6823F060631943A960FFF759
:10AC280029FF20232E60C0F88830002084F8840093
:10AC380070BD0220FCE7000038B5094D002455F826
:10AC4800043B33B90134E3B2052B64B2F7D10020D9
:10AC580038BD002CF6D01B6998470028F2D0F7E7DA
:10AC6800701000207FB50A2301A88DF8043003F086
:10AC7800D9F80038044B059A1A6018BF01204042E1
:10AC880007B05DF804FB00BF6810002070B50446EB
:10AC98000B46144962784A700020A2780A7208703C
:10ACA8001A884A729A788A72DB780B746368CB6068
:10ACB8000D4B1B68DA6A2AB1237803F0FB030B2BD0
:10ACC80000D09047094E002556F8043B1BB19B6AFB
:10ACD8000BB1204698470135EBB2052B6DB2F3D185
:10ACE80070BD00BF480800206C10002070100020C4
:10ACF80070B5044611480123037063784370A37844
:10AD08008372E368C360E378037623694376237923
:10AD180043720B4B1B689B6A03B19847094E002589
:10AD280056F8043B1BB1DB690BB120469847013547
:10AD3800EBB2052B6DB2F3D170BD00BF5C080020EB
:10AD48006C1000207010002038B501F011FE0C4D79
:10AD5800052455F8043B5BB15B694BB155F8043CDD
:10AD68009B682BB1984718B155F8043C5B69984724
:10AD7800013C14F0FF04ECD1BDE83840FFF75CBF9C
:10AD880070100020014B1868704700BF6810002041
:10AD980000B58BB0012368468DF8003002F0BCFC8A
:10ADA80038B99DF80400003818BF01200BB05DF8D1
:10ADB80004FB0020FAE7000030B58BB0054601F02F
:10ADC800BBFD0446002839D1FFF7E2FF012838D13E
:10ADD80068468DF8004002F09FFC10B14FF0FF303C
:10ADE80004E09DF80430AB4202D100200BB030BD26
:10ADF800012DF3D0022D11D0002DF7D1002BF4D066
:10AE080068468DF8045002F099FD0028E6D10E4BF3
:10AE18001B681B6B002BE8D09847E6E7002BDDD1B9
:10AE280068468DF8045002F089FD0028D6D1064BFB
:10AE38001B681B6B002BD8D02846EDE76FF001008C
:10AE4800D4E76FF00200D1E76C10002070B5324CE7
:10AE5800324B94F9042094F9055090B00126022849
:10AE68008DF804608DF809208DF80A500AD18DF804
:10AE78000800D871197202F09FFB01A802F0D2FFF6
:10AE880010B070BD4FF480701A715D71D88019725E
:10AE9800234B8DF808601B7853BB1E2306A88DF83A
:10AEA8001C208DF8183002F049FD1F238DF818304A
:10AEB80006A823798DF81C3002F040FD21238DF877
:10AEC800183006A863798DF81C3002F037FD20236E
:10AED8008DF8183006A863798DF81C3002F02EFD25
:10AEE80028238DF8183006A80E4B079302F026FD8C
:10AEF80002F062FB012306A88DF818308DF81C308B
:10AF080002F01CFD084B1B685B6A0BB103489847AD
:10AF18006078FFF751FFB3E7841000203008002065
:10AF280064100020000300016C10002008B501F037
:10AF380003FD40B9FFF72CFF012806D0084B197A0A
:10AF4800D879FFF783FF012008BD064B1B68DB6833
:10AF580098470028F7D1BDE80840FFF76DBE00BF4D
:10AF680030080020701000202DE9F04186B0054619
:10AF78000C46164601F0E0FC002840F08D8001F0F8
:10AF8800EDFC40B9FFF704FF012807D0444B197ABC
:10AF9800D879FFF75BFF6FF002046DE0414F3B6823
:10AFA800DB68984730B13A682B7812789A4201D01A
:10AFB800002B6ED13C4FDFF8F4803C72003C18BF88
:10AFC800012498F8043068788DF8044069468DF8B3
:10AFD800123002F049FB002840D000238DF80430DD
:10AFE8000393ADF810306FF0060495E80300304B7A
:10AFF80083E8030098F80430BB72314601A803F0D7
:10B0080009F82C4B059A1A6011283FD801A353F868
:10B0180020F000BF7BB00008A1B0000895B0000880
:10B0280095B0000895B0000895B0000895B00008E4
:10B038009FAF000895B0000895B0000895B00008CB
:10B048008FB0000895B0000895B00008A1B00008BE
:10B05800A1B00008A1B0000889B000082B788DF8CD
:10B0680008306B78ADF810306B6803934FF0FF34FD
:10B07800BBE7E31D18BF0024204606B0BDE8F081F9
:10B088006FF00404F8E76FF00504F5E74FF0FF34BC
:10B09800F2E76FF00304EFE76FF00104ECE700BF9D
:10B0A80030080020701000205C0800208410002068
:10B0B8006C0800206810002010B504468AB018B942
:10B0C8004FF0FF300AB010BD002368468DF80030FD
:10B0D80002F022FB0028F3D19DF804302370F1E739
:10B0E800F0B587B000220B462A498DF807200122C7
:10B0F8000A7042784A700446002A41D102790A72DD
:10B108001A884A729A788A72DB780B740369CB6062
:10B11800C378214D8DF80830037B8DF8093083689A
:10B1280003932B68DB6A0BB102A898472B689B6BCB
:10B1380013B1227E02B19847184E0025374656F8BB
:10B14800043B53B11A6A42B11A78E3789A4219D18A
:10B1580056F8043C20461B6A98470135EBB2052B8C
:10B168006DB2ECD10DF10700FFF7A6FF63793BB193
:10B178000021012204A8ADF810100591FFF7F4FE94
:10B1880007B0F0BD002DE8D13B68DB689847002880
:10B19800DED1E2E7480800206C1000207010002083
:10B1A80010B504468AB018B94FF0FF300AB010BD88
:10B1B8001F2368468DF8003002F0AEFA0028F3D15C
:10B1C800024A9DF9043023701371EFE784100020C0
:10B1D80000B58BB02223019068468DF8003002F04C
:10B1E800ADFB003818BF012040420BB05DF804FBEE
:10B1F80070B5634C014618228EB0204605F066FFF4
:10B20800F8F72EFF23784068012202FA03F1014083
:10B2180004D15C4B084607F04FFFFEE75A495B48EC
:10B228001A4602F011F818B14FF0FF300EB070BD99
:10B23800262304A88DF8103002F080FB544E554D9B
:10B24800002870D1012333702B68DB690BB1002013
:10B258009847262304A88DF8103002F05DFA059B64
:10B2680093F84820227093F8182193F81A316270E5
:10B27800A370454BD3E9020105F01AFE05460028E4
:10B28800D2D1454E062304A88DF8103002F044FAB6
:10B29800059B736104A802F051FB022304A88DF8F2
:10B2A8001030059602F038FA0836032304A88DF802
:10B2B8001030059602F030FA0F2605F0BDFE012386
:10B2C80004A88DF814308DF8106002F037FB1023B5
:10B2D8000DEB03008DF810308DF8145002F02EFBA2
:10B2E80004238DF8103004A8A3788DF8143002F0E8
:10B2F80025FB39238DF8103004A86369059302F003
:10B308001DFB02A920788DF8086003F051FF003872
:10B3180018BF0120E0711420FFF75AFFE07903F00D
:10B3280003F8284682E727238DF810302B681B691D
:10B3380043B104A802F0F0F92B6805981B694FF493
:10B34800EE619847262304A88DF8103002F0F6FA2B
:10B3580050B9012304A88DF8103002F0DDF99DF8EA
:10B368001430002B7FF46EAF3378002B7FF46CAF72
:10B37800052204A88DF81020059302F0DFFA78E77B
:10B3880084100020003F01089C100020B410002009
:10B39800641000206C1000204C10002037B50023EA
:10B3A8000D4601930446C0B900F0D0FA0190019B04
:10B3B800C3B10E4A0E4942F824300E4ADA620E4AE8
:10B3C8001A630E4A5A630E4A126892699A612846AD
:10B3D8005B68F2229847002006E001A900F0BCFA59
:10B3E8000028E4D04FF0FF3003B030BD70100020CB
:10B3F800580F002055AE000871AF00086DAC00086A
:10B408006C100020154B07B51860154B154A1A60CB
:10B41800154A5A60154A9A60154ADA60154B02684F
:10B428001A6042685A6082689A60C268DA60124A92
:10B4380001911A61114982695A610020FFF7AEFF34
:10B4480048B901A800F086FA003818BF0120404228
:10B4580003B05DF804FB4FF0FF30F9E76C100020F3
:10B46800B4100020F9AC0008E9B0000805B50008E0
:10B4780095AC00089C10002069F100083C080020E9
:10B4880051B118B1012804D000207047044B0B605B
:10B498007047044B0B60F7E74FF0FF30704700BF71
:10B4A800000300010300010108B502F059FF00285C
:10B4B80014BF6FF00100002008BD08B502F0A4F821
:10B4C800002814BF6FF00100002008BD10B5044625
:10B4D8008AB018B94FF0FF300AB010BD2023684673
:10B4E8008DF8003002F018F90028F3D1024A9DF9CE
:10B4F800043023705371EFE7841000202DE9F041E8
:10B508002F4D304F00232B7043786B703B689B6A3C
:10B518008AB004460BB128469847DFF8AC8000266D
:10B5280058F8043B1BB15B6A0BB1204698470136BB
:10B53800F3B2052B76B2F3D12378052B2FD00C2B41
:10B5480035D0012B25D1214C062368468DF80030D3
:10B5580002F0E2F80199E07905F0F0FC10B91C4B13
:10B56800019A5A611B48FFF71BFE1B48FFF7AEFF05
:10B578006B788BB9A371194B5878FFF71DFC3B68A2
:10B588005B6A0BB1114898476B7813B9E07905F0FD
:10B5980065FD0AB0BDE8F081FF23A371EFE7104B0A
:10B5A80001225A74227A9A74627ADA74F1E763781B
:10B5B800002BEED00AB0BDE8F041FFF753BB00BF47
:10B5C8005C0800206C10002070100020300800205B
:10B5D8004C1000203408002035080020841000207A
:10B5E8004808002030B58BB0FFF767FF0446F0B974
:10B5F80003F0BEFD831C1DD0F8B9134D2B685B69A1
:10B60800DBB1262368468DF8003002F085F82B68F8
:10B6180001985B694FF4EE61984703F0BBFD78B978
:10B628002CB9094B1B68DB690BB1012098472046F0
:10B638000BB030BD6FF00704EFE74FF0FF34ECE7D5
:10B648004FF0FF34F3E700BF6C10002030B5064D13
:10B65800064C30B129B12860A160627101232370C2
:10B6680030BD00232B60FAE7F0100020C410002042
:10B67800014B1878704700BFC4100020024B18789F
:10B6880000B15878704700BFC41000207047000010
:10B69800064B1A784AB15A783AB10278012A04D18D
:10B6A800027912B19A8901329A817047C410002038
:10B6B800074B1A7852B15A7842B10278052A05D157
:10B6C800017A427AD973012098731A74704700BFBF
:10B6D800C410002013B51A4C23783BB363782BB3FE
:10B6E800A27BA36862B10022A2730322A271052281
:10B6F8001A70E27B5A70227C9A700122A27004E0D0
:10B70800A278012A14D0042AF7D0E0228DF800206C
:10B718000C48A27901938DF8012008F049F80A4BEA
:10B728001B6B1BB1E17801226846984702B010BD37
:10B738000222A271A2895A70110A1970E5E700BFA6
:10B74800C4100020D810002078080020FFF7C2BFDE
:10B7580030B5794C23788DB0002B43D0437B002B38
:10B7680040D0657825B1837B13B9A3890133A381C0
:10B77800C178E02936D1002D36D1027B042A31D197
:10B788008368187801282DD1587801282AD198780B
:10B79800012827D1DB78012B24D102206380A071F6
:10B7A800E56002A863708DF80C3021718DF80820CF
:10B7B800257402F0C3F8284602F0B6FD5F4B1B68FB
:10B7C8005B6803B1984700225D4B00924FF0FF3150
:10B7D8005C4807F041FF41F288315A4808F022F8E6
:10B7E800FFF778FF0DB030BD83681A78A2700A2A77
:10B7F800F8D8DFE802F0062124282A3D44658D8F19
:10B808009900504807F086FF00236370A3814B4CD2
:10B8180004238DF80830236802A81B788DF80C30B3
:10B8280002F08CF82368587802F07EFD23689B6844
:10B83800002BD7D09847D5E70223A371D2E740F26F
:10B8480001136380CEE70123FBE7A568037BA3719F
:10B8580004222A7062799A4228BF1A4600230133CB
:10B86800D9B28A42BED98168C95C0131E954F6E788
:10B8780005238DF8083002A802F0D4FAB2E731485F
:10B8880007F048FF00236370A3812C4C04238DF834
:10B898000830236802A81B788DF80C3002F04EF8A7
:10B8A8002368587802F040FD23689B6803B19847E5
:10B8B800254BDB6A002B95D001210220984791E7A0
:10B8C800027B032A0DD106228DF80820B3F8013037
:10B8D8005BBAADF80C3002A802F0A4FA0123A370F9
:10B8E80080E7072AF7D18DF80820B3F8012052BA6B
:10B8F800ADF80C201A79D978120242EA0142597936
:10B908000A4364214A4304929B798DF81430E2E794
:10B918000A23AEE700228DF808205B788DF80C30FA
:10B9280002A802F00BF85DE70D228DF808205B787D
:10B938008DF80C309FE700BFC4100020F0100020E5
:10B9480055B70008D8100020780800200048704734
:10B9580078080020002070474FF0FF307047000043
:10B96800044B054A93F81831022B18BF062382F8B6
:10B978008034704764180020D81F0020034BD3F888
:10B98800483313B15B6903B118477047D81F0020CB
:10B99800034A137843F002031370FFF7EFBF00BFA9
:10B9A800D41F00201FB50A4B8DF8090093F87C209E
:10B9B8008DF80A2093F88C2093F848000D3202A9DC
:10B9C8008DF8082003F0F4FBC0B205B05DF804FB65
:10B9D8006418002010B50D4C04F57D7007F09AFE30
:10B9E80094F8103413B1012384F80F34084B93F8FA
:10B9F8001831022B02BF94F8813443F0100384F805
:10BA08008134BDE81040FFF7B9BF00BFD81F002040
:10BA18006418002010B50C4CD4F8403343F0800370
:10BA2800C4F8403394F8103413B10020FFF7D2FF64
:10BA380094F8813423F0120343F0120384F881341C
:10BA4800BDE81040FFF78CBFD81F00202DE9F0415A
:10BA58002C4D95F81831022B07460E4602D02A4B7A
:10BA6800DB6A984702F01BFD044628B1022002F069
:10BA78000CFD002002F00EFD95F81831012B17D1AE
:10BA880002F00FFD804630B1002002F0FFFC0020DC
:10BA980002F001FD444602F006FD48B1002002F024
:10BAA800F6FC002002F0F8FCBDE8F041FFF758BFB3
:10BAB800002CF9D1154C94F8802494F81034B2B9BC
:10BAC8000BB184F83574384602F090FEE86A07F046
:10BAD800E7FDD4F8B4339842E6D30D4807F01AFED0
:10BAE80094F8813443F0100384F88134DCE70BB117
:10BAF80084F83564304602F079FE95F81831022B47
:10BB0800EED1D1E7641800200C460108D81F0020A8
:10BB180070230020074A10B5137843F0010313700F
:10BB2800FFF72CFFBDE81040034B01220021022043
:10BB380007F0C2BAD41F0020493F0108074A10B5D0
:10BB4800137843F004031370FFF718FFBDE81040A3
:10BB5800034B01220021022007F0AEBAD41F0020B7
:10BB6800593F01082DE9F0410F4616461D4680460B
:10BB780007F08CFD0A4A0B4C1378278143F0080321
:10BB8800C4E90008137066812573FFF7F7FEBDE866
:10BB9800F041054B01220021022007F08DBA00BFB9
:10BBA800D41F0020E0240020693F010813B507F0E6
:10BBB8006DFD0D4B6C461860204607F0BBFC94E801
:10BBC80003000A4A0A4B83E80300137843F0100382
:10BBD8001370FFF7D3FE074B01220021022002B0A9
:10BBE800BDE8104007F068BAF0240020D41F0020F8
:10BBF80010230020763F01082DE9F04192B0064657
:10BC080002F04DFC002840F05681AC4D95F81831F3
:10BC1800012B09D02B6BAA4C93B194F80431BBB11A
:10BC2800042B6FD0032003E002F03BFC18B10F2077
:10BC380012B0BDE8F08102F036FC0028EAD0F6E741
:10BC4800B5F81E31D4F81424013B53432B63E4E7C1
:10BC58009C4803F0E4F9002840F0298194F80C315D
:10BC680023802B6B0C930DF1180895F839308DF85B
:10BC78003830404695F81C318DF83A3007F080FC92
:10BC8800D5F82431009302AF98E80600D5F82031A2
:10BC9800384607F00CFC97E803000FAB83E8030075
:10BCA800EB6A0D9300238DF844302388ADF84630B5
:10BCB80095F82C3101228DF839201BB98DF84420D4
:10BCC8008DF83930804B0093804B95F84800A3F1EC
:10BCD80073020CA903F0E1FAC0B10B28A8D1D4F87B
:10BCE800841499B1002EA3D0D4F84033784843F097
:10BCF8002003C4F8403307F095FD754807F058FD58
:10BD0800002095E76F4803F0BEF9A4E795F848705E
:10BD180095F9693095F9392095F87D106D4E3846BA
:10BD280003F0CDFA009641B2EB6C95F850203846F6
:10BD3800143603F063FA0096EB6C95F8502095F9E9
:10BD4800701095F8480003F059FAD4F8C413AB6D95
:10BD5800D4F8D8230B44C4F8B033EB6D1344C4F8BB
:10BD6800B43394F80431042B07D02B6E0B44C4F879
:10BD7800B0336B6E1344C4F8B4330023089395F8BA
:10BD88002C3183B108A802F061FC00284AD195F94A
:10BD9800390094F837629DF82070FFF703FE3E449F
:10BDA80080B2B0423CD300238DF8133095F8393077
:10BDB8008DF8213095F838308DF82230D5F880305C
:10BDC8000993D5F884300A93238894F81164ADF860
:10BDD8002C3095F84800404B8DF820600DF1130287
:10BDE80008A903F01FFA012384F8353495F839308F
:10BDF80084F836349DF8133084F83734D4F8143482
:10BE0800C4F84464C4F83C34C4F84C3402F04DFB24
:10BE180050B1D4F8140402F05AFB28B1102007E7F7
:10BE2800082005E7132003E795F81831012B01D105
:10BE380002F04FFB02F03CFB0023059394F8043119
:10BE480095F9395094F81164BBB1042B7FF4EAAE2C
:10BE580005A802F037FE60BB94F80C341BB994F8BF
:10BE68000E34012B02D9059B013B0593154B059810
:10BE78003246E9B202F098FE02E0124802F06CFE87
:10BE8800A8B9D4F8403394F80C11218043F0020388
:10BE9800C4F8403394F8103423B994F80C340133BF
:10BEA80084F80C340D4B0E489B6A984728E71120FC
:10BEB800BEE61220BCE60E20BAE600BF64180020D9
:10BEC800D81F0020E0200020941800205C240020C7
:10BED8004023002090230020EC2300200C4601087A
:10BEE800DA1F002073B5144C144D04F57876EB6C0A
:10BEF80095F8502095F9781095F84800009603F0C9
:10BF08007DF940F2012395F84800A4F8F23304F2D1
:10BF18001C42314603F07EF958B194F81C3484F879
:10BF28005E34074B00205B6B984794F8F33384F832
:10BF3800803402B070BD00BFD81F002064180020F4
:10BF48000C460108F8B5334D95F81841012C064602
:10BF58004BD0022C51D064B938B9D5E91B0105F191
:10BF6800740383E803002046F8BD01283DD0022869
:10BF780001D00324F7E7284F85F8180107F5737EE9
:10BF8800BEE80F0007F5787CACE80F00DEF800305B
:10BF9800CCF8003095F8E93087F8F363E3B195F809
:10BFA8000031022B18D1D5F804316B67C7F8E43398
:10BFB80095F87D3095F8082187F8F03395F88C309E
:10BFC80085F8782087F8F13397F8112487F8E0236B
:10BFD80040F20133A7F8F233002387F810340F4BEF
:10BFE800DB6A9847FFF77EFFBDE702F063FA044675
:10BFF8000028B8D185F81861B5E70028B9D1064BF3
:10C0080085F81801062283F88024044BDB6A9847D8
:10C018003446A8E764180020D81F00200C46010801
:10C02800F0B5484C484EB4F8DC202287D4E92D01FD
:10C0380094F8B12084F8692004F16C0282E80300C6
:10C04800D4E92F0104F1740282E80300B4F8C42093
:10C05800A4F87C20D4F8CC20C4F884208FB0D4F87D
:10C06800D020D4F8C810C4F888200025374AC4F86E
:10C0780080100123A4F81E31C6F80C24C4E94E55DB
:10C0880084F82C51A56284F81B5184F83A50C4F8FE
:10C098003051A4F8345186F8105484F841518DF881
:10C0A800143004F5087394F84800A4F84251039337
:10C0B80003A904F52D73049303F088F8E36EC6F81A
:10C0C800D03394F87D3086F8DC3394F88C3086F8D9
:10C0D800DD334FF48073A6F8DE3386F8CC5306F5CB
:10C0E80073770FCF06F578740FC43B68236040F26E
:10C0F8000123A6F8F233D6F8483386F81154CDE96F
:10C1080001551BB15A685B6901920293104B069363
:10C11800A3F144020792A3F1140208920D4A0A926D
:10C1280025330993A2F19C030B93A2F198030C9376
:10C1380001A9131D06A802F274620D9302F0A4F976
:10C148000FB0F0BD64180020D81F002000010100C6
:10C158003424002048190020F8B50D4F0D4C0E4E20
:10C168000D4607F0D7FA3B6B984796F8480004F25B
:10C178001C42294603F04EF848B194F81C3484F860
:10C188005E34706D7B6B9847EB7C84F88034F8BD27
:10C198000C460108D81F0020641800200D4890F8AC
:10C1A800113480F8B8330C4B93F8692080F8BB231E
:10C1B80093F87D2093F88C3080F8C933002380F8F9
:10C1C800C823A0F8CA3300F56E7100F56070FFF758
:10C1D800C3BF00BFD81F0020641800200F4890F884
:10C1E8008034CBB190F8113480F8CC330C4BDA6E34
:10C1F800C0F8D02393F87D2093F88C3080F8DD3395
:10C208004FF4807380F8DC23A0F8DE3300F57371F7
:10C2180000F56670FFF7A0BF704700BFD81F002069
:10C228006418002070B5344C2421204604F064FFC3
:10C23800636A984218BF60624FF01C012F4814BF10
:10C248000125002504F058FF636C984218BF60640C
:10C258004FF0FC012A4818BF45F0020504F04CFFD6
:10C26800D4F84431984218BFC4F844014FF0D401BF
:10C27800244818BF45F0040504F03EFFD4F81C32EA
:10C28800984218BFC4F81C024FF090011E4818BF0E
:10C2980045F0080504F030FFD4F8B032984218BFD2
:10C2A800C4F8B0024FF49461184818BF45F010055F
:10C2B80004F022FFD4F85437984218BFC4F8540742
:10C2C8004FF01401124818BF45F0200504F014FF80
:10C2D800D4F86C3798420F4B18BFC4F86C07D3F8E2
:10C2E800483318BF45F040052BB11B691BB12846E0
:10C2F800BDE87040184770BD641800208C180020F5
:10C30800AC180020AC190020841A0020181B00204B
:10C31800BC1F0020D81F00202DE9F04F91B0002647
:10C32800BD4F8DF81560054688469346ADF81860F0
:10C33800B146C14502D311B0BDE8F08F15F8090028
:10C3480002F0C2F948444045F5DC15F8093009F116
:10C358000104023BE4B2112BEDD801A252F823F0FC
:10C36800B1C30008E1C30008A1C40008CDC4000897
:10C378005DC5000881C50008F5C5000829C6000884
:10C38800A7C600083FC300083FC3000807C7000846
:10C398003FC300083FC30008BDC70008E3C7000843
:10C3A80027C8000865C80008052002F039FA88B1D6
:10C3B8000521002002F0F8F92B5D87F8503409F1C7
:10C3C800030409F102095FFA89F9E4B215F80930A2
:10C3D80087F85134A146ACE700238DF816308DF864
:10C3E80017308DF81C308DF82030002E52D18B4E2E
:10C3F800631E2B440D9396F81A318DF83A3096F84F
:10C408007C308DF8393096F839308DF83B3096F815
:10C4180038308DF83C3096F868308DF83D30D6F8D5
:10C4280028310C9308AB019307AB009396F84800AA
:10C43800A8EB09090DF117030DF116020CA98DF8E7
:10C44800389002F0FBFE8DF8150000F00700072871
:10C458000BD19DF8163086F839309DF8173086F8DC
:10C4680038309DF81C3086F8683000264FF00509F2
:10C4780006E001220DF11501032002F03BF8013618
:10C48800F2B29DF82030B3FBF9F19142F1D8013BAB
:10C498002344DCB201269DE72B5D604903F00F03BE
:10C4A800012281F81B3109F1020902FA03F3A1F80C
:10C4B8001E315FFA89F9002206A9042002F01AF851
:10C4C8004C4687E707238DF815302B5DC3F302121E
:10C4D80003F00F038DF8303009F10303DBB28DF858
:10C4E8003120EA5C09F10403DBB209F10504EB5CD5
:10C4F80009F102095FFA89F91B0443EA022315F8D6
:10C508000920DFF8189113436422534399F848002F
:10C518000D930CA902F0A1FE00F00703072BE4B26B
:10C528008DF815000ED19DF8303089F8703089F8F3
:10C5380078300D9BC9F86C30C9F874309DF83130EB
:10C5480089F869308DF81800012206A9052001F044
:10C55800D1FF3FE7D7F8483363B11B6853B1984719
:10C568000BF03F038DF818008DF81930022206A948
:10C578000620ECE7FF20F3E703238DF815302B5D49
:10C588008DF824300CAB089309F10303DBB209F1F1
:10C598000604EA5C09F10403DBB208A9EB5C1B049E
:10C5A80043EA022309F10202D2B209F10509AA5CA1
:10C5B8001343642253435FFA89F90C9300230D93C4
:10C5C80015F809308DF83830144B93F8480002F00C
:10C5D8004AFEC3B20028E4B28DF81530FFF6FAAE71
:10C5E8008DF81830012206A90720B0E72B5D03F06B
:10C5F8000F03012B4FF47A7238BF01235343074AC4
:10C6080009F10209936503F57A73D3655FFA89F92D
:10C61800002206A9082051E7D81F0020641800202E
:10C628002B5D9C4CC3F340128DF81D2094F84800F4
:10C63800C3F3001207A903F00F038DF81C208DF82F
:10C648001E3002F016FE09F1020901305FFA89F97D
:10C658003FF436AFBDF81C308F4AA4F87C309DF803
:10C668001E309DF81CA0D05CF5F7D0F90223C4F861
:10C6780080000CA994F848008DF830308DF832A06D
:10C6880002F096FD94F93930089040B29842B8BF4C
:10C69800184684F83900002206A909200EE703236A
:10C6A8008DF815302B5D8DF8303009F10303DBB2BE
:10C6B80009F10504EA5C09F10403DBB209F1020996
:10C6C800EB5C5FFA89F91B0443EA022315F8092099
:10C6D8001343642253430D936E4B0CA993F84800FF
:10C6E80002F0CDFDC3B20028E4B28DF81530FFF694
:10C6F80071AE8DF81830012206A90A2027E70A2012
:10C7080002F08EF800283FF465AE0A21002002F0FE
:10C718004BF80023ADF8263009F10203DBB24FF4E1
:10C728007A71EA5C09F10303DBB20DF1300AEB5CC4
:10C738001B0443EA02232A5D134309F10402D2B21F
:10C7480009F1060409F10509AA5C5FFA89F943EAC7
:10C75800026315F8092003934A4312125046ADF8B4
:10C76800242006F0E7FE039B03F1965303F5A91373
:10C7780003F5EC530893D7F83C3300930DF12009E7
:10C7880099E80600D7F838330AA806F090FE0B9B04
:10C7980000939AE806000A9B484606F06DFE99E861
:10C7A800030006F09FFE01F08FFE0123E4B287F834
:10C7B80030340FE60D2002F033F800283FF40AAEBB
:10C7C8000D21002001F0F0FF97F88034043B012B85
:10C7D8007FF600AE01F074FEFCE509F10203DBB25E
:10C7E8002A5DE95C09F10303DBB209F10504EB5C9E
:10C7F80009F104095FFA89F91B0415F8090043EAED
:10C80800012313436421594300F00F0001F059FE3E
:10C81800E4B28DF81800012206A9112097E60E202F
:10C8280001F0FEFF00283FF4D5AD0E21002001F0F5
:10C83800BBFF09F10203DBB2184AE85C2B5D126802
:10C8480009F1040409F103095FFA89F943EA0020B0
:10C8580015F80910E4B201F036FEBBE52A5D09F1CE
:10C86800020309F1040409F10309DBB25FFA89F94B
:10C87800E95C15F809301B0443EA012313436420DB
:10C88800584301F022FEE4B28DF81800012206A9EF
:10C8980013205CE664180020833F0108E024002090
:10C8A8000E4B93F88124920703D593F87F24012A2D
:10C8B80006D90B4A92F81A1111B1916A01319162A5
:10C8C800002283F80C2483F8102483F80F24D3F86B
:10C8D800402322F00202C3F840237047D81F0020EB
:10C8E8006418002010B5124C04F55A7006F012FFB7
:10C8F800D4F84033012023F02003C4F84033FFF775
:10C908007BF998B10B2811D00A4B93F8393084F889
:10C918003634092094F80E3484F8393484F8350410
:10C9280001F064FFBDE81040FFF7BABF10BD00BFBB
:10C93800D81F002064180020074BD3F84023012A91
:10C9480006D03AB993F88204013818BF012070471D
:10C958000020704701207047D81F0020034BD3F8F0
:10C968004003431E58425841704700BFD81F00205B
:10C978002DE9F04FA5B0EFF3108172B6C04A002040
:10C988001368106081F31088BE4C002B00F0DA8029
:10C99800D9065FFA83FB6BD5BB4D95F81831022B8E
:10C9A80002D0BA4BDB6A9847EFF3108872B6B84FDB
:10C9B80006F06CFE3E68D4F8B013361A3144B54818
:10C9C80006F030FFB34806F0F3FED4F8B413B248CB
:10C9D800314406F027FFB04806F0EAFE88F31088D5
:10C9E80095F81831022B02D094F810348BB1162325
:10C9F8000EA995F848008DF8383002F0D9FBD4F824
:10CA0800B4130C900144A54806F00CFFA34806F0A7
:10CA1800CFFE3B6894F81124EB620AAF38468DF8D4
:10CA28006020199306F0ACFDD5F82431009304AECC
:10CA380097E80600D5F82031304606F038FD96E82C
:10CA480003001BAB83E80300D4F814341A9395F859
:10CA58002C3195F84800003B18BF012318A98DF820
:10CA6800613002F0AEFB94F810340BB984F8353419
:10CA78001BF0080F3AD08A4B834D5F681E89B3F9C3
:10CA88000A8093F90C90D5F8E420039200230793C9
:10CA980084F83834A4F81A3484F81D34C4F82034DF
:10CAA800A4F8243484F82634C4F8283484F81834D4
:10CAB800C4F82C3484F83034744B94F88024DB6A3E
:10CAC80084F87F24A4F87C8484F87E94984772487C
:10CAD80006F020FE3146384601F0DFFC8246002889
:10CAE80000F0E680A4F8728484F874941BF0040FB4
:10CAF8001AD0654B93F81831022B02D0634BDB6ACE
:10CB080098470220FEF72CFF84F8350401F06EFEEA
:10CB180094F8103413B1012384F80F3494F8813455
:10CB280043F0100384F881341BF0020F03D0062170
:10CB38000520FEF78BFF1BF0010F03D00421032013
:10CB4800FEF784FF01F0C6FC94F88124D0065FD577
:10CB5800002384F88234D4F84033190644BF23F004
:10CB68008203C4F8403312F0050F00F0C5820C2090
:10CB780001F056FE002800F0BF8294F88134DF07E8
:10CB880000F1BA825E0740F1CB82D4F8403323F03B
:10CB98000203C4F84033D4F8402382BB94F881548C
:10CBA80015F001011EBF2B4662F3000384F881349F
:10CBB80094F881345E0744BF6FF3820384F88134AC
:10CBC800012384F8823421B1D4F8443335481B68F2
:10CBD80098476D070BD5344801F02EFE01F05CFE36
:10CBE80028B194F8813443F0040384F8813401F0C7
:10CBF80060FC94F881346FF3041384F881340123C2
:10CC080084F8823494F8813443F0200384F8813422
:10CC180094F8813418070AD56FF3C303234984F8BD
:10CC28008134D4F84433A1F12000DB68984794F8A4
:10CC3800813499070AD56FF341031C4984F881347C
:10CC4800D4F84433A1F164005B68984794F88034C1
:10CC5800022B01D1FFF746F994F881349A0640F186
:10CC6800EC826FF3451384F88134D4F84033002BF9
:10CC780040F0E38225B0BDE8F04FFFF7D3BA00BF1C
:10CC8800D41F0020D81F0020641800200C4601087B
:10CC9800F02400205823002070230020CC230020FB
:10CCA800E02400200C24002020240020542400200C
:10CCB80095F81831012B0CD101F0F3FB804668B1CF
:10CCC800504601F0E3FB504601F0E5FB042384F8ED
:10CCD8007F347EB9012384F819344AE101F0E3FB7B
:10CCE8000028F6D0404601F0D2FB404601F0D4FBC4
:10CCF8000523ECE73B7802935B09013B062B00F226
:10CD0800ED81DFE813F00700EB019200EB018F00E3
:10CD1800EB01DB01102EDDD995F82C310E97F6B218
:10CD28008DF83C60002BD5D118A804F0F9F80EAAAC
:10CD380018A9FF2002F04CF89DF84830C3F303030C
:10CD480007468DF8203095F8480095F87D308DF825
:10CD58002130072208A902F03EFA002F5AD10028F4
:10CD680058D09DF843309DF842201199C5F8E41039
:10CD78001B0443EA02239DF8412002201343C5F80F
:10CD8800E03004F0DBF89DF8483095F8480085F865
:10CD98002A71C3F30212C3F3030385F8703085F8D0
:10CDA80078309DF8493085F86920012B38BF012378
:10CDB8004FF47A725343AB651344EB654FF00108A7
:10CDC8000DF14A03113E0CA90C9385F868808DF883
:10CDD800346002F008FA0223404685F82C3101F04D
:10CDE8001FFD18B14146384601F0DEFC94F81034B6
:10CDF800002B00F0798194F8383413B10020FEF745
:10CE0800E9FD94F8813443F0100384F88134FEF787
:10CE1800A7FD6BE6012001F003FD0028E6D0012103
:10CE28000720E1E7012384F8183495F87D308DF860
:10CE3800223094F81C348DF8213095F88C3095F810
:10CE480048000D3308A98DF8203002F0B1F9A6F199
:10CE58000D031BB2069023EAE37300B283423FF747
:10CE680039AF0B2E7FF636AFA24B219318A8FF23BC
:10CE780018978DF864608DF8883002F075F8804650
:10CE880000287FF427AF9DF86C301A99C4F82C1449
:10CE980013F00F0203D09DF8800000286CD19DF894
:10CEA800880000286AD0002A7FF414AF9DF88020FB
:10CEB800002A0CBF0227032700220792D5F8EC208E
:10CEC80091425DD195F8E910002959D0D5F80C1197
:10CED80095F8EAA00968079195F81811022902D176
:10CEE800032184F87F14032F7FF4F4AE13F0600F4E
:10CEF8007FF4F0AE03924FF00108152395F848002F
:10CF08008DF8203008A902F053F995F82A310690D7
:10CF1800BAF1000F37D0BAF1010F3ED1012B34D14D
:10CF28006FF009063E4106F00106C6F10206F6B2A8
:10CF380081B2BDF86E2007AB304601F0CFFD70B36B
:10CF4800072824D1082384F8193495F82A315BB9C5
:10CF5800029B03F0E003A02B06D16A6B239B9A4245
:10CF680002D1012385F83A30079BC4F82834C4F865
:10CF78006034FEF74FFDB9E547469DE701279BE77B
:10CF88004FF0010AB9E70426D2E70326D0E70828BC
:10CF980003D10A2384F81934E6E70123FAE718AB2A
:10CFA80000930399079B3246504601F063FE20B177
:10CFB80002280CBF0B230C238DE6079BC4F82834EA
:10CFC800C4F860349DF86C3084F81904C3F3401336
:10CFD80084F8263484F8383494F87F3484F81A8432
:10CFE800012B98BFA862B8F1010FC4F8200484F897
:10CFF800240484F8350433D1022284F8182495F8DF
:10D008003A20002A3BD19DF86C20D20637D4012B58
:10D0180094F834149DF86C2005D8012901D196069E
:10D0280001D501F001FB022F37D0032F09D09DF85D
:10D038006C10012F4A4601F00F011CA831D0FFF7F0
:10D048006BF99DF8803084F81B34219BC4F8203498
:10D058009DF8883084F82434012384F8253426E0A8
:10D06800029A02F0E002A02A11D195F82A110122B1
:10D0780085F83A2009B92399696384F8182495F842
:10D088001821002AC3D1012284F81D24BFE70022F9
:10D0980085F83A2084F81824B5E79DF88810219877
:10D0A8004A46FFF739F99DF8803084F81B3494F824
:10D0B800813443F0020384F8813497E6DFF8348042
:10D0C800013EB2B2791C404604F000F80323A4F8EC
:10D0D8001834C4F8208484F82464E8E7012384F829
:10D0E8001934FEF797FC81E695F81831022B7FF486
:10D0F80088AE83E61022002094F881345D070FD5AE
:10D10800012001F08DFB88B3012001F05FFB08B915
:10D1180084F80C04D4F8403323F00203C4F84033F5
:10D1280094F88114C8077FF536AD94F834340BB100
:10D13800032B26D1424B94F80C0493F868209042B4
:10D1480008D28A0750D593F818311BB194F87F3468
:10D15800002B49D13B4806F0DDFAD4F8403323F0E0
:10D168002003C4F84033FFF79BFB14E5062001F0C9
:10D1780057FB0028CED1072001F052FB0028C9D167
:10D18800CEE7012B30D194F80F24002A3FF403ADE9
:10D1980094F80E3494F80D04834204D211F002027C
:10D1A80018BF94F83824264D95F82A11002941D142
:10D1B80032BB834218D20133DBB2DF0784F80E3466
:10D1C80012D522238DF8603095F87C308DF86230C6
:10D1D80095F8480095F839308DF8613018A901F0B4
:10D1E800E7FF0E9085F8390094F8813400206FF33A
:10D1F800041384F8813484F80F04FFF773FBCAE43E
:10D2080094F838648EB902238DF8683005F50873F0
:10D21800189395F8480005F52D7318A9199301F08E
:10D22800D5FF84F8106484F8386494F80E3484F8D0
:10D2380039348FE7002AD7D08CE725B0BDE8F08FC6
:10D2480064180020402300202DE9F04F8A468BB057
:10D2580091460746002800F08D81002900F08A8158
:10D268000368002B00F086814368002B00F0828160
:10D278008368002B00F07E81C368002B00F07A8160
:10D28800104601F091FF002800F07681BC4CBD4D9E
:10D29800384601F03FFA4FF4EE620021204603F0D1
:10D2A80029FF4FF4A1620021284603F023FFB64B63
:10D2B800C4F8283100264FF001080F2305A9484675
:10D2C8008DF8143084F8489084F8186184F88C60DC
:10D2D80085F80E8485F80D8401F06AFF801B18BF5D
:10D2E80001204FF00A0B84F81C0105A994F84800A6
:10D2F8008DF814B001F05CFF4FF0060984F8DC00EB
:10D3080005A994F848008DF8149001F051FF1023F6
:10D3180084F8DD0005A994F848008DF8143001F070
:10D3280047FF1123C4F89C0005A994F848008DF81C
:10D33800143001F03DFF1223C4F8A00005A994F8A9
:10D3480048008DF8143001F033FF1323C4F8A4000B
:10D3580005A994F848008DF8143001F029FF14232A
:10D368000DEB0301C4F8A80094F848008DF81430B8
:10D3780001F01EFF1723C4F8AC0005A994F8480073
:10D388008DF8143001F014FF182384F8B10005A9B2
:10D3980094F848008DF8143001F00AFF1923C4F8F6
:10D3A800B400C4F8BC0005A994F848008DF81430FE
:10D3B80001F0FEFEC0B21E2384F8B80084F8C00055
:10D3C80005A994F848008DF8143001F0F1FE1F23E8
:10D3D80084F8C40005A994F848008DF8143001F0C9
:10D3E800E7FE202384F8C50005A994F848008DF8C5
:10D3F800143001F0DDFE2123C4F8C80005A994F813
:10D4080048008DF8143001F0D3FE0B23C4F8CC008B
:10D4180005A994F848008DF8143001F0C9FE0C23D2
:10D42800A4F8D00005A994F848008DF8143001F04C
:10D43800BFFED4F89C306365D4F8A030A365D4F857
:10D44800A430E365D4F8A8302366D4F8AC3063661A
:10D4580004F5087307A90490A4F8D200079394F878
:10D4680048008DF8246004F52D73089384F8B08083
:10D47800C4F894B084F89890C4F84CB084F85090EC
:10D4880084F8688001F0A2FEC5F848A3FEF7C8FD3D
:10D4980032463E4B00964FF0FF3105F55A70C4E90D
:10D4A8000B66C5F8447385F8816484F81981C5F85A
:10D4B800408306F0D1F83246354B00964FF0FF31E5
:10D4C80005F5607006F0C8F83246324B00964FF00A
:10D4D800FF3105F5667006F0BFF832462E4B009610
:10D4E8004FF0FF3102AE05F57D7006F0B5F8304615
:10D4F80006F046F896E8030004F5907383E8030005
:10D50800264BC5F84C33264BC5F85433254BC5F884
:10D518005C33254F254BC5F85033254BC5F8583398
:10D5280005F553703B68984704F5A47003F016FBA3
:10D5380020B1112630460BB0BDE8F08F204601F02F
:10D548009DFA0028F5D100F0C7FFB8B9194801F0D5
:10D55800F7FA06460028ECD17B69984703F094FD5A
:10D56800BB6D94F819019847FB6A9847012385F821
:10D578008234DFE70326DDE70926DBE71326D9E750
:10D5880064180020D81F002000030001EDC800081F
:10D59800A5C10008E5C10008DDB90008B5BB000851
:10D5A8006DBB000899B900080C46010845BB000886
:10D5B8001DBB00084C19002008B5034B0020C3F818
:10D5C8004003FEF7CDF908BDD81F002010B5FFF7BE
:10D5D800B3F90A4C60B90A4B93F81831022B02D1FF
:10D5E800084BDB6A98470123C4F84033002010BD7C
:10D5F800D4F84003013818BF0120F8E7D81F0020ED
:10D60800641800200C46010838B5134C04F55A700C
:10D6180006F080F804F5607006F07CF804F5667092
:10D6280006F078F804F57D7006F074F800F040FF15
:10D638000A4B0025DB6A9847C4F84053FEF7F2FD11
:10D64800074908484FF4EE6203F040FD0123C4F88F
:10D658004033284638BD00BFD81F00200C460108BB
:10D6680064180020F410002030B52A4B89B0054614
:10D6780093F8DD008DF8020093F8DC009A6A8DF8C3
:10D6880003000020019202900C4600293ED005922A
:10D69800D3F8882006921A8FD3F82811039152BA2A
:10D6A80093F81A11ADF81C2093F87C2093F84830B1
:10D6B8008DF810008DF811108DF81E208DF81F3090
:10D6C8000DF1030201AB0DF1020103A800F06EFE9B
:10D6D8009DF90200FEF766F9607002A800F0B6FF37
:10D6E800B0B9029A0F2A0DD863789A420AD815441D
:10D6F800AB42A3EB02012CBF002001202170C00027
:10D7080009B030BD002323700820F9E70320F7E7AC
:10D718001320F5E7641800201FB50446002800F020
:10D72800FD8000783F2800F2F380DFE810F0400029
:10D7380046004B005000540058005D00F100F10015
:10D74800F100F100F100F100F100F100640068005F
:10D758006C0077007E0081008400890087008B00C0
:10D768008F009200950098009B009E00A200AA00DE
:10D77800A600AE00B100B500BE00BA00BC00F100C2
:10D78800C200F100F100F100F100F100F100F10038
:10D79800F100F100F100F100F100F100F100F100F9
:10D7A800CA00CE00D300D700DB00DF00E8005D4BE5
:10D7B80093F81831237104B010BD5A4B93F82C31EB
:10D7C800237102E0606803F065FB0020F3E76068FE
:10D7D80003F0A6FBF9E7534B93F81A31F0E7514BE6
:10D7E800D3F8E0306360F0E74E4B211D93F82C012D
:10D7F80003F0AEFBE9E74B4B93F81931E0E7494BEF
:10D8080093F88C30DCE71D238DF80830454B02A9CE
:10D8180093F8480001F0CCFC6060D6E7424B043432
:10D8280093E8030084E80300CFE7404B0434F7E7AC
:10D838003F4B0434F4E73F4B0434F1E71B23E3E7A1
:10D848001A23E1E7374B93F86830B9E7354B5B6D3E
:10D85800C8E7344B9B6DC5E7324BDB6DC2E7314BF4
:10D868001B6EBFE72F4B5B6EBCE72E4B93F8DD308A
:10D87800A6E72C4B93F83930A2E72A4B93F8DC3013
:10D888009EE7284B93F838309AE7264BDB6CA9E7DC
:10D89800244B93F8503093E7224BD3F884306360DD
:10D8A80093E7204B9EE7244B9CE71E4BD3F8CC30E4
:10D8B800F5E71C4BD3F82831636001F00DFDA0603B
:10D8C80083E7184BD3F890308CE7164BB3F88830C1
:10D8D800A3807AE7134BB3F88A30F9E7114BB3F812
:10D8E800D030F5E70F4BB3F8D230F1E70D4B93F892
:10D8F80048200AB1062A13D1B3F84C37E8E7094B98
:10D9080093F848200AB1062A0AD1D3F8503769E7B4
:10D91800204604B0BDE8104000F0CEBD03204AE721
:10D92800182048E764180020D01800201819002093
:10D93800D818002020190020F410002073B50446E0
:10D9480000285ED0A04DD5F840339A0700F15F82D9
:10D9580002783F2A00F25682DFE812F040004600C3
:10D968004E0056005A005F00640070007A007F0085
:10D97800840089008E00930098009D00A70054023F
:10D98800AC00CC00DF000601280119012C013C0184
:10D998004001440148014C01500162018A017801AB
:10D9A8009C01A201A901AE01B3015402180254025C
:10D9B80054025402540254025402540254025402AF
:10D9C80054025402540254025402540254022702CC
:10D9D8002C02310236023B0240024A02007902B0B0
:10D9E800BDE87040FEF7AEBA0379022B09D0774A3A
:10D9F80082F82C31002005E0406803F03DFA002849
:10DA0800F8D0032002B070BD406803F079FAF6E759
:10DA18006E4B027983F81A21ECE76C4B4268C3F825
:10DA2800E020E7E7694D416895F82C0103F086FA94
:10DA38000028E6D16368C5F8E430E3E741680029C7
:10DA4800DFD0002001F0A8F90028D3D01120D9E7B1
:10DA580041680029D5D00120F4E741680029D0D0D9
:10DA68000820EFE741680029CBD00920EAE74168A0
:10DA78000029C6D00C20E5E741680029C1D00D2057
:10DA8800E0E741680029BCD00E20DBE741680029A7
:10DA9800B7D00F20D6E74E4C4C4B007983F81901CC
:10DAA800A36D9847E36A9847A4E7484B027983F83F
:10DAB8008C209FE7454D037A8DF8003095F8480093
:10DAC80095F87D308DF801300722694601F083FB17
:10DAD800002896D0636895F84800009300226946AC
:10DAE80001F079FB00288CD06C35D4E9010185E878
:10DAF80003007FE7354D037A8DF8003095F848002C
:10DB080095F87D308DF801300722694601F063FBF6
:10DB180000283FF476AFB435E7E72C4D037A8DF84B
:10DB2800003095F8480095F87D308DF801300722CF
:10DB3800694601F050FB00283FF463AFD4E90101C6
:10DB480005F1740383E8030095F81831022B7FF47C
:10DB580051AF95F82C31002B3FF44CAF1C4BDB6ACE
:10DB68009847FEF7BFF945E7184D037A8DF800305E
:10DB780095F8480095F87D308DF801300722694600
:10DB880001F029FB00283FF43CAFBC35ADE7436802
:10DB9800009301238DF804300C4B694693F8480034
:10DBA80001F026FB00287FF425AF2AE7436800939D
:10DBB8000023EFE703795A1E0E2A3FF622AF034AE5
:10DBC80082F8683016E700BFD81F002064180020CC
:10DBD8000C460108904B42685A650BE78E4B426829
:10DBE8009A6507E78C4B4268DA6503E78A4B426817
:10DBF8001A66FFE6884B42685A66FBE6864C03794C
:10DC080094F848008DF800300622694601F0E3FADE
:10DC180000283FF4F6AE9DF8003084F8DD30E9E6E0
:10DC28007D4C03798DF8003094F8480094F87C30E6
:10DC38008DF802300522694601F0CDFA00283FF43C
:10DC4800E0AE9DF8003084F83930D3E6724C0379A1
:10DC580094F848008DF800300A22694601F0BBFAB2
:10DC680000283FF4CEAE9DF8003084F8DC30C1E6E1
:10DC7800694C037994F848008DF800300922694608
:10DC880001F0A9FA00283FF4BCAE9DF8003084F8F2
:10DC98003830AFE6604B4268C3F89420DA64A9E6EE
:10DCA8005D4B027983F8982083F85020A2E65A4BFE
:10DCB8004268C3F884209DE6574B4268C3F8CC20DD
:10DCC80098E6012B40F0A380544C2421204603F011
:10DCD80013FA636A984201D0172093E61C2104F1D5
:10DCE800280003F009FA636C9842F5D1FC2104F18D
:10DCF800480003F001FAD4F844319842ECD1D42119
:10DD080004F5A47003F0F8F9D4F81C329842E3D172
:10DD1800902104F5087003F0EFF9D4F8B032984276
:10DD2800DAD14FF4946104F52D7003F0E5F9D4F8D5
:10DD380054379842D0D1142104F5EB6003F0DCF994
:10DD4800D4F86C379842C7D1334E214630464FF449
:10DD5800EE6203F0BBF920464FF4EE62002103F0B7
:10DD6800C9F995F8113485F8E033736FC5F8E433D1
:10DD780096F87D3085F8F03340F20123A5F8F233A8
:10DD8800274B96F819019B6D984733E68379012B49
:10DD98003FF637AE204B42684068C3F8282100F0B0
:10DDA80089FE00283FF42EAE50E61B4B4268C3F8AC
:10DDB80090201FE6184B8288A3F888201AE6164B95
:10DDC8008288A3F88A2015E6134B8288A3F8D0200E
:10DDD80010E6114B8288A3F8D2200BE60E4B93F87D
:10DDE80048200AB1062A14D1A288A3F84C2701E6D4
:10DDF800094B93F848200AB1062A0AD16268C3F889
:10DE08005027F7E502B0BDE8704000F057BB01208D
:10DE1800F8E51820F6E500BF64180020F41000208B
:10DE28000C4601082DE9F04186B00023ADF800301A
:10DE38000646002800F0E280FEF77EFD20B10124AE
:10DE4800204606B0BDE8F08100F02CFD0028F6D190
:10DE580000F022FD014618B96948142203F04AF976
:10DE6800684D95F88134012243F0040385F849246C
:10DE780085F8813433788DF804300021013B8DF822
:10DE880005208DF807100D2B00F2B080DFE803F0B5
:10DE980007AEAEAE525A7DAEAE85AEA28F9ED5F815
:10DEA800404314F02004CAD1DFF85C81574FFEF7D5
:10DEB800B7F8224696F9051098F8480001F0E5F9F8
:10DEC80088F83900B37988F83830204607238DF868
:10DED8000530FEF737F8FF2307F58670A5F80C31F3
:10DEE80085F80441C5F8087103F01AF807F58A7037
:10DEF80002F0D0FF2046FDF77FFE044640B196F9B8
:10DF0800051098F84800012201F0BFF988F8390097
:10DF1800D5F884343361002C6CD000F0BDFC0028A7
:10DF28008ED195F8813485F8100460F3820385F862
:10DF3800813485E700226946022000F0DBFA10B33D
:10DF48001324E5E795F811348DF808302E4BB28884
:10DF580093F839108DF8091093F838108DF80A10D5
:10DF6800D3F880100391D3F88410049193F84800F3
:10DF7800ADF8142002A901F09DF9D5F8403343F01B
:10DF88000203C5F840330024C2E7214BB28896F952
:10DF98000C10B068DB6B9847EFE702A90D2000F082
:10DFA80027FB0028EFD0002269460D20C5E7164B55
:10DFB80093F81831D3B9347904F0070000F077FAF0
:10DFC8008DF80040012269461020B6E70022694614
:10DFD8001220B2E78DF8072000F05AFA044638B943
:10DFE80000F053FA204600F055FA91E702248FE733
:10DFF80001248DE701A800F0A1FB21E703241FE716
:10E0080020240020D81F002064180020DA1F0020D8
:10E018000C4601082DE9F04F91B000260391054602
:10E0280018B9032011B0BDE8F08FFEF785FC8246D1
:10E03800002840F06481B84C14220146074604F2D7
:10E04800344003F057F8012384F8353484F80E344B
:10E058002A789A4200F0B080032A00F0BF80002A94
:10E0680040F0C98084F80D34022295F80490D5F860
:10E078000880AE8995F90EB062F347179A46A74B08
:10E08800022493F87C2093F848008DF8244009A9CD
:10E098008DF8262001F08CF8BAF1000F00F02D81E0
:10E0A8009E4B93F81A21B2B940B25845B8BF5846AA
:10E0B80093F87C208DF814008DF8162093F848000A
:10E0C800052205A901F087F80028AAD0934B9DF8EE
:10E0D800142083F83920198F1A8F93F82C01029194
:10E0E800996A069152BA002800F0058193F81B013D
:10E0F80000B9186393F81801ADF83C20013893F87B
:10E108007C208DF83E20D0F1000B93F848208DF844
:10E118003F204BEB000B824A93F83A0093F81A41E0
:10E1280001900D914FF00100D3F88810D3F82831F1
:10E138008DF830000E910B93511C06AB0BA88DF88F
:10E14800314000F033F9019B4FEA0B1B4BEA431BAC
:10E158004FF0000A4BEA801B4BEAC413D0456E4CC3
:10E16800019308BF56463246414604F59C709B46CB
:10E17800CDE907AAA4F800A084F810A402F0A6FF2D
:10E18800F9B2A770C7F34217F2B2042F634E019B8E
:10E1980084F8372233D0072F00F09D80022F32D029
:10E1A8000220029B33875C4B002283F810245A4BD1
:10E1B800D3F884342B6135E7EB7B082B28BF082381
:10E1C80084F80D34042395F80490D5F80880AE89B6
:10E1D80095F90EB063F34717924650E784F80D346B
:10E1E800D5F804802E8995F90AB067F01F079A467A
:10E1F8004FF0000943E7D346D046D1463FE74FF0FA
:10E20800010084F81004474F84F80D11042084F8A5
:10E218000401FF20D6F8E41084F80C0184F81431C6
:10E2280007A807F59B73C4F8087184F82891C4F807
:10E23800101184F83021C4F82C3100F043FC002878
:10E2480057D1079BA4F8380408A8A4F81631C4F8D5
:10E25800403400F0FBF960BB089BABB196F939007C
:10E26800FDF7A0FB94F837322BB3089B0F2B19D876
:10E2780007F58B7208A90F2000F0F4F9C8B9089BBC
:10E2880063F3030B84F814B10398FDF7B5FC002879
:10E2980087D1069B86F83A00B36200F0B7F980B3DD
:10E2A800132080E707F2864208A900F0DBF900286E
:10E2B800EAD0132075E707F286473A4608A900F026
:10E2C800D1F90028F5D1089B84F82801C4F82C71ED
:10E2D80084F83031D8E7B8F1000FD5D0002AD3D070
:10E2E8004146E01C02F0F2FE94F8373201332380F5
:10E2F800CAE7122055E7072055E7204657E70120CF
:10E3080090E62B7884F8343494F8813443F0010390
:10E3180084F881344BE700BFD81F00206418002020
:10E328009C180020DA1F002037B50B4D8DF804002B
:10E3380004460F2295F8480001A900F04CFF40B1AF
:10E34800064A85F81C4192F8813443F0200382F88C
:10E35800813403B030BD00BF64180020D81F0020EE
:10E3680010B5FFF733F90446A0B90B4805F0D2F908
:10E378000A4805F0CFF90A4805F0CCF9094805F034
:10E38800C9F900F095F8FDF74BFE074BDB6A984793
:10E39800204610BD0124FBE740230020582300201D
:10E3A80070230020CC2300200C4601082DE9F04FF3
:10E3B80090F802908BB004468A460192B9F1000F9A
:10E3C80060D14579816890F9102090F91180196021
:10E3D800002D55D0817C8DF81610C07C4FF0020BB3
:10E3E80005A9CDE902238DF814B000F0E1FE029AE8
:10E3F80047B2BA421646B8BF3E46BA420CDC039B47
:10E40800C3F800904D46019B8AF8006083F80080AD
:10E4180028460BB0BDE8F08FA268A189E3898A423B
:10E428000B4434BF002501259A42ECD3082305A9E3
:10E43800E07C8DF8143000F0BBFEE289A368B3FBE2
:10E44800F2F102FB1133012B4FFA80F8DBD12223C2
:10E458008DF81430E07CA37C8DF8156005A98DF843
:10E46800163000F0A5FE46B2B742CCD12579002D72
:10E47800C9D0E07C8DF824B007A900F0A7FEC1E759
:10E488001646C0E70025C3E77047704770477047D6
:10E498000020704770477047704700207047002081
:10E4A8007047002070470020704700207047704771
:10E4B800704770470220704702207047022070475B
:10E4C8007047002070477047704700207047002051
:10E4D800704770477047000010B5054CFC22204675
:10E4E800002102F007FE0020C4E9000010BD00BFB3
:10E4F800F42400202DE9F04180461546002942D039
:10E50800244B002403F1010C1A462001103312F8A1
:10E51800016F002E39D19A42F9D11F4F3B680BB9D0
:10E52800C7F800C07B680BB1C3F800C03B180022D5
:10E5380001349A6083F80C800D302301AAB2384464
:10E54800FD50C7F804C002F0C1FDB8F1050F17D09F
:10E55800A8F10808B8F1020F8CBF4FF000084FF07F
:10E56800010807EB041400236371D7F8F83084F826
:10E57800048001332B44C7F8F8303046BDE8F081F9
:10E588004FF00108EDE70126F7E701340F2CB9D168
:10E598000226F2E7FB240020F424002010B510B373
:10E5A800124A1368984204D103681360002304E0F8
:10E5B8000B4613B119688842FAD15168884208BFDE
:10E5C80053600BB101681960D2F8F8308168013BDB
:10E5D80000245B1A04602146C2F8F830102202F0C9
:10E5E80089FD204610BD0120FCE700BFF42400206F
:10E5F800054B1B6813B11A798242FAD1002B0B60C4
:10E608000CBF032000207047F424002010B5054BF0
:10E61800186800B910BD037B04680BB9FFF7BEFF8B
:10E628002046F6E7F424002010B5074B186800B917
:10E6380010BD03790468052B02D0083B022B01D8D2
:10E64800FFF7ACFF2046F2E7F424002028B1044B82
:10E65800D3F8F8300360002070470120704700BFEE
:10E66800F42400202DE9F04107460E4615463AB33A
:10E6780031B3144B1C6800232CB93046FFF7E6FF72
:10E688000020BDE8F081A268F91A0132914210D346
:10E698002279EA54581C22895FFA80F8611D55FADC
:10E6A80080F002F013FDA368246898445FFA88F3A9
:10E6B800E2E720462468FFF771FF002CF9D1DCE778
:10E6C8000120DEE7F42400200238C0B211289ABFE6
:10E6D800014B185C00207047933F010830B50B4B85
:10E6E80093F820200446084672B100211C330578AF
:10E6F800A54208D001319842CDB20CBF044804307D
:10E70800AA42F4D8002030BD1046FCE7F0250020CE
:10E71800FC25002010B5084C00232060142204F1C9
:10E728000C00FF2184F82030C4E9010002F0E2FC6B
:10E73800012384F8213010BDF025002010B50E4AC1
:10E7480092F82010042915D8936804781C7044782E
:10E758005C70C078D87001310020987082F8201061
:10E7680002F11C018B4214BF043302F10C039360C5
:10E77800012010BD0020FCE7F0250020094B93F88C
:10E78800200068B15A6803F11C018A4200F1FF3089
:10E7980014BF043203F10C0283F820005A600120F0
:10E7A800704700BFF025002010B5074B93F82020D4
:10E7B8000446084632B15968FFF790FF10B10123AB
:10E7C8004470837010BD00BFF025002008B5064BCB
:10E7D80093F820202AB15968FFF780FF08B14078E4
:10E7E80008BD0120FCE700BFF025002030B50A4A2B
:10E7F80092F82010536882F8210061B191680124D1
:10E808001C32DD78587005B99C7093420CBF034BDD
:10E8180004339942F5D130BDF0250020FC250020B5
:10E8280008B5044B5968FFF759FF003818BF012095
:10E8380008BD00BFF02500202DE9F3410422154E44
:10E84800044600210DEB020096F8208002F052FCED
:10E858000025EBB2984502D802B0BDE8F081736894
:10E86800197821705A7862709F785FB133682046B2
:10E878009B689847FFF782FF17B901A8FFF75EFF6B
:10E888000135E6E7DB788DF804108DF805208DF862
:10E898000730EFE7F0250020014B93F82000704780
:10E8A800F0250020034B93F82000042894BF002093
:10E8B80001207047F02500201FB50024CDE902444F
:10E8C800C41F8DF800408DF801100C0AADF8042023
:10E8D800090C120C8DF803108DF806208DF80730FE
:10E8E80002461B0A012168468DF802408DF808305F
:10E8F80002F05DFA002818BF0F2004B010BD2DE902
:10E90800F04188B017460D460F9A064600284DD0AC
:10E9180000240121CDE904448DF810109DF8381029
:10E928008DF81510ADF81630190CCDE900441B0E02
:10E93800CDE902448DF81930ADF81A20130C120EE7
:10E9480007948DF818108DF81C308DF81D20E3B24F
:10E958004FEA0318002D5FFA88F803DC002008B09E
:10E96800BDE8F081013310218DF81F303A466B461F
:10E978000DEB010002F0B1F90346C8B9102DAC4601
:10E98800A8BF4FF0100CDAB2624503F1010303DBB4
:10E99800103D2DB20134DAE708EB020020326A4458
:10E9A800315C12F8202C4A403254ECE70A20D6E7B2
:10E9B8000F20D4E70138032815D8DFE800F0020853
:10E9C8000C100A4B1B681B690B6000207047074B33
:10E9D8001B685B69F8E7054B1B689B69F4E7034B09
:10E9E8001B68DB69F0E70520704700BF142600208C
:10E9F8002DE9F041C4B00C464A9E17461D46804694
:10EA0800B8B3B1F5807F36D84FF4887200216846D4
:10EA180002F070FB492300934FF48073ADF8043083
:10EA28002B0C8DF80830330CADF80650ADF80A60A1
:10EA38008DF80C3022460023414604A82D0E360ED0
:10EA48008DF80E308DF809508DF80D608DF80F4057
:10EA580002F03CFB04F110014B9A3B4689B2684630
:10EA680002F025F910B1012818BF0F2044B0BDE805
:10EA7800F0810A20FAE70E20F8E7000010B590B1FF
:10EA88000A4C28220021206002F034FB2368084A3F
:10EA98001A6000204FF0FF32C3E90302C3E90522E0
:10EAA800C3E9072210BD0920FCE700BF1426002097
:10EAB80000010101024B1B6818600020704700BF6D
:10EAC8001426002030B1044B1B68DB680133036057
:10EAD800002070470A2070471426002073B50E46A0
:10EAE800002101911D4633B301A9FFF763FFD0B997
:10EAF800019C631C04D0A3B2D31A002B10DDE218CA
:10EB08000E4B2A601B689B786BB9121B63EB0303DF
:10EB1800B24273F10003ACBF01200020C00002E044
:10EB280003D12C60072002B070BD230C1B0403F531
:10EB380080331A44E4E70A20F5E700BF14260020D2
:10EB480028B1044B1B681C334362002070470A201D
:10EB5800704700BF142600201FB50446F0B10023FB
:10EB680003A8039302F07AF90E4ABDF80C30126834
:10EB780020469380E38200F052FA60B904F118034A
:10EB8800009321680123132202F088F840B9204637
:10EB980000F045FA00B1112004B010BD0A20FBE7CF
:10EBA8000F20F9E714260020F0B5054687B01C466B
:10EBB8003BB32F4E3368DB68834257D894F8202044
:10EBC800002A14BF09220822834205D3204600F0F8
:10EBD8005AFA70B111200AE0002301900093A3684B
:10EBE80094F82810606AFFF78AFE0028EED007B074
:10EBF800F0BD23792168B4F808C0A768043B9AB22D
:10EC080009B90A20F3E7B2F5807F2DD8ADF80EC018
:10EC18008DF817304FEA174C04F12C033F0E8DF88E
:10EC2800117000932F0C08234FF0490EADF80C001B
:10EC38008DF814708DF816002F0E0DEB0300CDF82B
:10EC480008E08DF810C0ADF812508DF8157002F07C
:10EC580025F808B10F20CAE7204600F014FA00286A
:10EC6800B8D13368DD60C2E70E20C0E70620BEE7F2
:10EC7800142600202DE9FF410A9D80460F461646BE
:10EC88001C46002D5AD0002303A910460393FFF712
:10EC980091FE18B1062004B0BDE8F081039B9C42A8
:10ECA80001D80133F6D1284600F05EF9002847D193
:10ECB800264B1A78424503D01A79424542D10120A1
:10ECC800AA68BA4240D103EB8002EB6A92F801804D
:10ECD8002979CDE900430439927828683B4689B2FE
:10ECE800FFF786FE0028D6D195F820300194002B36
:10ECF8004FF00103009314BF4246082295F82810EC
:10ED0800686A3B46FFF7FBFD0028C4D1013E032E8D
:10ED1800C1D8DFE806F002070B0F0D4B1B681C611A
:10ED28001C62B8E70A4B1B685C61F9E7084B1B6873
:10ED38009C61F5E7064B1B68DC61ACE70A20AAE793
:10ED48001020A8E70C20A6E70220A4E7B4080020BA
:10ED5800142600201FB50A460B2A4FF00001CDE902
:10ED68000011CDE9021107D00C2A13D00A2A0FD0BE
:10ED78000B2005B05DF804FB012802D120238DF893
:10ED88000030684602F013F8002818BF0F20F0E79B
:10ED98003023F4E70B21F4E738B5054602F002F812
:10EDA800044678B97DB9094B1B680B219878FFF7A1
:10EDB800D1FF38B90C21FFF7CDFF18B90A21FFF7A9
:10EDC800C9FF00B10F24204638BD00BF142600201B
:10EDD8002DE9F04380468FB00C461746002A6BD0C9
:10EDE800002969D0002529461D2206A8059504F0AA
:10EDF800A3FE8DF81350344D2B680DF114099E882D
:10EE0800CDF804900DF1130302933B7900933B680E
:10EE180032462146404601F0E6FF00284ED13868C8
:10EE28003A79494602F052F9384600F04FF800287E
:10EE380046D13C7AFA79BB79240444EA02241C437B
:10EE48002B689A6894423DD99C609DF813000B2169
:10EE5800FFF780FF034658BB0C21FFF77BFF0346F3
:10EE680030BB0A21FFF776FF034608BB7B7ABA7AE4
:10EE7800FF7A3F0447EA02271F433A4633462146B2
:10EE88000920FFF719FD034690B933463A46214653
:10EE98000820FFF711FD034650B92A689DF81310A2
:10EEA80091700021D1604FF0FF31C2E904119161E6
:10EEB80018460FB0BDE8F0830A23F9E70F23F7E7F8
:10EEC8001023F5E70323F3E71426002010B50446C2
:10EED800002845D00168002942D011F8013B437150
:10EEE8000322063002F0F2F82046032250F8091BEC
:10EEF800043102F0EBF82168CB79E3600A7A43EA3F
:10EF08000223E3604A7A43EA0243E3608A7A43EAE7
:10EF18000263E360CB7A23740B7B63742379212B20
:10EF28001AD110220D3104F1120002F0CFF81D227F
:10EF38002168501C8B5C6362085C43EA0023901CC8
:10EF48006362085C033243EA004363628A5C43EA13
:10EF580002636362002010BD112B03DC0D22E7E77A
:10EF68000220F8E70120F6E710B50446002854D03F
:10EF78000168002951D00B7843714B7883608A78F7
:10EF880043EA02238360CA7843EA024383600A792A
:10EF980043EA026383604B7903738B79C381CA792F
:10EFA80043EA0223027BC38102F00F0208311030CA
:10EFB80002F08CF8237B002203F00F0384F8202052
:10EFC80084F82820227903F10800111A04290DDD9C
:10EFD80021680933043AD21A085C84F82000D2B2B6
:10EFE800606A84F82820194402F070F823792268AE
:10EFF8001A44002012F8043CE36212F8031C43EAA6
:10F008000123E36212F8021C43EA0143E36212F8A7
:10F01800012C43EA0263E36210BD0220FCE710B54D
:10F02800044660B3036853B30279162A29D9427992
:10F038001A700146082251F8060B013002F050F808
:10F048002146082251F80E0B093002F049F82368CE
:10F05800E28A5A74E38A22681B0A93742368A269B5
:10F06800DA74A36922681B0A13752368628B5A75C0
:10F078002368E27E9A7517232371002010BD0120B2
:10F08800FCE70220FAE738B50446002863D0016897
:10F09800002960D0037B90F8282003F00F03002A92
:10F0A80057D10833207904321344984255D36379F1
:10F0B8000B702368A2685A70A36822681B0A9370B1
:10F0C80023686289DA702368E27A1A712368227BDE
:10F0D8005A712368E2899A71E38922681B0A2146DA
:10F0E800D371227B51F8100B02F00F02083001F0A7
:10F0F800EDFF237B94F8282003F00F0303F10805A4
:10F108002AB1226894F82010515503F109052068A6
:10F1180094F82820616A284401F0D8FF94F8283030
:10F128002268E16A2B44D1545A1CE16A206892B2E1
:10F13800090A81549A1C2168E08D92B28854DA1C1D
:10F14800216894F82F0092B2043388542371002068
:10F1580038BD0933A6E70120FAE70220F8E70000E6
:10F16800024B1A8810431880704700BF18260020E9
:10F1780008B5074B1B883BB1FEF728FA00280CBFDF
:10F1880000206FF0020008BD6FF00100FBE700BF30
:10F198001826002010B5034B00241C80FEF70CFA3B
:10F1A800204610BD18260020B0FA80F040097047AC
:10F1B80082B018B9084602B000F0D0B8002002B0FA
:10F1C800704710B9084600F083B9704710B908466F
:10F1D80000F09AB970470346084611460BB900F08B
:10F1E800E7B90020704710B9084600F045BD7047E0
:10F1F80010B9084600F008BA0020704710B4044659
:10F20800084611461A46019B14B910BC00F01ABAF8
:10F2180010BC70470346084611460BB900F044BAC3
:10F228000020704710B40446084611461A4614B91F
:10F2380010BC00F0B1BA002010BC704730B40546CD
:10F24800084611461A46DDE902341DB9029430BC5D
:10F2580000F02EBB002030BC704710B9084600F003
:10F26800DFBB0020704710B9084600F043BD0020FE
:10F27800704710B9084600F0EEBB0020704710B97F
:10F28800084600F0EBBB00207047034608461146CD
:10F298000BB900F005BC0020704710B404460846BE
:10F2A80011461A46019B14B910BC00F0FBBB09209B
:10F2B80010BC704710B9084600F03CBD704710B448
:10F2C8000446084611461A4614B910BC00F05CBD45
:10F2D800C8B210BC70470000004870470300010125
:10F2E800064B10B51B6A0446984730B10448054BD5
:10F2F800204498428CBF0020012010BD0C46010814
:10F30800403576C9405DC600F0B5114B85B00C4656
:10F3180010491F56054601F045F80F4BE4B25E6AE6
:10F32800072D4FF00103CDE9024301460AD105221A
:10F338000023CDE900234FF47A727A431846B04788
:10F3480005B0F0BD08220020CDE900203A46F5E7D7
:10F35800CF3F0108A83F01080C4601081FB500234C
:10F3680000930378013B382B00F28580DFE803F037
:10F378001D2383838320838383834042444B8353A9
:10F3880056595C5F6265836D206F74797B7E7E80E1
:10F398008725838383838383838383838383838989
:10F3A8008B908383899083929600C378002B62D0D8
:10F3B800022300935FE08378F8E743788DF8043000
:10F3C80007238DF805308378003B18BF01235B00C5
:10F3D8008DF8063010238DF80730334B1B6801A8D1
:10F3E80003F59062CDE9022300F0BCFF009042E0F3
:10F3F8004023DEE72023DCE7827890F9013042B928
:10F408002A4AD35CD5E7827890F901300AB9284AAC
:10F41800F7E7284AF5E740F6B833CAE74FF47A73B6
:10F42800C7E74FF4FA63C4E741F28833C1E741F212
:10F438007073BEE74FF48043BBE71F484FF47A71FF
:10F4480001F028FE00F5FA60D0E71C4BB1E7164B37
:10F458001B6803F59063ACE7134B1B6803F28C43FE
:10F46800A7E71023A5E7104B1B68A2E70123A0E735
:10F478004FF083430093009805B05DF804FB104BF0
:10F48800F8E7104B95E740F21123ADF80030F2E7AA
:10F4980003238EE790F901300B4AB2E70B4990F944
:10F4A800010000F07FFFA1E720260020DF3F0108D0
:10F4B800EF3F0108E73F010818FCFFFF00EA0637A5
:10F4C8009A99094040F70937CF3F0108A83F01083A
:10F4D80037B50B4B02781B680C2101FB02335B7AB2
:10F4E80003EB4304074B1D6803690093C368427824
:10F4F800816805EBC40000F0D5FC03B030BD00BF47
:10F50800202600201C26002030B587B0027A64230C
:10F51800ADF80030012A4FF00003CDE90133CDE901
:10F52800033301468DF802308DF8143027D0022AB3
:10F538002ED012BB006800B34B68F3B1194A1A4CBD
:10F54800106069461822236001F0C0FD174B24683B
:10F5580093E807000C3384E8070093E8070004F1F8
:10F568000C05032385E80700A4F88C34012204F273
:10F578008C4104F5906000F086FC07B030BD0A4964
:10F5880008684360036100F28C4100F59060F2E77F
:10F59800054B1B68B3F88024B3F88C140A43A3F80E
:10F5A8008024EAE71C26002020260020FC3C0108D5
:10F5B80008B503460A2924D8DFE801F006232323E7
:10F5C800230B161B23212100BDE808400068FFF724
:10F5D80087BE90F900009978072271B900F013FCF2
:10F5E800003818BF012008BD052293F9000000214A
:10F5F800F4E790F900005978EEE70221EEE70722D8
:10F60800F3E70020EFE7000010B504791CB1012CE6
:10F618000BD0002010BD0A4B01681B68012203F5BE
:10F62800906000F030FC0120F4E7054B01681B688E
:10F63800224603F28C4000F026FC2046EAE700BF91
:10F6480020260020F7B50728144D1C46A8BF072020
:10F6580058700E462946174600F0A4FE94F901306A
:10F66800A070072B13D1322000F09CFD0C4BDB6DF2
:10F678000546984704F10C020834034601920094A9
:10F688003A463146284600F092FD03B0F0BD054ADF
:10F6980055F82310D05C00F07DFDE7E7A83F01088E
:10F6A8000C460108CF3F01082DE9F04F344F90F97F
:10F6B80001607B68D0F804908BB004468846984770
:10F6C8000546002859D1E37C73B92E4A237812687D
:10F6D80003EB4303990002EB8303D3F80490B9F1D9
:10F6E800000F01D152F80190274B484613F906B094
:10F6F800FB689847A37CD7F818A022890993072E9E
:10F7080028D100230121CDE90223204A0693CDE91F
:10F718000431CDE907330521CDE900214FF47A7290
:10F7280002FB0BF24CF250311846D047637C13B3FE
:10F73800174B995D7B6D0D31C9B228469847E07C1F
:10F748003246494600F040FE88F8006001200BB0C0
:10F75800BDE8F08F002101250823CDE90013CDE98C
:10F768000715CDE90511CDE903110292A1782B46C1
:10F778005A462846D9E7074BDBE70020E7E700BFF2
:10F788000C46010820260020CF3F010885450100CE
:10F79800EF3F0108DF3F01082DE9F04F8DB090F9E8
:10F7A8000130DFF8F8A0DFF8F890CDE90A123D4AF9
:10F7B800017812F903B0DAF800203B4B0C2505FB61
:10F7C80001221B68527A182101FB0233044693F97F
:10F7D800021090F9020000F0E0FD3449064694F961
:10F7E800010000F0DFFDA26861688046304600F045
:10F7F80006FD2178DAF80020D9F80C30694307466D
:10F8080050589847D9F81C309C4694F90130002587
:10F81800072B4FF47A63CDE90753CDE905552DD170
:10F828000123CDE903530523CDE901534FF47A733E
:10F8380003FB0BF300933946434646F2A8122846C9
:10F848006746B8472378DAF800200C214B4394F92F
:10F858000110D05800F0DAFDA18994F90100FFF7F2
:10F8680053FD0B9B217B1860D9F8543028469847E4
:10F878000A9B01201E700DB0BDE8F08F01200823FF
:10F88800CDE90350CDE901032A46CDF800B065461D
:10F8980043463946A84701200546D3E720260020DD
:10F8A8000C460108CF3F01081C260020A83F01088C
:10F8B8002DE9F04F8FB0002405468A4691469846B8
:10F8C8000494ADF81440ADF8024007264FF0010B40
:10F8D8002B7AA34206D9686804A9204400F0F4FBF7
:10F8E80000285DD102238DF8083002A86B7A8DF8C4
:10F8F8000A30FFF733FDAB7A8DF81D309DF81130D3
:10F908008DF81E309DF812308DF81F309DF810309C
:10F918008DF82030EB7A8DF821302B7B8DF8223052
:10F928006B7B8DF8233010238DF81C608DF8243004
:10F938003A4E8DF82C000DF102030A930723326822
:10F948008DF82D30ADF834302B680C9206930DF1FC
:10F95800120204AB0DF1110106A800F0CFFB072835
:10F9680005460BD130680C22002100F5906001F0AB
:10F97800C1FB3368BDF80220A3F880249DF811303C
:10F988008AF800309DF8123089F800309DF8103060
:10F9980088F80030189B28461C700FB0BDE8F08F1F
:10F9A8009DF81330BDF81470ADF802702044C4B24D
:10F9B800F3B917B3194A00201168072602464FF019
:10F9C8000C0C062B1BD10CFB00FE51F80EE0BEF10F
:10F9D800000F04D00BFA00F23A4397B2012201302B
:10F9E8001028EED1002A3FF473AFADF802706FE72C
:10F9F8005A1E042A01D9062BDCD0062668E747FAE6
:10FA080000FE1EF0010FEAD00CFB00FE51F80EE0DC
:10FA1800BEF1000F08BF0626E1E700BF2026002040
:10FA280038B505464068FFF75BFC0722841D0021B6
:10FA380095F90000E4B200F0E6F908B904F0FD0415
:10FA480095F901000722002100F0DDF908B904F05A
:10FA5800FB04204638BD00207047000010B503782D
:10FA68000F2B044618D84068FFF73AFC22780B4958
:10FA780002EB42020968831C01EB820051F8222044
:10FA8800DBB21AB903F0FD0358B210BD032B06BF51
:10FA9800626842600223F7E70020F6E7202600208C
:10FAA800022070472DE9F0413A4D0446286896B087
:10FAB8000E46904600211F460122032300F5906060
:10FAC800CDE90411CDE906118DF80C108DF80D1053
:10FAD800ADF80E3000F0B9F930B92A68B2F88034C0
:10FAE80043F00303A2F880342A68637A8DF8203043
:10FAF80002F59061CDE90912274A94F90830126895
:10FB08000B921022ADF830200DF10E020D922268F2
:10FB18000E9262680F92D4E90301A27A8DF8402010
:10FB280001228DF8412011AA82E80300227DE18A92
:10FB38008DF8213018468DF84C20FFF7E5FB08AB0F
:10FB480015930DF10D0314900093CDF8048003ABC9
:10FB580004AA39460EA800F0C1FB044678B99DF8FE
:10FB68000C10013901F096FA00F158030DEB03006F
:10FB780010F8483C3370204616B0BDE8F0810C28D8
:10FB880001BF2A68B2F8803443F00303A2F8803436
:10FB9800F1E700BF202600201C260020F8B50679D2
:10FBA800012E054601D80620F8BD0F2E2BD8036874
:10FBB800187A40F303000722002140B200F023F92D
:10FBC8002B680446187A40F303100722002140B23C
:10FBD80000F019F9A8B1B4FA84F4640929680B7A19
:10FBE800086843F3030243F3031352B25BB29A4229
:10FBF800C8BF0124FFF774FB48B9002CD3D10420F7
:10FC0800D2E70124EAE70320CEE70520CCE7002C61
:10FC1800FBD10C4F29683B6806EB460003EB8000DC
:10FC28000C2201F053FA3A680C2303FB0623204602
:10FC38005C72B2F880140123B3400B43A2F88034FD
:10FC4800B2E700BF2026002010B4017801290ED9A0
:10FC5800084B18680C234B43C4180022C250C4E94F
:10FC6800012200F5906010BC102200F0D5B80020E9
:10FC780010BC7047202600202DE9F04186B05023A3
:10FC88008DF814300379102B074630D10368DD7BDB
:10FC98006DBB0224A8466426062C14D83A68535D26
:10FCA80003932A44517843EA01230393927843EA61
:10FCB80002437343CDE9033863B968468DF80040C1
:10FCC800FFF7C2FF0DE0CDF80C808DF81480CDF859
:10FCD8001080F2E703AB01A801938DF80840FFF705
:10FCE8005DFF0134E4B2102C05F10305D4D106B050
:10FCF800BDE8F0811FB502680379116851B901A800
:10FD08008DF80430FFF7A0FF78B9002040B205B0A5
:10FD18005DF804FB02A802928DF80C30FFF73EFF55
:10FD28000628F2D8024B185CF0E70320EEE700BF84
:10FD3800C83F010870B5114E01783268104B0C2588
:10FD480005FB01221B68527A182101FB0233044685
:10FD580093F9021090F9020000F01FFB2378326833
:10FD680061686B43D558A26800F049FA054BA2892F
:10FD7800DB6B01462846BDE8704018472026002066
:10FD88001C2600200C460108074B9B56C91A431E27
:10FD98005842584140008842B8BF08460528A8BFC5
:10FDA8000520C0B2704700BFD73F0108F0B59A429E
:10FDB800069D03DB9DF914309A4220DD0020F0BD3A
:10FDC80003EB430331F814C005EB830300264CFA18
:10FDD80006F7FF0707D51F7A07F00F0E724502DBFB
:10FDE800B2EB171F0DDD0136102E03F10C03EED117
:10FDF8000134E4B22301DBB29842E1D8DEE7002403
:10FE0800F8E70120DBE7884204DB9042CCBF002002
:10FE1800012070470020704710B51409B4EB111F7A
:10FE280003464FEA11100ED391420CD202B201F0F0
:10FE38000F0133F81240012000FA01F124EA010110
:10FE480023F8121010BD0020FCE7F0B528B100EB34
:10FE5800410501270020914200D3F0BD002435F868
:10FE680002CB234607FA04F636EA0C0608BF01332C
:10FE780004F1010408BFDBB2102CF3D1184401319E
:10FE8800C0B2C9B2E7E710B500B149B910BD31F841
:10FE9800134020F813400133DCB2A242F7D8F5E74B
:10FEA8000023F9E782B030B5048804936AB9B3F542
:10FEB800616F18D349F6AF2542F21072AB4298BF72
:10FEC8004FF47A72944238BF1446012C38BF01248B
:10FED8006143BDE83040C3688B428CBF5B1A002386
:10FEE800C36002B070476422ECE700002DE9F04FD0
:10FEF80091B01546DDF86C8004939DF8683009933D
:10FF08000C46064603F0C2FB684ADFF8A4B1059028
:10FF1800A8F5F633303BB3FBF2F3534303F5F6325F
:10FF280003F5A83303F5C0730393182313FB0543A4
:10FF380030320692089300254FF0FF3A089BA342FF
:10FF480007D1002D14BF50464FF0FF3011B0BDE867
:10FF5800F08FBDF97030ADF82C300B99CDF86C806E
:10FF68004046CDF8288003F021FBB4F800906EB924
:10FF7800B8F5616F5BD349F6AF2242F21073904532
:10FF880098BF4FF47A73994538BF99464B46012B71
:10FF980038BF01230793002E52D1B9F1640F48D11D
:10FFA800A0605F46A1680EA803F022FB0F9B009398
:10FFB800DDE90A120E9B0CA803F079FA049B0C9A4F
:10FFC8000BB9099B2BB12369BB4202D1394B9A4229
:10FFD8000DD9394BE760984509D90023ADF834307D
:10FFE800069B0D990C93184603F0E0FAA060606830
:08FFF80000B9E760276126B1A2
:020000040801F1
:1000000003F052FBE3680344E360D4E90332934214
:10001000059B1D996360079B88BFE2604B43E168C5
:10002000994202D20498A8B9A6B101231D442375B0
:10003000EDB2183486E76423A9E7B9F57A7F0ABFE1
:10004000204F214FA060B1E7049B0BB9C4F80CB05E
:100050005F46D0E700209342207506D85B1A9A4588
:1000600005F1010528BF9A46EDB2002EE1D1B9F1A4
:10007000640F164AADF8346019D049F6B023B9F5CB
:100080007A7F18BF1346904584BF039A9B180C9340
:100090001C9B00930CAF97E806001B9B384603F0AF
:1000A0000AFA97E8030003F085FA8246C1E74FF4A5
:1000B0006163E8E78051010040771B007F51010038
:1000C0002FEC010080A81201002E930230EC0100F9
:1000D0000378032B14D1437803F00F021B098A70B5
:1000E0004B7083788B80C27843EA02238B8003793C
:1000F000C3F3021203F00F03CA700B7005207047A0
:10010000002070472DE9F34798464379057990F927
:1001100007609146044690F906208A4683B190F91B
:10012000087075B30F2A12D194F909200F2E1ED131
:1001300094F90A60072D24D1002F08BF012720E081
:1001400090F90B7090F9092090F90A60E9E7A3692A
:10015000019394F915300093216994F91430207BB0
:10016000FFF728FE0028E1D105F0FD05DEE794F950
:100170001D30B3420FDC94F91C30B342DADA05F0DB
:10018000FB0528468AF8002089F8006088F800708E
:1001900002B0BDE8F0871E46CCE70000024B03FA30
:1001A00000F0B0FBF1F0704740420F004FF4FA53FB
:1001B000B3FBF0F0704730B54FF47A750C1F6A430B
:1001C00000FB042252001EBF00F1FF341219B2FBE3
:1001D000F0F2914238BF1146039A11608200484301
:1001E0001CBF013040084FF47A71121A01FB13232F
:1001F000002BCABF03F2E73393FBF1F1B3FBF1F13C
:10020000049B196030BD38B5400014460D46F1F727
:1002100001FC01462846F1F74BFB2146F1F748FB6C
:10022000F1F73AFA03F0D8FCF1F716FB40B238BD0B
:100230002DE9F74F019300231F469C461C01058AB8
:100240005FFA84FE04F0F004A54206D8019B82F810
:1002500000C01F7003B0BDE8F08F0EEB4E054FEAF3
:100260004309AD000024466836F809602641F607C8
:1002700027D5866806EB050A765916B3067836B98F
:10028000466926B136F809602641F60719D59AF86D
:10029000086090F901B046F303084FFA88F8D84592
:1002A0000FDC46F3031676B25E450ADB9AF8096066
:1002B00006EB4608C66806EBC806367D4EB9013720
:1002C000FFB20134102C05F10C05CCD10133DBB2A7
:1002D000B4E70CF101060EEB040801F80C805FFA9C
:1002E00086FCEEE72DE9FF4704464068DDE90C6730
:1002F0001D468A46914603F0D7F923681B1A3B60D6
:100300004FF000080123337085F80080636813B153
:100310002368834224D8CAF80080D4F81CC0A3699B
:100320009CF800E00393D4E9030101AB83E80300E8
:10033000237D0093DCF80C10237A627A7046FFF775
:10034000D9FD334638602A46E0694946FFF770FF19
:100350002B782BB1C7F80080002004B0BDE8F087EF
:100360003378002B14BF0B200C20F6E737B590F93B
:10037000002090F90250954204460FD0013A52B243
:1003800095420BD0A368019394F901300093616802
:10039000E0782B46FFF70EFD0028EFD0104603B0A3
:1003A00030BD8842B8BF08467047000051F82000B1
:1003B000054B984205D0054BC31A5842584140009E
:1003C00070470120704700BF90D0030020A10700B4
:1003D00005281FB50ED80C4B53F820300093CDE9FB
:1003E00001120A4B01220021022002F069FE05B031
:1003F0005DF804FBCDE90012054B0122002102202B
:1004000002F05EFEF3E700BF64400108F73F010819
:100410001640010807B5054BCDE900010122002176
:10042000022002F04DFE03B05DF804FB32400108EB
:1004300010B5102204460021F13000F05FFE0021CB
:10044000C4F814112046F022BDE8104000F056BE5A
:1004500002460846102100F0A5B92DE9F0430446F4
:10046000D0F8140185B00E46154604F2011988B380
:10047000C0F110089045474628BF1746BAB2484415
:1004800000F028FED4F814313B440F2BC4F814318B
:100490002DD9A8452BD204F1F00304F5807113F88F
:1004A000012F187C8B4282EA00021A70F7D104F106
:1004B000F10810224146684600F00CFE22466946CB
:1004C000684600F0E9F910226946404600F002FE55
:1004D0003E44ED1B04F5807804F1F107102D09D896
:1004E000AAB23146484600F0F5FDC4F8145105B0F3
:1004F000BDE8F08304F1F003711E13F8012F11F829
:10050000010F434582EA00021A70F6D110223946E3
:10051000684600F0DFFD22466946684600F0BCF9F7
:1005200010226946384600F0D5FD1036103DD5E75B
:10053000F0B589B00C46102200210546684600F04F
:10054000DDFD22466946684600F0A6F99DF90030B7
:10055000002B6A464FF0000143DA137812F8010FBE
:1005600001315B0043EAD0130F2902F8013CF4D1BA
:100570009DF80F305B0083F08703D4F81401DBB2E1
:1005800010288DF80F303BD104F58073694604F5CF
:10059000887013F8016F11F8012B984282EA060265
:1005A0001A70F6D104F1F00304F5807113F8012FED
:1005B000187C8B4282EA00021A70F7D110220DEBF0
:1005C000020004F1F10100F085FD2246294604A84D
:1005D00000F062F910220021684600F08FFD09B09A
:1005E000F0BD137812F8010F01315B0043EAD0131C
:1005F0000F2902F8013CF4D19DF80F305B00BCE7F5
:100600009DF90030002B6A464FF0000137DA13786D
:1006100012F8016F01315B0043EAD6130F2902F88B
:10062000013CF4D19DF80F305B0083F08703471C39
:10063000DBB28DF80F30102F04EB0003C0F10F0672
:100640004FF0800288BF002600F5817083F80121F9
:100650000021324620443E4403F072FAC4F814618B
:1006600004F58073694604F5887013F8016F11F87A
:10067000012B984282EA06021A70F6D192E71378AB
:1006800012F8016F01315B0043EAD6130F2902F81B
:10069000013CF4D19DF80F305B00C8E70A7803787D
:1006A000534003704A784378534043708A78837884
:1006B00053408370CA78C3785340C3700A79037972
:1006C000534003714A794379534043718A7983795E
:1006D00053408371CA79C3795340C3710A7A037A4C
:1006E000534003724A7A437A534043728A7A837A38
:1006F00053408372CA7AC37A5340C3720A7B037B26
:10070000534003734A7B437B534043738A7B837B11
:1007100053408373CA7BC37B5340C373704710B588
:100720000B7814786340037054784B7863404370BF
:1007300094788B7863408370D478CB786340C370AF
:1007400014790B796340037154794B796340437199
:1007500094798B7963408371D479CB796340C37189
:10076000147A0B7A63400372547A4B7A6340437273
:100770008B7A947A63408372D47ACB7A6340C37263
:10078000147B0B7B63400373547B4B7B634043734D
:10079000947B8B7B63408373CB7BD27B5340C3734F
:1007A00010BD0000A1F11003DBB2102B2DE9F047C2
:1007B00004D8374C24FA03F3DB0705D4002382F86E
:1007C000F030FF20BDE8F087531E4418A0424ED100
:1007D00001F11C039B005FFA83F9C3F30313013B90
:1007E0002C4D82F8F03001240B46D618B3FBF1F003
:1007F00001FB103010F0FF0016F804AC16F803EC03
:1008000016F802CC16F8017C36D115F80E8015F8D2
:100810000CE015F807C015F80A70E00900EB40007D
:1008200084EA080800EBC0006400C0B2E4B24440AF
:10083000C246581AC0B212F800808AEA080A02F8C2
:1008400003A01044043390F801808EEA080E86F865
:1008500001E090F802E08CEA0E0C86F802C0C07845
:10086000DBB247409945F770BFD80020AAE710F8DF
:10087000015B03F8015FA9E71829DAD9102801BF45
:1008800015F80AA015F80EE015F80CC0EF5DD0E7DA
:10089000010101007C4201082DE9F04FA3B092F85C
:1008A000F0301D911B920193002B00F05381014603
:1008B0001EA8FFF734FF1B9BA74CA84DA84E103372
:1008C0000293002303939DF87C0004909DF886001A
:1008D0000590205C06909DF87B000790205C0890B6
:1008E00004989DF881C0205C099014F80C000A90CF
:1008F0009DF880000B909DF885009DF878809DF80C
:100900007DE09DF882A09DF887900C909DF87A007C
:10091000029B1C9314F80A2014F8093014F80810EC
:1009200014F80E700D90205C0E909DF87F000F90D3
:10093000205C10900B98205C11900C98205C129019
:100940009DF8840013909DF8790014909DF87E0026
:100950001590205C16909DF883001790205C1890ED
:100960001398205C19901498205C1A900398013019
:1009700003900298DDF804B0103002909DF80C004E
:10098000834536D88DF878108DF87A2009990E9A1B
:100990008DF87C108DF882201199069A8DF88010C0
:1009A0008DF87E201999169A8DF884108DF886207E
:1009B0000A99189A8DF87D108DF887201299109A4F
:1009C0008DF87B301B9B8DF881108DF883201A9950
:1009D000089A1D988DF885108DF87F201EA903EBCD
:1009E0000B128DF87970FFF79AFE002023B0BDE856
:1009F000F08F15F808B082EA03008BEA000016F8C1
:100A00000EB080EA0B008DF8780015F80E004B4010
:100A1000434016F80A0043408DF8793081EA070315
:100A200015F80A10594016F80930594016F80830E0
:100A30008DF87A107A40534015F8092053408DF80C
:100A40007B30089A069B5340049AAA5C534016F8E0
:100A50000C2053408DF87C30DDE908325A4015F8FF
:100A60000C305340059AB25C53408DF87D30DDE97F
:100A700009325A40059BEB5C5340079AB25C5340E5
:100A80008DF87E30069B0A9A5340049AB25C5A4015
:100A9000079BEB5C5A408DF87F200E9B109A5340C9
:100AA0000B9AAA5C53400C9AB25C53408DF880308C
:100AB000DDE910325A400C9BEB5C53400D9AB25C5E
:100AC00053408DF88130DDE911325A400D9BEB5CCB
:100AD00053400F9AB25C53408DF88230129A0E9BAD
:100AE00053400B9AB25C5A400F9BEB5C1C995A40E6
:100AF0008DF88320169B189A5340139AAA5C534092
:100B0000149AB25C53408DF88430DDE918325A40B3
:100B1000149BEB5C5340159AB25C53408DF88530C2
:100B2000DDE919325A40159BEB5C5340179AB25CD1
:100B300053408DF886301A9A169B5340139AB25C34
:100B40005340179AAA5C1EA853408DF88730FFF7D0
:100B5000A5FDB8E6FF2049E77C4201087C4001087A
:100B60007C41010808B538B1044A05491060D82213
:100B700000F0B0FA002008BD0220FCE72426002087
:100B8000AC4701080A4B1A6870B5002302F118053A
:100B900003EB03142E5D864204D1183422440A600C
:100BA000002070BD01330B2BF2D10320F9E700BF09
:100BB000242600202DE9F041CCB00646DDF848811E
:100BC00017461C460D4631B3B8F1000F23D006A8D6
:100BD000FFF72EFC204601A9FFF7D4FF0446B0B969
:100BE000019906A80131FFF733FC26B110223146E6
:100BF00006A8FFF732FC3A46294606A8FFF72DFC67
:100C000006A902A8FFF794FC029BC8F80030204612
:100C10004CB0BDE8F0810224F9E7000030B595B092
:100C200013A90446FFF7AEFF002830D11B490C235F
:100C300003FB00F2555CA5422BD1139B187C10904E
:100C4000D87B0F90987B0E90587B0D90187B0C9062
:100C5000D87A0B90987A0A90587A0990187A089066
:100C6000D87907909879069058790590187904906A
:100C7000D8780390987802900A445B78019393683F
:100C800000930022064B1146022002F019FA15B01B
:100C900030BD01300B28CBD1F9E700BFF444010887
:100CA0007C4301080B2B10B402D810BCFFF782BFA5
:100CB000032010BC704730B50D4685B01446014680
:100CC00068B103AA002000922A460390FFF772FF42
:100CD00018B90398001B18BF012005B030BD0220D1
:100CE000FBE72DE9F0430D46BFB014469946804618
:100CF00020B31BB311F00F0122D1F02201A800F0A4
:100D0000FDF920466946FFF73DFF044648B90098C3
:100D100001AA10210130FFF745FD2E46AF1BFFB29F
:100D20001EB920463FB0BDE8F08301AA09EB0701D8
:100D300008EB0700FFF7B0FD103EEFE70224F0E7F5
:100D40000524EEE7F0B5184E3468024685B0084633
:100D5000002304F1180103EB03154F5D97421ED1E8
:100D60000D2A05F1190513D10023CDE90033CDE992
:100D700002330C2210216B46FFF7B3FF04463068A4
:100D800010226946284400F0A5F9204605B0F0BDC0
:100D900001461022601900F09DF90024F5E70133A7
:100DA0000B2BD8D10324F0E72426002009B1FFF74C
:100DB000C9BF022070471FB51446A0B10C2A01D14B
:100DC0000B2912D10023CDE90033CDE902330A46C5
:100DD0006B461021FFF785FF18B969462046FFF7DB
:100DE000B1FF04B010BD0220FBE70320F9E7F8B51E
:100DF0001E46DDE907479DF818505BB354B34FB367
:100E0000212D29D819462A46204600F063F90122EF
:100E1000631C691EB018FFF764FFF8B9E37ADB09B9
:100E20003B70EBB96319204613F8012C13F8021C30
:100E3000120642EA014213F8041C0A4313F8031C89
:100E4000012342EA0122291FFFF735FF003818BFAE
:100E50000120F8BD0220FCE70520FAE70720F8E7AB
:100E60000420F6E710B5044628B1044B5B699847A7
:100E70002060002010BD0220FCE700BF0C460108E6
:100E800008B5014630B1044B0822186800F022F979
:100E9000002008BD0220FCE72426002008B530B160
:100EA000044B0822196800F015F9002008BD022043
:100EB000FCE700BF242600207FB5124E0023044625
:100EC00002A801930D46FFF7E9FF33685B690193C0
:100ED0006CB102AA082312F8011B41B9013B13F0BF
:100EE000FF03F8D102A8A04702A8FFF7C9FF35B158
:100EF000019B23B901A8A8473368019A5A610020D1
:100F000004B070BD2426002008B5014638B1054B59
:100F100018680822104400F0DDF8002008BD022007
:100F2000FCE700BF2426002008B538B1044B19683F
:100F30000822114400F0CEF8002008BD0220FCE792
:100F400024260020034B1B6802280CBF196159613D
:100F5000002070472426002041B1054B1B68022861
:100F60000CBF1B695B690B60002070470220704753
:100F70002426002030B58FB0002405460CA8099423
:100F8000FFF78CFF9DF8373007939DF836300693B6
:100F90009DF8353005939DF8343004939DF8333037
:100FA00003939DF8323002939DF8313001939DF800
:100FB00030300093224621461E4B022002F080F87A
:100FC0000AA8FFF7B1FF9DF82F3007939DF82E3048
:100FD00006939DF82D3005939DF82C3004939DF8D1
:100FE0002B3003939DF82A3002939DF8293001930A
:100FF0009DF82830009322460F4B2146022002F034
:101000005FF809A92846FFF7A7FF9DF8243003934E
:101010009DF8253002939DF8263001939DF82730E6
:1010200000932246054B2146022002F049F80FB0FA
:1010300030BD00BFD84301081644010854440108DC
:1010400008B50020FFF7EAFD0120FFF7E7FD0920C2
:10105000FFF7E4FD0820FFF7E1FD0020FFF78AFF1E
:10106000002008BD10B504460B20FFF7D7FD0C206B
:10107000FFF7D4FD0920FFF7D1FD0820FFF7CEFDD3
:101080000A20FFF7CBFD2046FFF774FF002010BDBC
:10109000014B1860704700BFBC0800200B4A30B5F8
:1010A00014680B4D43F2390305FB04331360091A2E
:1010B0006FF00042B3FBF2F2C2EBC27201319B1A35
:1010C00093FBF1F201FB1233184430BDBC08002041
:1010D0006D4EC64101380A44914200D1704711F863
:1010E000013B00F8013FF7E710440A44914200D168
:1010F000704711F8013B00F8013DF7E702F020BD11
:1011000030B530B10A4D01444FF0FF33814201D177
:10111000D84330BD10F8012B5340082243F300049C
:10112000013A2C4092B284EA5303002AF6D1EDE74B
:101130002083B8ED01207047054B4FF400529A62AE
:10114000044B1B6813B15B6803B11847704700BFBD
:101150000004004828270020054B4FF480529A6273
:10116000044B1B6813B1DB6803B11847704700BF1D
:101170000004004828270020012070470120704704
:1011800001F048B901F036B910B501F019FE0E2191
:10119000044640F61F1001F02DF92046012101F010
:1011A000F9FDBDE8104001F0D7BA000070B50C4E53
:1011B00001EB40030D46B3654FF6FF710023044673
:1011C0001A46084601F05EFB96F85600002101F031
:1011D000E1FD29462046BDE8704001F095BA00BF08
:1011E0004427002010B5044601F0AAFE01281CD1B6
:1011F00001F0AEFE34B11248214602F017FB104850
:1012000002F0DAFA0F4C104B00214FF48052A16526
:101210009A6194F8560001F0BDFD63786BB16FF0F0
:101220007F40BDE8104001F053BA002340F2622134
:101230001A46084601F026FBDCE7A0688001F0E7CB
:101240002C2700204427002000040048002001F043
:10125000BFB9000008B501F0C7F80438C0B20328D0
:1012600096BF024B0020185C08BD00BF084601086D
:1012700008B501F0BAFD033008BD01F049B901F02D
:1012800009B908B501F000FD00B208BD38B50D463A
:10129000144601F05DFB284601F092FD0E21054643
:1012A00040F61F1001F0A6F828460121074D01F075
:1012B00071FD01F051FA4FF47A716143284602F052
:1012C000B5FA2846BDE8384002F076BAA0270020DB
:1012D00001F03EBB08B5084B002193F8560001F021
:1012E00059FD00234FF4C0711A46084601F0CAFAAE
:1012F000BDE8084001F024BA4427002010B5044698
:1013000001F01EFE01281CD101F022FE34B112486A
:10131000214602F08BFA104802F04EFA0F4C104BA7
:1013200000214FF48052A1659A6194F8560001F0B3
:1013300031FD63786BB16FF07F40BDE8104001F084
:101340007DB9002340F262211A46084601F09AFA5C
:10135000DCE7A0688001F0E72C270020442700206C
:101360000004004808B54FF0040001F017F9BDE88B
:1013700008400220F1F7C4BB08B500231A461946FD
:10138000184601F07FFABDE8084001F06DB9000091
:101390001D4B73B51D4D186000241D486C70C5E9C8
:1013A0000144AC6501F098FAAC8101F003FA2146E2
:1013B000204601F04BFC21460422012001F0FCFAFA
:1013C000144E154D4FF6FF7123462246084601F094
:1013D00059FAFFF7C7FF2246104B00944FF0FF3138
:1013E000304602F03DF90E4B009422464FF0FF319B
:1013F000284602F035F9304602F090F9284602B04E
:10140000BDE8704002F08AB9282700204427002058
:10141000D9230108A02700202C270020391101081A
:10142000591101080128084805D1084BC1771970E6
:101430000E3001F0A7BB437D012B03D1034B817517
:101440001970F5E7704700BF44270020C00800204E
:101450000D4B10B5044618735873012000F016F8B0
:101460005CB134214FF4E86000F0C4FF4421BDE8D2
:10147000104040F2417000F0BDBF14214FF4E8600D
:1014800000F0B8FF2421F2E74427002038B5114CC2
:101490000546207001F061FD052D04D8DFE805F058
:1014A000090B03171709032001F070FA0023637377
:1014B00038BD0020F8E7012001F068FA207B637B4B
:1014C0008342F5D06073BDE83840FFF7C1BF02200A
:1014D000EAE700BF442700202DE9F0431E4687B00D
:1014E00000230546CDE901330C46174601F027FDE0
:1014F000032D61D8DFE815F07B00C3000E01040066
:10150000A27C082A04D94FF0FF3007B0BDE8F08371
:10151000A16801A801F0DCFE21680029F3D042F2A5
:1015200010729142E37C864D51D80322AA7385F84C
:101530003820E96385F844304FF002086368A17DE4
:10154000DB002B820423AB74A37CDB00EB74022949
:101550004FF000032B75637D02D0227D022A42D119
:1015600003F10F02D2B2012A01D9012BCBD1754B65
:10157000754A196803944FF0010903A88DF8149077
:1015800001F0DAFC0028BED1287685F8179068753E
:10159000FFF75CFE4046FFF779FF6C4801F086FAE2
:1015A0006B4801F0EFFA01A800F084FF208A00F0F8
:1015B00055FFA08900F09AFF384601F001FC604C0D
:1015C00084F8560001F0C0FC666000209DE74FF0F3
:1015D0000008E963890885F80E8085F8388085F869
:1015E00044302964AAE7EB7529766A75D0E7236849
:1015F000002B88D0A27C082A85D8514DA16801A86B
:1016000001F066FE002385F838302268EA63E27C48
:1016100085F84420A269AB732A646268A17DD20078
:101620002A820422AA74A27C2B75D2000229637D2F
:10163000EA7402D0227D022A1DD103F10F02D2B238
:10164000012A02D9012B7FF45EAF3E4B3E4A196856
:1016500003944FF0010803A88DF8148001F06CFC8E
:1016600000287FF450AF287685F817806875FFF75B
:10167000EDFD00208FE7EB7529766A75F7E7304DB1
:10168000012185F83810227885F85020637885F894
:101690005130A37885F85230E3788B4202D0022B88
:1016A00003D03BB985F8533004E00B3A012A29D81E
:1016B00085F853104FF0010885F80E80A388AB839E
:1016C000A379AB77E37985F82030237A85F8213048
:1016D000FFF7BCFD4046FFF7D9FE1C4801F0E6F9D4
:1016E0001B4801F04FFA95F85130062B40F689005F
:1016F0000AD100F08FFE00F0FB0140F6890000F0F7
:1017000079FE59E70023CDE700F084FE40F00401A4
:10171000C9B2F2E72368013BB3F57A7FBFF4F3AEB9
:101720000320FFF7B3FE0648022380F83830236811
:101730008364162380F84C30383001F0B7F93BE76A
:101740004427002028270020A02700207C270020F5
:10175000522700202DE9F041002686B01F4614468E
:10176000CDE9016680460D4601F0E9FBB442764CB6
:1017700016BF0123334637466370B8F1000F06D019
:10178000B8F1010F7CD0002006B0BDE8F081AB6855
:10179000002B00F0D680EB68002B00F0D280AA7FEF
:1017A000082A00F2CE80296901A801F091FD28687D
:1017B000003818BF012000F0D9FF84F83880AB68EA
:1017C000E36395F8203084F84430686801F05AFBF0
:1017D00084F80E8084F84500EB68DB002382EB7F01
:1017E000A374AB7FDB00E37495F82130237595F883
:1017F0002230002B3ED12A7D95F82410A2750229B3
:1018000095F8232001D0022B36D102F10F03DBB271
:10181000012B02D9012A40F0948000238DF8143066
:101820004A4B4B4A1968049503A801F085FB002830
:1018300040F0878001232076E3756075FFF706FD91
:101840000020FFF723FE434801F030F9424801F041
:1018500099F901A800F02EFEA88B00F0FFFD288B5F
:1018600000F044FE4FF4FA53AA687B43B3FBF2F353
:10187000A36088E7FF22BFE7E27521766375DDE7A5
:101880002B8E002B5DD095F83230A86A012B0CBF4F
:1018900095F814804FF0FF08003818BF012000F0C1
:1018A00065FFF8B200F06EFF012184F8381095F85A
:1018B0002C2084F8502095F82D3084F8513095F87C
:1018C0002E3084F8523095F82F308B4202D0022B04
:1018D00003D03BB984F8533004E00B3A012A28D8EE
:1018E00084F853102B8EA38395F83230A377AB8EF8
:1018F00023840126A67384F81F80FFF7A7FC3046D7
:10190000FFF7C4FD134801F0D1F8134801F03AF98C
:1019100094F82130B34240F236700CD100F07AFDD9
:1019200000F0FB0140F2367000F064FD4FF6FF73EB
:101930009EE70023CEE700F06DFD40F00401C9B240
:10194000F0E74FF0FF301FE7442700202827002052
:101950002C2700207C270020522700202DE9F04F63
:1019600085B082460E9DBDF840B09DF844709DF84C
:101970004890019288461E4601F0E1FABAF1010F43
:10198000524C54D0BAF1040F00F09180BAF1000F1C
:101990003AD10B22304684F8442084F838A0E5631D
:1019A00001F070FA019B23644FEACB03B9F1000FF9
:1019B000238241F60403638214BFF2230123E375FB
:1019C00087F001070123237684F8450084F80EA0F0
:1019D00084F814A06775FFF739FC5046FFF756FDF1
:1019E00004F1380001F062F804F10E0001F0CAF8C9
:1019F000374A1068516802AB03C302A800F05AFDD1
:101A000040F2FF1000F02AFD404601F0D9F90E2106
:101A100084F8560040F61F1000F0ECFC94F85600D5
:101A200001F092FA169B636005B0BDE8F08F29497A
:101A300084F838A0EAB2895D84F8502076BB0B3D6B
:101A4000012D8CBF00250125053A012A04D8BBF1E0
:101A50000C0F38BF4FF00C0B1F4B9DF83C201B7830
:101A600084F85350E37701259DF8543084F85110E1
:101A700084F8522084F82130A573A4F81CB0A7770D
:101A800084F82090FFF7E2FB2846FFF7FFFC13489D
:101A900001F00CF8124801F075F8B5E7012E04D1F9
:101AA000A5F10C035D425D41CEE70025CCE7504631
:101AB000FFF7ECFC022384F8383004F138001623D9
:101AC000A56484F84C3000F0F1FF9DE74427002026
:101AD000143D0108D6450108C00800207C270020DD
:101AE000522700202DE9F04F87B0DFF8B4B29DF8FF
:101AF00064A09DF84C90029314469DF854309DF8D4
:101B00005020BDF84880039205468BF801A0BDF82F
:101B1000446001930F4601F012FABAF1000F18BFAA
:101B20004FF00008DFF87CA2039AB9F1000F08BF5C
:101B3000FF22012D8AF8002000F0C880052D48D032
:101B4000002D40F0C080284600F010FE0B223846E1
:101B50008BF844208BF83850CBF83C4001F092F9D8
:101B6000019B8BF8450041F60402002BABF81220D4
:101B70009AF800208BF8162014BFF22201228BF86D
:101B80001720F600012289F001098BF818208BF844
:101B90000E50ABF810608BF814508BF81590FFF7CF
:101BA00055FB2846FFF772FC0BF1380000F07EFF72
:101BB0000BF10E0000F0E6FF7B490868496804AAB3
:101BC00003C204A800F076FC40F2FF1000F046FCCF
:101BD00071E0012000F0CAFD09224FF000098BF8E6
:101BE000442038464FF44872CBF840208BF83890A8
:101BF000CBF83C4001F046F94FF48052ABF812208C
